:100000000C94DB150D94030F0D94D80E0D94AD0ECA
:100010000D94820E0D94570E0D942C0E0D94010E1E
:100020000D94D60D0C940C160C940C160C940C1606
:100030000C940C160C940C160C940C160C94D0CF3B
:100040000C940C160C940C160C940C160C940C16A8
:100050000C940C160C940C160C940C160D94410C6C
:100060000C940C160C9469BB0C943FBB0C940C16AE
:100070000C940C160C940C160C940C160C940C1678
:100080000C940C160C940C160C940C160C940C1668
:100090000C9439BD0C94AFBC0C94F1BC0C9468D199
:1000A0000C940C160C940C160C940C160C940C1648
:1000B0000C940C160C940C160C940C160C940C1638
:1000C0000C940C160C940C160C940C160C9415BB7A
:1000D0000C94EBBA0C940C160C94C1BA0C9497BA0D
:1000E0000C940C1607634236B79BD8A71A3968568A
:1000F00018AEBAAB558C1D3CB7CC5763BD6DEDFD4A
:10010000753EF6177231BF000000803F0800000006
:10011000BE922449123EABAAAA2ABECDCCCC4C3EFC
:1001200000000080BEABAAAAAA3E00000000BF00EB
:100130000000803F0000000000084178D3BB4387E7
:10014000D1133D190E3CC3BD4282AD2B3E68EC82FB
:1001500076BED98FE1A93E4C80EFFFBE01C4FF7F80
:100160003F00000000000C94E2B00C944CFC0C9496
:10017000CB470C94F03C0C94D7160C947B200C9439
:1001800083650C94CFB90D9405010C9498470C9499
:10019000037E0C9498A60C94DDDF0C94DE2F0C9457
:1001A000C1FF0C94E1AC0C94FB4E0C946ECE0C94FD
:1001B000ABA20C944E1C0C94C5770C9427C40C94E1
:1001C000A04C0C94B3220C946F170C94F06D0C940B
:1001D000CF6E0C9408E70C9494FF0C9414AE0C941E
:1001E0004BD80C94DC640C94F12F0C94C42E0C941A
:1001F000F46E0C940A6C0C9473AD0C9493170C94DD
:10020000CAFF0C94CFFF0C943CB90C944D1F0C9476
:1002100097AC0C9481C10C94EEF80C94C5A40C948A
:10022000B3FF0C9441C80C945C3D0C94E9AD0C9464
:10023000F7C60C9432170C94F5B80C947A7E0C9493
:100240001B170C9468A40C94574D0C9494650C9453
:100250007AA50C9496AD0C9468FC0C94B6C70C94DB
:1002600082AF0C94FBDE0C9468C70C94F75C0C9482
:1002700039A40C94EEA40C94614D0D947D000C9463
:100280004C160C948AFF0C949CAE0C945BE50C9479
:100290004AAC0C94B01E0C94CCB70C943D670C94F3
:1002A000E8AA0C9416F90C94E2BF0C94016E0C941D
:1002B000001D0C948BD60C9405300C94CAA60C949B
:1002C0004F3C0C9429210C947A1F0C9407F90C9440
:1002D0003DB50C9476BF0C949CFF0C943EFC0C94A2
:1002E00014D90C942BB00C9470C40C9439220C9437
:1002F000921F0C9498FF0C948BC60C94DAF40C9417
:1003000071DF0C944CF90C94D4AA0C94AFAB0C9400
:100310008AAD0C948FAB0C948F3E0C948FC60C94CA
:10032000187E0C94572A0C942F170C94BC1C0C9418
:10033000FA5C0C942DB00C940BB10C94D45B0C941F
:10034000C5FF0C944FB00C94CC210D94F1000D948A
:1003500096000C942A2F0C94B82F0C94097A0C94C4
:10036000DA4C0C94C3650C94133E0C9478650C9491
:100370004F160C94FB3C0C9487AE0C94AE330C944B
:1003800056C30C94D02D0C94C92D0C9443E70C94B7
:10039000B9A20C949F5C0C9445FC0D94F1070C944D
:1003A000A62F0C942B2A0C948B2F0C94866E0C94F5
:1003B000C51D0C94942F0C943F190C94CC820C9472
:1003C0000E160C948A200C94EB3D0C941E5D0C943C
:1003D000F93D0C94F4960C94CF220C94CF160C9407
:1003E0003E1F0C946C3C0C94FEE80C942F5C0C9417
:1003F0008B6D0C94CB160C94515C0C947FAA0C94CE
:10040000C73D0C94B17D0C94A0EC0C94176E0C9429
:10041000006D0C945E470C942A1A0C9474650C942D
:10042000DB160C94A9FF0C9437FC0C940DAE0C94C5
:100430002DC00C946D1F0C9465BF0C94C3E80C94F4
:1004400045AD0C9475650C942D3D0C9448670C9447
:10045000196E0C94462A0C94B42A0C94D5180C945A
:100460005C170C9418670C94903D0C94AACE0C94D5
:100470003A3D0C9442B10C9452690D94D4070C94FB
:100480001A4C0C94FB2F0C9475520C947B1E0C94FC
:1004900095850C9449AD0C94F1160C9460AD0C94B8
:1004A00073DF0C9486A30C94736A0C94DD9A0C94FD
:1004B00070200C94F6790C944D4D0D94FB000C9427
:1004C000693C0C94DCE80C94583E0C945D2D0C9423
:1004D000113D0C94031D0C94C1AE0C9444B60C94C5
:1004E000DB4B0C9446C40C946BA50C94283E0C94E6
:1004F000A1E90C949D2F0C94B7830C94CF1C0C9401
:10050000EBAE0C9477210C94BDFF0C944D210C9410
:100510008E740C94C5950C94183E0C94F4BF0C94F6
:10052000F51C0C94E5AE0C94343C0C943D1E0C94DC
:1005300025B00C9407410C9486170C94C4AE0C940F
:10054000E67C0C94346E0C9449D70C94A81C0C9443
:10055000F5F80C94D5170C946EC30C948B840C9402
:10056000F94E0C94EAAD0C940FC80C949FFF0C94B8
:10057000AFFF0C9416670C94735B0C940F1D0C94D6
:1005800094A70C94D77D0C941D820D946A170C943B
:10059000156E0C942FAD0C9467B00C94DBF40C9496
:1005A00071180D94F4070D94DD000C94A7A70C941A
:1005B000DFA60C9459AD0C9474AD0C94CFAC0C9494
:1005C00076AC0C94BC2E0C94741F0C94AAAE0C94B4
:1005D000DE6E0C9447A40C9441AE0C94B62E0D9490
:1005E0000F010C9465210C9429B00C9473A30C9406
:1005F000D13D0C942D170C94D79A0C9498220C94FE
:10060000D7170C9423320C940B190D9482000C9480
:1006100033A40C94662D0C94E61C0C9422E70C94E5
:100620007B520C94CBFF0C9494AD0C94E0A40C94EE
:100630009A650C942FA90C943C850C94A27A0D9485
:10064000CE000C9459AC0C94FF4E0D94A8000C9461
:10065000602D0C94AD1E0C941C820C94293E0C94BD
:1006600021B00C94B1C30C94C4E60C946BAD0C9403
:10067000EF460C9490FF0C946A5C0C94382A0C940E
:10068000859D0C94C5AA0D94BA000C94BE460C949A
:10069000ECB80C942D9D0C944D7E0C94CF650D946C
:1006A000A0000C94EA7A0C94073E0C9465200C94FC
:1006B0008D2A0C94A5790C942E2B0C943C3D0C9413
:1006C00011170C94823C0C947FBF0C9407300C944F
:1006D000E8AC0C94654C0C9474DF0C94BF2E0C9415
:1006E000B7FF0C94C7160D9474170D94B0000C94BA
:1006F000A5AC0C9427B00C94B8B40C94E8AE0C9450
:10070000E3790C94245B0C941BAD0C9496BF0C9471
:1007100069CB0C94CB2F0C94D3160D94C4000C947D
:10072000132B0C94A75B0C94A96D0C94C9730C94B7
:10073000A63D0C94CEE90C9438760C9435F90C94C3
:100740002F7E0C9417AD0C942F1F0C949F2A0D94A0
:10075000E7000C94ED5B0C9431E70C94EB660C9481
:10076000261F0C9472DF0C9461FC0C94111C0C94E9
:10077000BF2A0C94553E0D9475000C94F6AA0C9467
:10078000F94C0C945E190C94FAEF0C945A5B0C948F
:10079000F21C0C94486D0C94116E0C94A5FF0C94F3
:1007A000D2B10C94172A0C94754D0C940A1E0C941B
:1007B00049B90C94946E0C94EE5A0C94EF7D0C9401
:1007C00074E90C946EB10C946C520C94EBAD0C94D7
:1007D00053650C94CC6D0C9462B50C9423B00C94BE
:1007E000FCB00C94D9C70C9449220C9464E80C9486
:1007F00052160C94B1330C945AFC0C94736B0C94F9
:10080000B92E0C94FD5C0C94EEAE0C94E4F70C94B1
:10081000FAAD0C942CDF0C94379D0C9491200C9421
:100820001ECF0C9429170C948FB80C9414670C9459
:1008300096D80C94361E0C94AF3E0C94134D0C9429
:100840002F2C0C94461F0C9449170C942FB00C9429
:10085000831F0C94666D0C94DF160C94F6CA0C94EE
:1008600023A10C948E7D0C9485170C9412670C9424
:1008700081C70C947A780C948E650C942D4D0C9451
:1008800042AB0D948C000C949FB70C946C3D0D946E
:10089000D5070C9455160C947C6E4E414E494E492A
:1008A0005459494E46CDCCCC3D0AD7233C17B7D13D
:1008B0003877CC2B329595E6241FB14F0A000020E3
:1008C000410000C84200401C4620BCBE4CCA1B0E62
:1008D0005AAEC59D746364696E6F70737578585BAA
:1008E00000556E6B6E6F776E207375666669782043
:1008F00000556E6B6E6F776E20636D642000636CC5
:10090000724374723A2000454F46002F00496E3AF8
:1009100020003D00494E3A003D004C4547414359B7
:1009200020494E3A002500C2B04320483D002044F3
:100930004854323220747970652E20543D00494E5F
:100940003A00204E6F20656D6974206461746121E6
:100950000020436F756E74657220747970652E2067
:1009600076616C3D00494E3A0020436F756E7465A8
:100970007220747970652E20494E434F5252454380
:100980005420496E74657272757074206E756D6254
:100990006572212121004952513A002D3E0020006C
:1009A00023002D3E00200050656E6465643A2023CC
:1009B000007261770076616C0074656D7000736120
:1009C00074006875650066616E00524742004853C6
:1009D00056006D6F646500536574436D643A00534F
:1009E000746F726564204558543A00737566666981
:1009F00078436F64653A0020666F7220286D732912
:100A00003A004354524C3A205363686564756C65F0
:100A100020636D642000206D73203A0041726D6583
:100A20006420666F7220002044697361726D656492
:100A300000584F4E0048414C54002074696D653A8F
:100A4000004354524C3A205265733A002054533AB2
:100A50000020543A003D0050696E3A004354524C15
:100A60003A20436F6D6D616E6420626C6F636B65DD
:100A70006420627920647269766572206F722063E7
:100A800068616E6E656C2066726F7A656E004354A5
:100A9000524C3A204F4E3A416C7265616479204164
:100AA00063746976650A004354524C3A2048414CBD
:100AB000543A416C726561647920496E616374696E
:100AC00076650A004354524C3A20584F4E3A20441F
:100AD000697361626C65640A004354524C3A205851
:100AE0004F4E3A416C726561647920416374697656
:100AF000650A004354524C3A20584F464620736BC7
:100B000069707065642E205072657620636D643A5A
:100B1000004354524C3A205475726E6564206F66DF
:100B2000662066726F6D3A004354524C3A2052650B
:100B300073746F7265642066726F6D3A004354522D
:100B40004C3A2049676E6F7265642C206368616E51
:100B50006E656C20636D643D0020457865633A00E6
:100B60004354524C3A204163746976653A004354C9
:100B7000524C3A2048414C543A416C726561647958
:100B800020496E6163746976650A004354524C3A99
:100B900020584F4E3A2044697361626C65640A00C4
:100BA0004354524C3A20584F4E3A416C726561643E
:100BB00079204163746976650A004354524C3A20A7
:100BC000584F464620736B69707065642E205072D2
:100BD000657620636D643A004354524C3A20547554
:100BE000726E6564206F66662066726F6D3A0043B0
:100BF00054524C3A20526573746F72656420667269
:100C00006F6D3A004354524C3A204E6F7420656E1B
:100C10006F756768206D656D6F727920666F7220E1
:100C200067726F7570206F7065726174696F6E00A6
:100C3000496E76616C69642061726700496E766105
:100C40006C696420617267004354524C3A20556EBF
:100C50006B6E6F776E2073756666697800536B698B
:100C60007070656420686F6D696520737475666661
:100C7000002000205375623D00204974656D3D00E1
:100C80004354524C3A2052414D3D004354524C3A49
:100C9000204F75744F664D656D6F72793A2000284C
:100CA0002D292000282B2920002076616C756520D5
:100CB0006973200020756E6B6E6F776E0A005D3D64
:100CC000005B0020696E76616C6964002000206F13
:100CD0006B003A00206661696C6564003A005265F9
:100CE000747279696E6720564354454D5020434DC8
:100CF000440A005265747279696E67205643204336
:100D00004D440A005265747279696E67206D6F6494
:100D100062757320434D440A005265747279696E9E
:100D20006720434D440A00206572726F723D004D8A
:100D3000423A20706F6C6C696E6720002056616CBF
:100D40003A20004D423A20004D423A204E6F742026
:100D5000737570706F727465642072656720747942
:100D600070650A004D423A20706F6C6C696E6720A6
:100D700064696D6D657220004D423A20496C6C6566
:100D800067616C20617267756D656E74730A00200F
:100D90006572726F723D004D423A20706F6C6C69E3
:100DA0006E6720504920002D004D423A20504920C6
:100DB00056616C203A004D423A20706F6C6C696E3F
:100DC0006720504920004D423A20706F6C6C696E6C
:100DD0006720464D206661756C7420002065727234
:100DE0006F723D004D423A20706F6C6C696E6720E7
:100DF000002D004D423A20464D2056616C203A00AD
:100E00004D423A20706F6C6C696E6720464D200031
:100E10004354524C2F706F6C6C3A204F75744F6670
:100E20004D656D6F72793A2000207365632072659D
:100E30006D61696E696E67005374617475732064C7
:100E4000656666657265640A002D3E005075623AFB
:100E500020006374726C00454E41424C450046527E
:100E600045455A450044495341424C45002D3E00FA
:100E70005075623A2000636D640046414E5F4F4EEC
:100E80004C590044525900434F4F4C00484541547F
:100E9000004155544F002D3E005075623A200073BA
:100EA00065740064656C002D3E005075623A200048
:100EB0002D3E005075623A2000556E6B6E6F776E56
:100EC00020636D64200A004F4646004F4E002066A6
:100ED00061696C65643A004D6F64627573206F7070
:100EE00020004D423A206F6B003D004D423A2056A3
:100EF00043230020636D643D003D004D423A20567F
:100F0000435F6865617423004D423A204E6F742040
:100F1000737570706F727465642072656720747980
:100F200070650A002056616C3A30780020543A000F
:100F3000205265673A3078004D423A20416464722D
:100F40003A00444D58000000000000444D585247FC
:100F500042570000444D5852474200000050574D40
:100F60000000000000004D42555344494D0000541C
:100F70004845524D4F00000052454C415900000079
:100F80000047524F555000000000564354454D5005
:100F90000000004D42555356430000004143484174
:100FA00049455200005350494C45440000004D4F04
:100FB000544F52000000005049440000000000005F
:100FC0004D425553000000000055415254425244D6
:100FD000470052454C415950574D00444D585247D7
:100FE0004257570056454E545300000000454C45AB
:100FF0005641544F5200434F554E544552000048FD
:10100000554D0000000000004D4552435552590017
:101010000020002D3E00436F6E76657274696E6726
:1010200020002D3E0057726F6E6720417373696711
:101030006E6D656E742000524742783A200020762B
:101040004C6576656C3A0020436F6E76563A002008
:10105000436F6E76533A0020486F743A00436F6CCA
:10106000643A0020436F6E76657274656420563A68
:1010700000436F6E76657274656420533A002D3EAE
:101080000057726F6E672041737369676E6D656E8E
:101090007420002D3E0057726F6E67204173736994
:1010A000676E6D656E74200053617665643A00006A
:1010B00000000000000000004F4E00000000000093
:1010C000004F464600000000000052455354000007
:1010D000000000544F47474C4500000048414C5425
:1010E0000000000000584F4E000000000000584F64
:1010F00046460000000000494E435245415345001A
:10110000444543524541534500454E41424C4500FC
:10111000000044495341424C450000554E4652455B
:10112000455A4500465245455A4500000041555430
:101130004F000000000046414E5F4F4E4C590048A2
:1011400049474800000000004D454449554D000006
:10115000004C4F570000000000004845415400007B
:10116000000000434F4F4C00000000004452590063
:10117000000000000053544F500000000000524790
:10118000420000000000004853560000000000002C
:1011900020537566663A002041543A002069732056
:1011A0000044656C6574696E6720636F6E662E20FF
:1011B00052414D207761733A0053746F70706564CB
:1011C000006E6F7468696E6720746F2073746F703F
:1011D0000053746F7070696E67206368616E6E652E
:1011E0006C73202E2E2E004E6F7420756E6C6F6304
:1011F0006B656420696E20313073202D20636F6E23
:1012000074696E7565202E2E2E00556E6C6F636BA3
:10121000696E6720636F6E666967202E2E2E00430D
:101220006F6D706C6574652E2052656D6F766520EC
:10123000746F706963200024636F6D6D616E64006C
:10124000536B697070696E672E2E00436C65616E1A
:1012500055702072657461696E656420746F706981
:10126000632000220022004F75744F664D656D6F3C
:10127000727921005D20003A5B000A005D00456D37
:101280007074793A205B000A003A004D41433A00FD
:10129000476F7420495020616464726573733A002B
:1012A000276970205B69705B2C646E735B2C6777B9
:1012B0005B2C7375626E65745D5D5D5D27202D200E
:1012C000736574207374617469632049500A004621
:1012D00061696C656420746F20636F6E6669677501
:1012E00072652045746865726E6574207573696EE9
:1012F0006720444843502E20596F752063616E204B
:10130000736574206970206D616E75616C6C7921F4
:1013100000204D41534B3A002047573A0020444E9D
:10132000533A004C6F616465642066726F6D20668D
:101330006C6173682049503A000A757365732044E4
:101340004843500A005374617274696E67206C617F
:101350006E00546F6F206D616E79204D5154542092
:10136000636F6E6E656374696F6E206572726F7203
:10137000732E2052657374617274204C414E0020AC
:1013800074727920616761696E20696E20352073FF
:1013900065636F6E6473006661696C65642C2072AE
:1013A000633D004177616974696E6720666F7220E2
:1013B00072657461696E656420746F70696373002F
:1013C000636F6E6E65637465642061732000202E08
:1013D0002E2E0020757365723A003A000A4174742B
:1013E000656D7074696E67204D51545420636F6E43
:1013F0006E656374696F6E20746F20006469736337
:101400006F6E6E6563746564005573696E67204D19
:101410005154542070617373776F72642066726FD9
:101420006D20636F6E666967004465766963652049
:101430004E616D653A004174206C6561737420647F
:101440006576696365206E616D6520616E642062FA
:10145000726F6B6572204950206D757374206265E0
:1014600020636F6E6669677572656400246E6F64D1
:101470006573004F4E2C4F46462C48414C542C521D
:101480004553542C584F4E2C584F46462C544F47DA
:10149000474C450024666F726D617400656E756D12
:1014A0000024646174617479706500687376006308
:1014B0006F6C6F7200302D32353500696E74656760
:1014C000657200666C6F617400332E302E3100241B
:1014D000686F6D696500757074696D652C667265FD
:1014E000656865617000326532313336325F3230A3
:1014F00032332D31312D3132004C696768744875B3
:10150000622000246E616D6500526562696E642020
:10151000737563636573732E204950206164647230
:101520006573733A004572726F723A207265626930
:101530006E64206661696C0052656E657765642033
:10154000737563636573732E204950206164647200
:101550006573733A004572726F723A2072656E65F8
:10156000776564206661696C000A4E6F206C696E55
:101570006B0033307320454550524F4D2069732026
:101580006E6F742072656C6F616465642E205265A5
:10159000626F6F7400416363657074696E67206386
:1015A0006F6D6D616E64732E2E2E0A004E6F204D8E
:1015B00051545420636F6E66696775726564004CA0
:1015C0006F6164696E6720636F6E6669672066721B
:1015D0006F6D20706F7274616C2064697361626CEE
:1015E00065642E2075736520676574204F4E2074E6
:1015F0006F20656E61626C6500436F6E666967207F
:1016000069732076616C696400436F6E74696E75EE
:101610006520776974682070726576696F75736C80
:1016200079206C6F6164656420636F6E6669670022
:1016300043757272656E74204C414E20636F6E6606
:1016400069672869702C646E732C67772C737562D8
:101650006E6574293A000A55736520746865736570
:1016600020636F6D6D616E64733A202768656C70DE
:1016700027202D207468697320746578740A276D9B
:1016800061632064653A61643A62653A65663A6608
:10169000653A3030272073657420616E642073745E
:1016A0006F7265204D41432D6164647265737320D0
:1016B000696E20454550524F4D0A276970205B697D
:1016C000705B2C646E735B2C67775B2C7375626E3A
:1016D00065745D5D5D5D27202D20736574207374D6
:1016E000617469632049500A277361766527202D4C
:1016F00020736176652063757272656E7420636F06
:101700006E66696720696E204E5652414D3B204FF0
:101710004E7C4F4646202D20656E61626C652F64BD
:10172000697361626C65206175746F736176650AB7
:101730002767657427205B636F6E66696720616445
:1017400064725D27202D2067657420636F6E666963
:10175000672066726F6D207072652D636F6E6669AB
:1017600067757265642055524C20616E64207374F5
:101770006F726520616464722C204F4E7C4F464628
:10178000202D20656E61626C652F64697361626CE7
:101790006520646F776E6C6F6164206F6E20737468
:1017A00061727475700A276C6F616427202D206C3C
:1017B0006F616420636F6E6669672066726F6D206B
:1017C0004E5652414D0A2770776427202D206465BC
:1017D00066696E6520616E642073746F7265204D5A
:1017E0005154542070617373776F72640A276F7459
:1017F0006170776427202D20646566696E652061BD
:101800006E642073746F72652048545450204150A8
:10181000492070617373776F72640A276C6F672059
:101820005B73657269616C5F6C6F676C6576656C24
:101830005D205B7564705F6C6F676C6576656C5D71
:1018400027202D20646566696E65206C6F67206CAB
:101850006576656C2028302E2E37290A276B696C37
:101860006C27202D2074657374207761746368641D
:101870006F670A27636C65617227202D20636C6592
:10188000617220454550524F4D0A2773656172635E
:101890006827202D2073656172636820312D776978
:1018A0007265206465760A277265626F6F742720FF
:1018B0002D207265626F6F7420636F6E74726F6C2F
:1018C0006C657200536F6674207265626F6F746925
:1018D0006E672E2E2E00206E657700206973200023
:1018E0003157543A003157543A2053656172636856
:1018F000696E67206465760052414D3D000A312DC6
:101900007769726520000A6D71747420000A6D6F2A
:1019100064627573207632000A6D6F64627573209D
:10192000763120282B29000A696E707574732000A7
:101930000A6974656D7320000A436F6E6669677586
:101940007265643A003157543A207365747570209B
:101950007265736F6C7574696F6E20003157543AFD
:10196000204453323438322D313030206E6F7420A1
:1019700070726573656E74003157543A2044533267
:101980003438322D3130302049324320726573743F
:101990006F726564000944533234383220726573C3
:1019A0006574206572726F720009526573657420E8
:1019B000646F6E650009436865636B696E672066D6
:1019C0006F7220312D576972652064657669636591
:1019D000732E2E2E003157543A204453323438326D
:1019E0002D3130302070726573656E7400457272EF
:1019F0006F7220312D7720696E69740046726565BB
:101A00003A004453323438325F3130305F49324328
:101A10005F544F5F31575F42524944474520696EDA
:101A2000697400444D584F75742E20467265653AAE
:101A300000444D58696E2042756666657220616C7F
:101A40006C6F632065727200496E697420696E2044
:101A500063683A003B003D0050696E3A003B003D30
:101A60004C4F5700546865726D6F3A004F6E652099
:101A7000776972652052656164790A00467265650E
:101A80003A00444D58206F75742073746172746508
:101A9000642E204368616E6E656C733A2000444D7D
:101AA0005820696E20737461727465642E204368D7
:101AB000616E6E656C733A004170706C79696E6727
:101AC00020636F6E66696700436F6E6669672061A9
:101AD00075746F736176653A000A5379736C6F673A
:101AE000206465627567206C6576656C3A005365A5
:101AF0007269616C206465627567206C6576656CDF
:101B00003A0053617665640A005365742064796E07
:101B1000616D69632049500A00454550524F4D2080
:101B2000636C65617265640A004D515454205061C4
:101B30007373776F726420757064617465640A00F2
:101B40004F54412050617373776F726420757064D5
:101B5000617465640A00636F756C64206E6F742035
:101B600070617273653A2000557064617465640A2F
:101B7000004E6F2049502061647265737300526596
:101B80006C656173696E6720736F636B6574206148
:101B90006E6420726574727900205361766564000A
:101BA0004C6F6164696E67204854545020636F6EB7
:101BB000666967206F6E20737461727475703A0085
:101BC0004F4646004F4E002B002D00455461673AAA
:101BD000200047657420455441473A20004854543A
:101BE000502F312E310025733A2025730D0A002025
:101BF000485454502F312E310D0A486F73743A20D7
:101C000025730D0A4163636570743A202A2F2A0DEB
:101C10000A436F6E6E656374696F6E3A20636C6F12
:101C200073650D0A0025730020000D0A0047455416
:101C3000006661696C656420746F20636F6E6E6509
:101C400063740A004552524F523A205365727665CA
:101C5000722072657475726E65642000436F6E66E3
:101C60006967206E6F74206368616E6765640A003F
:101C7000446F6E652E0A00436F6E6669672070615F
:101C80007273696E67206661696C65640A00676FCC
:101C90007420436F6E6669670A00687474702072FE
:101CA0006574636F64652000667265652000436F2C
:101CB0006E666967205552493A20687474703A2FED
:101CC0002F002044656661756C7420636F6E6669D1
:101CD000672073657276657220757365643A2000BB
:101CE0006C617A79686F6D652E7275000A282B29F0
:101CF0004D554C544956454E54000A282B295057EF
:101D00004D5F52454C4159000A282D294D444E53F0
:101D1000000A282D29554152544252494447450052
:101D20000A282D295359534C4F47000A282B295074
:101D30004944000A282D294D4350323330313700B1
:101D40000A282D294152544E4554000A282D294F66
:101D50005441000A282B29535049204C4544000A7D
:101D6000282B294D4F544F5220435452000A282B00
:101D7000294143204841494552206F6E20536572E6
:101D800069616C32000A282B2943435338313120D2
:101D9000262048444331303830000A282B29524548
:101DA00053544152545F4C414E5F4F4E5F4D51541E
:101DB000545F4552524F5253000A282D2948415230
:101DC0004452455345542C207573696E6720736FD8
:101DD0006674000A282B29434F554E544552000A79
:101DE000282B29444854000A282B294453323438DC
:101DF000322D313030000A282B294F5749524500E7
:101E00000A282D2949504D4F44425553000A282B8A
:101E1000294D4F444255532030783036206174208C
:101E200053657269616C332073706565643A393645
:101E30003030000A282B294144414652554954204C
:101E40004C4544000A282B29444D58000A282B29C8
:101E500057697A6E657435313030000A282B29466F
:101E600072656552616D207072696E74696E67008B
:101E70000A282B295741544348444F47000A282B2E
:101E800029434F4E54524F4C4C494E4F000A46691D
:101E9000726D77617265204D4143204164647265C3
:101EA00073732064653A61643A62653A65663A66BE
:101EB000653A3037006C617A79686F6D652E72759E
:101EC000000A436F6E666967207365727665723AC1
:101ED000003230313130334C0020432B2B207665DB
:101EE0007273696F6E3A00326532313336325F3267
:101EF0003032332D31312D3132000A4C617A79681C
:101F00006F6D652E7275204C696768744875622024
:101F1000636F6E74726F6C6C65722000204F464662
:101F200000204F4E002042595041535300726561CA
:101F300064790024737461746500757074696D65EB
:101F400000667265656865617000247374617473FE
:101F5000002054696D65723A00204C6F636B733AD0
:101F6000002000204C6F636B733A000A52414D3DD4
:101F70000020457870697265640A00202D746172D2
:101F8000676574207A6F6E652D0020416C61726DFB
:101F900020457870697265640A0020636D643A00B8
:101FA000204375723A00205365743A005361766598
:101FB0006420746F20454550524F4D00536176693F
:101FC0006E6720636F6E66696720746F20454550A9
:101FD000524F4D2E2E004C6F616465642045544174
:101FE000473A004E6F2073746F72656420636F6EA2
:101FF000666967004C6F616465642066726F6D206E
:10200000454550524F4D006C6F6164206661696CAC
:102010006564004A534F4E2064657465637465645B
:10202000004C6F6164696E6720436F6E666967205C
:1020300066726F6D20454550524F4D006363733893
:10204000313120697320616C726561647920696E39
:10205000697469616C697A656400686463313038F9
:102060003020697320616C726561647920696E69E2
:102070007469616C697A6564004844433130383072
:10208000206E6F7420696E697469616C697A656429
:10209000006363733831313A2064617461206E6F7C
:1020A0007420617661696C61626C6500636373388A
:1020B0003131206E6F7420696E697469616C697A60
:1020C000656400203C3C0041433A200041433A20F3
:1020D00053657269616C2075736564206279204173
:1020E00043202D2064697361626C696E672073659B
:1020F0007269616C206C6F6767696E6720616E64DE
:1021000020636D640041433A204F7574206F662050
:102110006D656D6F72790041433A20496E69743A7A
:10212000200041433A2044652D496E69743A2000ED
:102130004F4646004452590046414E5F4F4E4C595F
:10214000004845415400434F4F4C00455252004116
:10215000433A204F4B00203E3E200041433A2000AE
:1021600041433A20506F6C6C696E67004C4F5700CA
:102170004D454449554D0048494748004155544F45
:1021800000726177007175656974007377696E67B5
:10219000006C6F636B00556E6B6E6F776E2073759E
:1021A000666669782000556E6B6E6F776E20636D82
:1021B000642000436F756E7465723A2000444D5878
:1021C0002D4F757420496E69743A2000444D582D86
:1021D0004F75742073746F703A2000417373696790
:1021E0006E65643A00444D58206374726C3A200066
:1021F00069313600016933320002753136000375EA
:1022000033320004693868000569386C0006753897
:1022100068000775386C00087831300009313030BB
:10222000000A44656661756C742073657269616C3F
:10223000206D6F6465204E383120757365640038F9
:102240004531002600384E31000600384532002E58
:1022500000384E32000E00384F31003600384F3211
:10226000003E00374531002400374532002C00374E
:102270004F31003400374F32003C00374E310004FC
:1022800000374E32000C004D4255533A204D6F64DA
:102290006275732074656D706C617465206E6F7407
:1022A00020666F756E643A20004D4255533A2049BE
:1022B0006E76616C69642074656D706C6174652EF6
:1022C000002C002C002C002C004D4255533A20636A
:1022D0006F6E666967206661696C65643A004D429D
:1022E00055533A20636F6E666967206572726F722C
:1022F000004D4255533A20636F6E666967206C6FDC
:102300006164656420004D4255533A204F75742036
:102310006F66206D656D6F7279004D4255533A209E
:10232000506F6C6C696E67206572726F7220004D21
:10233000425553443A2049676E6F726564202D20E0
:10234000657175616C207769746820736574746554
:10235000642076616C004D4255533A2041646420FC
:1023600040533A20004D425553443A204E65737411
:1023700065644D61707065643A004C6173744B6EB6
:102380006F776E2076616C75653A200053656172D7
:102390006368696E67207265673A2000726567231B
:1023A000206F7574206F662072616E6765005365DB
:1023B00061726368696E672072656723004D4255DC
:1023C00053443A204D61707065643A003A002066CB
:1023D000726F6D207479706520004D425553443AF8
:1023E0002020676F7420002076616C3A0020005234
:1023F00065733A200020696E7465726E616C20739B
:10240000656E64206572726F72202D206E6F20726F
:1024100065672F636F696C0020696E7465726E6109
:102420006C2073656E64206572726F72202D206E51
:102430006F2074656D706C6174650020696E7465E1
:10244000726E616C2073656E64206572726F7220AB
:102450002D206E6F2073746F7265004D425553448A
:102460003A20656E64506F6C6C20004D42555344A9
:102470003A20506F6C6C2000206E6F7420666F7570
:102480006E64004D4255533A2020706172616D2098
:10249000002073656E64206572726F722E20004D8D
:1024A0004255533A2020004164642040563A2000AF
:1024B0002056616C3A20004D425553443A207375C2
:1024C000666669783A00206F72207375666669786F
:1024D00020004D4255533A204E6F2074656D706C4C
:1024E00061746520666F7220004D6F746F723A20C0
:1024F00074696D656F757400556E6B6E6F776E20C5
:10250000636D64004D6F746F723A20466F7263653D
:102510006420657865637574696F6E004D756C74C1
:102520006956656E7420636F6E66696720666169BF
:102530006C6564004D756C746956656E7420696EC7
:102540006974004D756C746976656E742044652DF0
:10255000496E697400204F75743A00206D33002075
:1025600066726F6D2000204D61782072657175650F
:1025700073743A002066616E253A002061637469C5
:10258000766520563A00546F74616C20563A0050BC
:1025900049443A20616C726561647920696E69749E
:1025A00069616C697A6564005049443A20496E76E5
:1025B000616C696420706172616D20617272617911
:1025C0002E002C002C002C002C005049443A206393
:1025D0006F6E666967206661696C65643A00504990
:1025E000443A20636F6E666967206572726F72008D
:1025F0005049443A20636F6E666967206C6F61646E
:10260000656420005049443A204F7574206F66205D
:102610006D656D6F7279005049443A2044652D49CB
:102620006E69742000203C414C4D3E0020443A002D
:1026300020493A0020503A0020696E3A0020736524
:10264000743A005049443A20005049443A20496EB7
:1026500076616C696420706172616D206172726173
:10266000792E00536574206F757420746F200020DC
:1026700050494420616C61726D2E20002050494405
:1026800020616C61726D3A20636C6F7365640050F9
:1026900049443A20556E6B6E6F776E20737566668F
:1026A000697820005049443A20556E6B6E6F776E02
:1026B00020636D64200020536574706F696E743AF6
:1026C000005049443A200020496E707574207661AC
:1026D0006C75653A005049443A200020696E69746F
:1026E00000200050574D2D4F757420230020737427
:1026F0006F7000200050574D2D4F75742023003D02
:102700000050696E3A0020696E69740052656C6110
:10271000792D4F75742023002073746F70005265FB
:102720006C61792D4F75742023003D3E003A007096
:10273000756220616374696F6E200069646C650066
:102740006F66660068656174696E670066616E0039
:10275000647279696E6700636F6F6C696E670020E1
:10276000697320004F75742000556E6B6E6F776E25
:10277000207375666669782000556E6B6E6F776E94
:1027800020636D642000616374696F6E0072656C14
:1027900061794374723A200053686F770020636D4B
:1027A000643D002D002072656164206572726F7255
:1027B00020666F7220003E2000203C003157543AC2
:1027C000003157543A206E6F7420696E697400317D
:1027D00057543A206C6F7374204453323438322D7E
:1027E000313030003157543A206572726F720031C7
:1027F00057543A20312D776972652073686F72746F
:102800006564003157543A204453323438325F45BE
:1028100052524F525F434F4E464947003157543A48
:1028200020312D776972652073686F72746564005A
:1028300020002E00696E00735F6F7574006D7968FB
:102840006F6D65004354524C2F657865633A204F95
:1028500075744F664D656D6F72793A2000202D3E7C
:102860002000456D69743A2000202D3E20004974F7
:10287000656D436D643A2000202D3E20004974654B
:102880006D3A200009445332343832207265736542
:1028900074206572726F72000952657365742064EA
:1028A0006F6E6500005EBCE2613FDD83C29C7E20EE
:1028B000A3FD1F419DC3217FFCA2401E5F01E3BD1C
:1028C0003E6082DC237D9FC1421CFEA0E1BF5D0310
:1028D00080DE3C62BEE0025CDF81633D7C22C09E04
:1028E0001D43A1FF4618FAA427799BC584DA3866F0
:1028F000E5BB5907DB856739BAE406581947A5FBDC
:102900007826C49A653BD987045AB8E6A7F91B45CF
:10291000C6987A24F8A6441A99C7257B3A6486D8C3
:102920005B05E7B98CD2306EEDB3510F4E10F2ACAF
:102930002F7193CD114FADF3702ECC92D38D6F319B
:10294000B2EC0E50AFF1134DCE90722C6D33D18F8F
:102950000C52B0EE326C8ED0530DEFB1F0AE4C1283
:1029600091CF2D73CA947628ABF517490856B4EA6F
:102970006937D58B5709EBB536688AD495CB29775B
:10298000F4AA4816E9B7550B88D6346A2B7597C94F
:102990004A14F6A8742AC896154BA9F7B6E80A5443
:1029A000D7896B35436F6E6E65637465642E004323
:1029B0006F6E6E2E2061626F72746564003E3E2001
:1029C00000496E76616C696420636F6D6D616E6441
:1029D00000000020002300260029002C002F0032D8
:1029E00000000100000301060109013E3E3E004EC9
:1029F0006F204D414320636F6E6669677572656431
:102A00003A20736574206669726D77617265277309
:102A1000204D41430A00454550524F4D2073696790
:102A20006E6174757265206F6B00496E69746961BF
:102A30006C697A696E6720454550524F4D2E0000F3
:102A4000002200250028002B002E00310034000257
:102A5000010000050108010B0100000A0B02090C2E
:102A60000D0E080703040100000000000000000034
:102A70000000000000000000000000000000000056
:102A80000000000000121110000000000000000013
:102A90000000000000000000000000000000000036
:102AA000002100240027002A002D003000330001FF
:102AB000010000040107010A01010210202008089A
:102AC0001020401020408002010201080402010190
:102AD0000204081020408080402010080402018079
:102AE00004020180402010080402010804020101D0
:102AF00002040810204080010204081020408005D4
:102B0000050505070508080808020202020A0A0866
:102B1000080404040401010101010101010303038C
:102B20000303030303040707070C0C0C0C0C0C0C29
:102B30000C0202020206060606060606060B0B0B30
:102B40000B0B0B0B0B57726F6E67207061796C610A
:102B500064004354524C2F7478743A204F75744F6C
:102B6000664D656D6F72793A2000202D3E204154EC
:102B70003A004368616E20747970653A004E6F20A8
:102B800073746F7265642076616C756573202D2097
:102B900064656661756C743A2000536176656420E3
:102BA000455441473A0053657420455441473A2003
:102BB00000007303C50211241FBECFEFD1E2DEBFB8
:102BC000CDBF00E00CBF1AE0A0E0B2E0ECE4F0E61C
:102BD00002E00BBF02C007900D92AC3DB107D9F7E0
:102BE00021E1ACEDBAE001C01D92A53DB207E1F7CD
:102BF00015E1CAEDD5E100E006C021970109802F5B
:102C0000FE010F94EA27C93DD10780E00807A9F724
:102C10000F94C31A0D9414300C940000FC018481AD
:102C200095810895DC011696ED91FC91309739F06D
:102C300080858F70823019F486819781089590E0A5
:102C400080E00895FC01A481B581109721F11896C8
:102C50009C9118979F708EEF890F823010F0911120
:102C60001AC019964D935D936D937C931C97A48124
:102C7000B58118969C911897907F926018969C93B6
:102C80000480F581E02D8085982F907F903619F48F
:102C90008F70806A8087089581E090E0089587E0D2
:102CA00090E008958AE090E0089588E090E008952B
:102CB000FC01238130E090E080E0FC01EE0FFF1F7B
:102CC000E85EF44FA081B181A217B30761F4880FC9
:102CD000991F880F991FFC01EC5FF44F40835183CB
:102CE000628373830895A081B181AB2B19F4208195
:102CF0003181EDCF019685309105F9F60895FC01FB
:102D0000238130E090E080E0FC01EE0FFF1FE85EE1
:102D1000F44F408151814217530761F4880F991F86
:102D2000880F991FFC01EC5FF44F608171818281F3
:102D30009381089540815181452B89F4318320830B
:102D4000880F991F880F991FFC01EC5FF44F1082C8
:102D500011821282138260E070E0CB010895019627
:102D60008530910589F6F7CF880F991F880F991F35
:102D7000FC01E451F54F80819181A281B3810196DC
:102D8000A11DB11D80839183A283B383089585E043
:102D900090E00C94B41684E090E00C94B41683E0B8
:102DA00090E00C94B41682E090E00C94B41681E0AC
:102DB00090E00C94B41690E080E00C94B416CF939D
:102DC000DF93EC01E881F9810484F585E02D199504
:102DD00029893A892F5F3F4F3A8B298BDF91CF9119
:102DE0000895CF93DF93EC018E8581110DC081E0B2
:102DF00090E049895A892C853D854217530708F090
:102E000080E0DF91CF910895E881F9810484F58510
:102E1000E02DCE0119958F3F910549F780E090E0B4
:102E2000F0CFFC01848595856817790708F4CB01FC
:102E3000928B818B0895DC011E962C911E97222384
:102E400039F0ED91FC910190F081E02D6FEF199434
:102E50000895FC0187859089089581E0089590E0A8
:102E600080E00895FC0122813381232B49F0868183
:102E700097818130910539F01CF00397039730F06A
:102E800090E080E0089581E090E0089582E090E095
:102E90000895DC011296ED91FC91309761F001905C
:102EA000F081E02D309739F0862F8295807F608504
:102EB0006F70682B60870895DC011296ED91FC918C
:102EC000309751F00190F081E02D309729F0808506
:102ED00082958F7090E0089590E080E008950F93C0
:102EE0001F93CF93DF9300D000D01F921F92CDB7D6
:102EF000DEB781E028960FB6F894DEBF0FBECDBFD7
:102F0000DF91CF911F910F910895089590E080E097
:102F1000089564EA7CE0811102C06FE97CE089EDEC
:102F200090E10D94A612DC0155962C915597273708
:102F300081F4ED91FC91008CF18DE02D199567E005
:102F400079E089ED90E10F94A61289ED90E10D945E
:102F500055100895DC011296ED91FC91309771F0B7
:102F600090859F70923039F0953041F4CF010E94E6
:102F700052F990E0089581E090E0089590E080E0BB
:102F8000089565E0FC01808191810E94C0F800975E
:102F900049F0FC018085982F907F21F082958F70F9
:102FA00090E0089590E080E008950D94B91D0D948F
:102FB000B91DCF93DF93009709F490C0FC012081E5
:102FC000222309F48BC0EC016FE97EE00F945920B5
:102FD000892B09F45FC062E57EE0CE010F94592091
:102FE000892B09F45AC066E77EE0CE010F94592080
:102FF000892B09F455C062ED79E0CE010F94592078
:10300000892B09F450C06EEC79E0CE010F94592061
:10301000892B09F44BC06AEC79E0CE010F9459205A
:10302000892B09F446C066EC79E0CE010F94592053
:10303000892B09F441C062EC79E0CE010F9459204C
:10304000892BE9F16EEB79E0CE010F945920892BA1
:10305000C9F169EB79E0CE010F945920892BA9F1D0
:1030600065EB79E0CE010F945920892B89F163EA51
:103070007EE0CE010F945920892B69F161EB79E054
:10308000CE010F945920892B49F58DE090E0DF9116
:10309000CF91089582E090E0FACF89E090E0F7CFF9
:1030A00081E090E0F4CF88E090E0F1CF85E090E01F
:1030B000EECF86E090E0EBCF87E090E0E8CF8AE0CB
:1030C00090E0E5CF8BE090E0E2CF8CE090E0DFCFC6
:1030D00083E090E0DCCF84E090E0D9CF90E080E026
:1030E000D6CFCF92DF92EF92FF920F931F93CF93A1
:1030F000DF93CDB7DEB7C054D1090FB6F894DEBF69
:103100000FBECDBF8091D90C9091DA0C059709F4D0
:1031100049C06115710509F445C069017A018B0147
:1031200040E450E0CE0101960F94852C6FE270E0F0
:10313000CE0101960F944C2C892B41F4980143E069
:1031400050E060E4CE0101960E9495DB4FE350E031
:10315000B601CE0101960F94672C0E942CF88823AB
:1031600009F18091D90C9091DA0C0697D9F48091ED
:10317000C40B811117C0B701CE0101960F94E3046F
:1031800081E090E0C05CDF4F0FB6F894DEBF0FBE69
:10319000CDBFDF91CF911F910F91FF90EF90DF9006
:1031A000CF90089590E080E0EDCFCF92DF92EF9244
:1031B000FF920F931F93CF93DF93CDB7DEB7609746
:1031C0000FB6F894DEBF0FBECDBF7C016B01CA0104
:1031D000B9012AE0AE014F5F5F4F0F94F220D70193
:1031E000ED91FC910488F589E02D9801AE014F5FC7
:1031F0005F4FB601C701199560960FB6F894DEBF10
:103200000FBECDBFDF91CF911F910F91FF90EF9037
:10321000DF90CF900895CF92DF92EF92FF920F93BD
:103220001F93CF93DF93CDB7DEB760970FB6F894B7
:10323000DEBF0FBECDBF7C016B01BA01A901CE017B
:1032400001960E94BDDCD701ED91FC910488F589BF
:10325000E02D9801AE014F5F5F4FB601C701199590
:1032600060960FB6F894DEBF0FBECDBFDF91CF9151
:103270001F910F91FF90EF90DF90CF9008951F93D3
:10328000CF93DF93FC01162FC389D489818992895A
:103290009C012F5F3F4F328B218BC80FD91FCE016E
:1032A0000F944D27181721F0612FCE010F94552749
:1032B00081E090E0DF91CF911F910895FC01818919
:1032C0009289248535858217930740F423893489B0
:1032D000820F931F0F944D2790E008958FEF9FEF7B
:1032E00008958F929F92AF92BF92CF92DF92EF920A
:1032F000FF920F931F93CF93DF93E091DB0CF0913C
:10330000DC0C309709F467C0812EF02E932EC22E6C
:10331000A52ED42EB72EE62EBC01CF010E940EF8AA
:10332000EC01892B19F481E090E057C088858F70FB
:103330008530C9F760E0CE010E94C0F88C0161E0E1
:10334000CE010E94C0F8FC01C185D285D801199632
:103350002D913C912130310561F13CF46F2DCE016E
:10336000232B09F70E94B9D0DECF2230310531F18D
:1033700027303105C1F6892BB1F280858F708530F9
:1033800091F6C681D781209771F288858F7084303D
:1033900061F40F2D182D2C2D392D4D2D5A2D6E2DFC
:1033A0007B2D89859A850E9471190A80DB81C02D49
:1033B000EACF6F2DCE0103960E94B9D06E2DCE01BB
:1033C0000E94B9D06D2DCE0101960E94B9D06C2D0E
:1033D000CE010296C7CF90E080E0DF91CF911F91A0
:1033E0000F91FF90EF90DF90CF90BF90AF909F90A4
:1033F0008F900895CF92DF92EF92FF920F931F93D9
:10340000CF93DF93E091260BF091270B3097C9F013
:1034100090859F709530A9F469017A01EB01682FBE
:10342000CF010E94C0F8FC0190859F70943049F450
:1034300081859285009729F09601A701BE010E941F
:103440007119DF91CF911F910F91FF90EF90DF9055
:10345000CF9008958F929F92AF92BF92CF92DF92BA
:10346000EF92FF920F931F93CF93DF938091240BE2
:103470009091250B892B09F48BC021E030E0D0E03E
:10348000C0E0CC24C394D12C46010C2E02C0880C81
:10349000991C0A94E2F7092C000CAA08BB087901D0
:1034A00084E0E80EF11CC90150E040E060912E027A
:1034B00070912F02FC016817790720F4E0912E0229
:1034C000F0912F026091D80B7091D90BE60FF71F86
:1034D000A081E091240BF091250BBC016150710992
:1034E000E60FF71F60816A17F1F06091E10A7091B1
:1034F000E20A63307105B4F04091E70A5091E80A9E
:103500006091E90A7091EA0A482959296A297B29B8
:103510004093E70A5093E80A6093E90A7093EA0A35
:10352000A08351E041E00196E816F90609F0BECF0C
:103530004423D9F18091E10A9091E20A0196909397
:10354000E20A8093E10A5523E9F0E091240BF0911F
:10355000250BE20FF31F028110E0218130E0408152
:1035600050E03197608170E0CE010E94FA1980E04E
:103570000E946DD66093E30A7093E40A8093E50A93
:103580009093E60A21969701C430D10509F07CCFCB
:10359000DF91CF911F910F91FF90EF90DF90CF902F
:1035A000BF90AF909F908F9008951092E20A109272
:1035B000E10AC9CFCF93DF9300D000D01F921F92B2
:1035C000CDB7DEB7FC01862F8F706181607F682BDD
:1035D000618388E0DE01119601900D928A95E1F7F2
:1035E00029813A814B815C816D817E818F819885B3
:1035F00028960FB6F894DEBF0FBECDBFDF91CF91F6
:103600000895CF93DF9300D000D01F921F92CDB7C3
:10361000DEB7FC01608398E0DE01119601900D9207
:103620009A95E1F729813A814B815C816D817E8198
:103630008F81988528960FB6F894DEBF0FBECDBF58
:10364000DF91CF9108956F927F928F929F92AF9268
:10365000BF92CF92DF92EF92FF920F931F93CF937F
:10366000DF93CDB7DEB7A0970FB6F894DEBF0FBEDD
:10367000CDBF8C01862E7A01DC018D919C91119732
:10368000892B09F466C01496ED91FC91309709F4EA
:1036900060C080818071BFEF6B135DC0B1F481E0C9
:1036A000A0960FB6F894DEBF0FBECDBFDF91CF91CD
:1036B0001F910F91FF90EF90DF90CF90BF90AF9050
:1036C0009F908F907F906F9008954330510539F30C
:1036D000818082942FE0822267EA79E089ED90E18F
:1036E0000F94A6124AE050E0D80113966C9189ED30
:1036F00090E10F94701065EA79E089ED90E10F9404
:10370000A612D8011496ED91FC9161816F704AE088
:1037100050E089ED90E10F94701062EA79E089ED54
:1037200090E10F94A6124AE050E0682D89ED90E1F7
:103730000F94701089ED90E10F945510D8011496F4
:10374000ED91FC9181818F70881207C080818F7EFE
:10375000808380E0A5CF8111FCCF198E1A8E1B8E3D
:103760001C8E1D8E1E8E1F8E18A28A8D8F708A8FC2
:10377000D8011496ED91FC9181818F708815A9F183
:10378000B3E0EB16F10489F160EA79E089ED90E1AC
:103790000F94A6124AE050E0F801638189ED90E1B0
:1037A0000F9470106EE979E089ED90E10F94A61204
:1037B000D8011496ED91FC9161816F704AE050E060
:1037C00089ED90E10F9470106BE979E089ED90E15B
:1037D0000F94A6124AE050E0682D89ED90E10F9415
:1037E000701089ED90E10F945510F801208131811E
:1037F000FCE0F81508F416C1E82DF0E08827EC5F2E
:10380000F34E8F4F0D94EA27111C4E1CCF1CE61C63
:10381000F21CCF1CA81CCF1CF51C001DBC1C031DDA
:103820000F1DD8011496CD90DC90F60181818F7028
:10383000853009F4F7C050F48230C1F06DE975E0CD
:10384000C9010E940EF83C01912C4BC08730D1F089
:103850008A30A1F766E975E0C9010E940EF83C01C3
:10386000D6019C9092FA992490F83BC060E975E0EB
:10387000C9010E940EF83C01D6019C9090FA99244F
:1038800090F82FC06FE875E0C9010E940EF83C0166
:10389000F601908091FA992490F823C062EA75E0CD
:1038A000C9010E940EF83C01D8011496ED91FC91DB
:1038B000808180FB992490F8982F9E7F80FF9160F3
:1038C00090836114710469F461E0CE0149960E940D
:1038D000011B298B3A8B4B8B5C8B6D8B7E8B8F8B7B
:1038E000988FF801A080B18068ED75E0C5010E9455
:1038F0000EF86C016DED75E0C5010E940EF85C01DB
:10390000892B81F4C114D10469F460E0CE01499699
:103910000E94011B29833A834B835C836D837E83E2
:103920008F839887D8011496ED91FC9161147104EE
:1039300009F07CC0898D811179C0B82DBF708B2EA4
:103940008181807F882A818280818F7E8083A7CE3B
:1039500067EA75E0C9010E940EF83C01D80114968F
:10396000ED91FC91808181FB992490F8982F9D7FA7
:1039700081FF92609083B5CF6DEA75E0C9010E9426
:103980000EF83C01D8011496ED91FC91808182FBE8
:10399000992490F8982F9B7F82FF9460EBCF6DE97C
:1039A00075E0C9010E940EF83C01892B09F04CCF4B
:1039B00062E0CE0149960E94011B29873A874B8716
:1039C0005C876D877E878F87988B3ECF63EB75E032
:1039D000C9010E940EF83C01D8011496ED91FC91AA
:1039E00090804CCF68EB75E0F3CF6EEB75E0C901CA
:1039F0000E940EF83C01D8011496ED91FC9149CF3C
:103A000064EC75E0F4CF6BEC75E0C9010E940EF830
:103A10003C01D8011496ED91FC91908023CF61ED8B
:103A200075E0F3CF912C712C612C5BCF83E0E8160D
:103A3000F104B9F0982D9F70892E8181807F882AAA
:103A4000818280818F7E8083E98CFA8C0B8D1C8D26
:103A50002D8D3E8D4F8D58A1692DC3010E9423E00D
:103A60001ECE81818F70881509F419CE829490EF53
:103A70008922882A81828081806168CFCF93DF93F9
:103A800000D000D01F921F92CDB7DEB7FC0191810C
:103A90009F70906B9183448355836683778388E01E
:103AA000DE01119601900D928A95E1F729813A8104
:103AB0004B815C816D817E818F81988528960FB6C0
:103AC000F894DEBF0FBECDBFDF91CF910895CF93A5
:103AD000DF9300D000D01F921F92CDB7DEB7FC015C
:103AE00091819F70906A9183448355836683778325
:103AF00088E0DE01119601900D928A95E1F7298107
:103B00003A814B815C816D817E818F819885289679
:103B10000FB6F894DEBF0FBECDBFDF91CF910895F1
:103B2000CF93DF9300D000D01F921F92CDB7DEB7A6
:103B3000FC016F3F710519F014F06FEF70E077FD35
:103B400060E09181892F82958F7081508230C8F416
:103B5000648388E0DE01119601900D928A95E1F769
:103B600029813A814B815C816D817E818F8198852D
:103B700028960FB6F894DEBF0FBECDBFDF91CF9170
:103B800008959F7090619183E3CFCF93DF93CDB77A
:103B9000DEB760970FB6F894DEBF0FBECDBF1982B7
:103BA0001A821B821C821D821E821F8218868A81B5
:103BB0008F708A836FEF70E0CE0101960E94901D96
:103BC00060960FB6F894DEBF0FBECDBFDF91CF91E8
:103BD0000895CF92DF92EF92FF92DC01362F11967B
:103BE000EC911197E295EF70EC3008F0B6C0F0E080
:103BF0008827E250F24E8F4F0D94EA27B01E361EF2
:103C0000361EAD1EAD1EAD1E7B1E3D1EAD1EAD1E75
:103C10000A1E0A1E14968D919D910D90BC91A02DA7
:103C2000662399F0B7FD9FC08F3F9105A105B105AF
:103C300029F024F08FEF90E0A0E0B0E02FEF30E02B
:103C4000A901481B590BCA010CC0B7FD89C08F3FA1
:103C50009105A105B10529F024F08FEF90E0A0E0D7
:103C6000B0E0FF90EF90DF90CF90089514962C91E4
:103C7000822F90E06623A9F3E1CF1496CD90DD90DA
:103C8000ED90FC901797662301F120E030E0A90148
:103C9000C701B6010F94292687FD65C020E030E0FA
:103CA0004FE753E4C701B6010F94312918160CF4FD
:103CB00057C0A701960160E070E08FE793E40F948E
:103CC0001C280F94FB28CB01CCCF20E030E0A901C9
:103CD000C701B6010F94292687FD42C020E030E0DD
:103CE0004FE753E4C701B6010F9431291816DCF1F0
:103CF000C701B601E6CF14966D917D918D919C918F
:103D000017973323B1F06D395FEF75078507950776
:103D100054F1611524E67207810591050CF52CE933
:103D20003FEF4FEF5FEF0F949527C90181509F4FF1
:103D300098CF6D394FEF7407840794078CF06115A5
:103D400054E675078105910574F424E630E040E0FF
:103D500050E00F949527C90184CF8FEF9FEF81CF5B
:103D600090E080E07ECF8FEF90E07BCFCF93DF932A
:103D7000EC01DB01898182958F708630E1F128F4B6
:103D800081508230C8F080E014C0873009F18A5039
:103D90008230C8F72FEF30E00F94012824E630E09E
:103DA00040E050E00F9495272C833D834E835F8342
:103DB00081E0DF91CF9108952FEF30E00F9401283B
:103DC00024E630E040E050E00F9495272C83F0CFBC
:103DD0002FEF30E00F94012824E630E040E050E07F
:103DE0000F949527CA01B9010F9430266C837D8307
:103DF0008E839F83DDCF2CE933E60F94012824E6E0
:103E000030E040E050E00F9495272C833D834E83B3
:103E10005F83B9CFDC011196EC911197E295EF70B9
:103E2000E150EB3008F039C0F0E08827E55EF04E55
:103E30008F4F0D94EA273E1F3E1F4D1F261F261F42
:103E40002F1F461F461F461F261F261F14966D91C3
:103E50007D918D919C9117970F943026089514961B
:103E60006D917D918D919C91179724E630E040E013
:103E700050E00F949527CA01B901EECF14966C91CA
:103E800070E090E080E00F942E26089514966D91D6
:103E90007D918D919C911797089560E070E0CB0122
:103EA0000895DC011196EC911197E295EF70E150C5
:103EB000EB3008F037C0F0E08827EE59F04E8F4F16
:103EC0000D94EA27741F741F921F6D1F6D1F831FAF
:103ED0007A1F7A1F7A1F6D1F6D1F14966D917D9149
:103EE0008D919C911797089514966C9170E090E0D5
:103EF00080E0089514966D917D918D919C91179716
:103F00000F94FB28089514966D917D918D919C914D
:103F1000179724E630E040E050E00F949527CA015F
:103F2000B901089560E070E0CB0108958F929F92EF
:103F3000AF92BF92CF92DF92EF920F931F93CF93E6
:103F4000DF9300D000D01F921F92CDB7DEB7FC01E7
:103F500009831A832B833C834D835E836F83788729
:103F6000808191810097A1F490E080E028960FB6BF
:103F7000F894DEBF0FBECDBFDF91CF911F910F919F
:103F8000EF90DF90CF90BF90AF909F908F9008956B
:103F90008F010E9452F9C82ED12C86E0C816D10498
:103FA00064F40E946FFCBC01F801808191810E9441
:103FB000BFFBFFEFCF1ADF0AF0CF65E0F801808189
:103FC00091810E94C0F88C01892B71F28981803126
:103FD00058F6CE0101960E94511F161617061806B4
:103FE000190644F4F8018085982F9D70A1F08F7018
:103FF000873089F0F80180858F70808767E27AE0EA
:1040000089ED90E10F94A61289ED90E10F9455107F
:1040100081E090E0ABCF0F9446044B015C01CE01F0
:1040200001960E94511F860E971EA81EB91EF80108
:1040300081869286A386B48682E0E11087E099812A
:104040009295907F892BF80180876CE17AE089ED69
:1040500090E10F94A612CE0101960E94511FAB0170
:10406000BC012AE030E089ED90E10F944F1166E148
:104070007AE089ED90E10F94A612F801418552850E
:10408000638574852AE030E089ED90E10F944F114B
:10409000BBCFDC011196EC911197E295EF70E150E6
:1040A000EB3008F03EC0F0E08827E65AFF4D8F4F16
:1040B0000D94EA27702070209120652065208A20C9
:1040C0007B207B207B206520652014962D913D91DF
:1040D0004D915C911797A4E6B0E00F94B427089532
:1040E00014966C9184E6689FB0011124072E000C91
:1040F000880B990B089520E030E048EC52E41496C8
:104100006D917D918D919C9117970F948F260F94AF
:10411000FB28089514966D917D918D919C91179730
:10412000089560E070E0CB010895FC01A7812A2F7B
:104130002E7FD1F0818182958F7081508330A0F4E1
:10414000A695A150BB0B2BE531E00F94012824E686
:1041500030E040E050E00F949527DA01C90187561E
:104160009F4FAF4FBF4F08958FEF9FEF08952F924E
:104170003F924F925F926F927F928F929F92AF92F7
:10418000BF92CF92DF92EF92FF920F93CF93DF9384
:1041900000D01F92CDB7DEB77C017A8369835C8340
:1041A0004B83DB011C92FC016081662309F44EC045
:1041B00030FF4CC0F9E06F9FB001112461557F4E74
:1041C000CD010F949020D70111968C91807F41F002
:1041D0004B815C816CEC76E089819A810F94672C2D
:1041E000E981FA8101900020E9F7319729813A812C
:1041F000E21BF30B19012E0E3F1E4B815C814E1BFF
:104200005F0B415051095C834B83D7011196EC91B0
:1042100011978E2F807F09F4F7C0E295EF70E1507F
:10422000EC3008F0F1C0F0E08827E65EFE4D8F4FDD
:104230000D94EA272921CC2139229822B322772113
:1042400049224922492265214D21CF2229803A80E5
:10425000DCCFF7018481282F30E050E040E00023DC
:1042600059F030E0A4E6B0E00F94C7272FEF30E01C
:1042700040E050E00F9495275F934F933F932F9327
:1042800082EE95E09F938F93FC81FF932B812F9378
:104290003F922F920F949F2CB2C017968C91179734
:1042A0008F9316968C9116978F9315968C911597E0
:1042B0008F9314968C918F9385EE95E09F938F93B7
:1042C000BC81BF93EB81EF93E3CF17968C91179747
:1042D0008F9316968C9116978F9315968C911597B0
:1042E0008F9314968C918F9389EE95E0E7CF149677
:1042F000CD90DD90ED90FC901797F7FE34C084E6EA
:10430000882E912CA12CB12CC701B601A5019401D6
:104310000F9495279B01AC0188279927DC01821B0C
:10432000930BA40BB50BBF93AF939F938F9366270B
:104330007727CB016C197D098E099F09A50194018E
:104340000F9495275F934F933F932F938DEE95E0B6
:104350009F938F933C813F934B814F933F922F923A
:104360000F949F2C4CC0C701B60124E630E040E01A
:1043700050E00F9495279F938F937F936F935F9354
:104380004F933F932F938EEE95E09F938F939C8155
:104390009F93AB81AF93E2CFC7010E949520BC01F0
:1043A000D7011696CC9016971796DC901797D0FAEF
:1043B000DD24D0F814969C9114971596FC90EB8010
:1043C000BC80292F30E050E040E077FD35C001117E
:1043D00035C07F936F931F921F921F929F931F92DE
:1043E000FF92DF92CF9287EF95E09F938F93FC81AE
:1043F000FF932B812F933F922F920F949F2C0FB6F8
:10440000F894DEBF0FBECDBF89819A810F900F90C7
:104410000F900F90DF91CF910F91FF90EF90DF9071
:10442000CF90BF90AF909F908F907F906F905F9054
:104430004F903F902F900895002361F0292F30E096
:10444000A4E6B0E00F94C7272FEF30E040E050E043
:104450000F9495275F934F933F932F931F92FF9253
:10446000DF92CF928AEF95E09F938F93BF92EF9266
:1044700075CF15968C9115971F928F9316969C91D8
:10448000169717968C9181708F939F938DEF95E07F
:1044900015CF14968D909D90AD90BC90179720E00D
:1044A00030E0A901C501B4010F942926240135018A
:1044B00087FF04C077FA709477F87094C301B20153
:1044C0000F94FB286B01072E000C880B990B0F949F
:1044D00030269B01AC01C301B2010F941C2820E0DF
:1044E00030E04AE754E40F948F260F9486290F9406
:1044F000FB28062F772E20E030E0A901C501B4018A
:104500000F94292687FF07C07F920F93DF92CF92E7
:1045100083E096E0D3CE7F920F93DF92CF9284E038
:1045200096E09F938F933C813F934B814F93B0CE06
:1045300014968C9114971F928F9315968C911597C2
:104540001F928F9316968C911F928F938AEF95E00E
:104550009F938F93BC81BF93EB81EF933F922F92F8
:104560000F949F2C4CCF17968C9117971F928F9377
:1045700014968C9114971F928F9315968C91159782
:104580001F928F9316968C911F928F9387EF95E0D1
:104590009F938F93BC81BF93EB81EF93DFCE1496F3
:1045A0006D917C914B815C81C1010F94852C2CCF46
:1045B000EF92FF920F93CF93DF93CDB7DEB7A09723
:1045C0000FB6F894DEBF0FBECDBF7C0100E020E047
:1045D00033E040E250E0BE016F5F7F4F0E94B720A2
:1045E000BE016F5F7F4F89ED90E10F94B01167E9D5
:1045F00071E189ED90E10F94A612F7016181629556
:104600006F704AE050E089ED90E10F94701060E91E
:1046100071E189ED90E10F94A612F70161816F704D
:104620004AE050E089ED90E10F94701089ED90E13F
:104630000F945510A0960FB6F894DEBF0FBECDBFF5
:10464000DF91CF910F91FF90EF900895CF93DF937B
:10465000EC016115710539F48F8181708F8381E0E0
:10466000DF91CF9108958981982F92959F7029F1BC
:1046700080E09430A8F79B01770F440B550B295924
:10468000310941095109A4E6B0E00F94B4272BE5A4
:1046900031E040E050E00F94952737FF02C030E052
:1046A00020E02536310514F024E630E02F5F220F9C
:1046B0008F818170282B2F83D2CF8F708062898366
:1046C000DACFFC019181892F82958F7021F08230A1
:1046D00029F080E008959F70906291839B0177FF9D
:1046E00002C030E020E02E3681E0380714F02DE6DD
:1046F00031E02683878130FB80F9878381E008954C
:10470000EF92FF920F931F93CF93DF93FC01892BBE
:1047100069F19081992351F19D3291F180ED890FDA
:104720008A3070F1C8E0D0E0953211F1CEEFDFEFC2
:104730009B37F1F0C7E1D0E09332D1F08F0188EBE5
:10474000E82E80E1F82EC1E0D0E0C7010F94692087
:10475000AC01B701C8010F948220892B49F0219642
:1047600089E0E80EF11CC931D10579F7CFEFDFEF11
:10477000CE01DF91CF911F910F91FF90EF9008959F
:10478000D0E0C0E0F5CFEF92FF920F931F93CF934D
:10479000DF93EC01892B51F188858F70843009F506
:1047A000E984FA84C7010E9480238C011816190637
:1047B000ECF4C7010E94CCBEC801012E000CAA0B6C
:1047C000BB0B89879A87AB87BC878885807F82608F
:1047D0008887C801DF91CF911F910F91FF90EF90D3
:1047E0000895823019F409851A85F3CF10E000E0AE
:1047F000F0CF2F923F924F925F926F927F928F9263
:104800009F92AF92BF92CF92DF92EF92FF920F935F
:104810001F93CF93DF93CDB7DEB76C970FB6F894A5
:10482000DEBF0FBECDBF6115710549F528E0FC0163
:10483000DE01119601900D922A95E1F729813A81C6
:104840004B815C816D817E818F8198856C960FB6DE
:10485000F894DEBF0FBECDBFDF91CF911F910F91B6
:10486000FF90EF90DF90CF90BF90AF909F908F9090
:104870007F906F905F904F903F902F9008956B01C5
:104880008C016CE277E0C6010E940EF8FC01892BD6
:1048900009F40EC180858F70843009F452C08530D0
:1048A00009F006C1E680F780E114F10409F400C1C3
:1048B000F70180858F70823011F4E280F380E1147B
:1048C000F10409F4F5C0F70180858F70853011F08F
:1048D000F701F3CFC7010E9452F98230C9F760E0B7
:1048E000C7010E94C0F85C010E94C32361E0C701B8
:1048F0000E94C0F84C01FC0180858F70823041F726
:10490000C8010E94511FF40141845284638474845D
:104910006415750586059705D9F6A114B10409F447
:10492000C7C019821A821B821C821D821E821F82AE
:1049300018868A818F708A83F5016185CE01019680
:104940004EC069EE76E0818592850F94572C892BB5
:1049500009F0AEC0C8010E94511F611571058105A3
:10496000910509F48BC0660F771F881F991F2FEFE1
:1049700030E040E050E00F94952757FD15C02330FC
:104980003105410551050CF05FC0DA01C9010196FE
:10499000A11DB11D82309105A105B105D9F1039783
:1049A000A105B10509F450C019821A821B821C822C
:1049B0001D821E821F8218868A818F708A8367E01B
:1049C000CE0101960E94DA1A29873A874B875C87C5
:1049D0006D877E878F87988B62E1CE0109960E9452
:1049E000011B298B3A8B4B8B5C8B6D8B7E8B8F8B5A
:1049F000988F49895A896B897C898D899E89AF896D
:104A0000B88D49835A836B837C838D839E83AF8368
:104A1000B88714CF19821A821B821C821D821E82C3
:104A20001F8218868A818F708A8367E0CE01019683
:104A30000E94DA1A29873A874B875C876D877E87C1
:104A40008F87988B61E1C9CF19821A821B821C82E1
:104A50001D821E821F8218868A818F708A8367E07A
:104A6000CE0101960E94DA1A29873A874B875C8724
:104A70006D877E878F87988B60E1AFCF19821A820E
:104A80001B821C821D821E821F8218868A818F7063
:104A90008A8367E0CE0101960E94DA1A29873A8755
:104AA0004B875C876D877E878F87988B62E095CF79
:104AB0006CE076E0C6010E940EF85C01009709F4F4
:104AC000C5C0FC0180858F70853009F0AEC0C5017E
:104AD0000E9452F9843009F0B9C060E0C5010E941B
:104AE000C0F84C0161E0C5010E94C0F83C0162E0E1
:104AF000C5010E94C0F8FC01C184D284E384F4841F
:104B000063E0C5010E94C0F85C01C8010E94511F0A
:104B10006C157D058E059F059CF419821A821B82F7
:104B20001C821D821E821F8218868A818F708A8352
:104B300040E050E0BA01CE0101960E943E1D51CFE7
:104B4000F4010184F285E02DFA8FE98FF3012184CD
:104B50003284F5010184F285E02DFC8FEB8F198200
:104B60001A821B821C821D821E821F8218868A81E5
:104B70008F708A83298D3A8D4901330FAA08BB08AB
:104B800026010D2C000C66087708C8010E94511FF1
:104B90009B01AC012419350946095709B101032CC1
:104BA000000C880B990B681979098A099B090F94E5
:104BB0006327EB8DFC8D9F01FF0F440B550B2419D0
:104BC0003509460957090F949527820E931EA41E96
:104BD000B51EC101298D3A8D821B930B6B8D7C8D87
:104BE0006C197D090F94D62777FF02C06F5F7F4F46
:104BF00075956795CB01770FAA0BBB0B880E991E95
:104C0000AA1EBB1EB7FC0CC0A401B5013FEF831662
:104C10009104A104B10409F00CF48DCF4FEF01C051
:104C200040E050E060E070E086CF81110FC0198253
:104C30001A821B821C828A818F708A8349815A81E1
:104C40006B817C8180E090E0DC01DBCEF80140816B
:104C500051816281738184819581A681B781D1CE92
:104C60004F925F926F927F928F929F92AF92BF927C
:104C7000CF92DF92EF92FF920F931F93CF93DF9328
:104C8000CDB7DEB760970FB6F894DEBF0FBECDBFCD
:104C90006115710539F528E0FC01DE0111960190DE
:104CA0000D922A95E1F729813A814B815C816D81D2
:104CB0007E818F81988560960FB6F894DEBF0FBE17
:104CC000CDBFDF91CF911F910F91FF90EF90DF90BB
:104CD000CF90BF90AF909F908F907F906F905F909C
:104CE0004F9008956B018C016CE277E0C6010E9441
:104CF0000EF85C01F801F080FF2009F44EC0009727
:104D000009F44BC0FC0180858F70843009F4BFC06A
:104D1000853009F042C060E176E089ED90E10F94C2
:104D2000B01189ED90E10F945510F501E680F78000
:104D3000E114F10491F1F70180858F705701823001
:104D400061F0B12CA12CE114F10409F41DC1F701AB
:104D500080858F70853021F0F701E280F380F3CFFA
:104D6000C7010E9452F98230B9F760E0C7010E9482
:104D7000C0F80E94C3234C0161E0C7010E94C0F843
:104D8000F80120812815190439F7FC0120852F70BE
:104D9000223011F7009709F001C16CE076E0C601FE
:104DA0000E940EF87C01F8018181807F09F407C11F
:104DB000E114F10409F47DC0F70180858F7085301E
:104DC00009F001C1C7010E9452F9843009F0FBC00B
:104DD000C8010E94511F4B015C0160E0C7010E94A5
:104DE000C0F8FC0181859285A385B48519821A8259
:104DF0001B821C821D821E821F82188688169906BD
:104E0000AA06BB060CF499C08A818F708A8363E07E
:104E1000C7010E94C0F85C0162E0C7010E94C0F8AF
:104E2000FC01418452846384748461E0C7010E9460
:104E3000C0F84C0160E0C7010E94C0F8FC01C184C9
:104E4000D284E384F484C8010E94511FF5012185B6
:104E500032854385548524193509460957096C194B
:104E60007D098E099F090F946327F40121853285FE
:104E7000438554852C193D094E095F090F949527E8
:104E8000BA01A901440D551D661D771D31C069EE9B
:104E900076E0818592850F94572C892B09F07DCF80
:104EA000F0E1FF1609F460C0FF1568F082E0F81623
:104EB000E1F1F801408151816281738184819581A2
:104EC000A681B78129C0E1E1FE16F1F1F2E1FF12FE
:104ED000F0CF19821A821B821C821D821E821F82C1
:104EE00018868A818F708A8344E150E060E070E028
:104EF000CE0101960E943E1D29873A874B875C8729
:104F00006D877E878F87988B49855A856B857C85D1
:104F10008D859E85AF85B88949835A836B837C8351
:104F20008D839E83AF83B887BECE19821A821B827F
:104F30001C821D821E821F8218868A818F708A833E
:104F400040E050E0BA01D4CF19821A821B821C8241
:104F50001D821E821F8218868A818F708A8340E894
:104F600050E060E070E0C4CF19821A821B821C827C
:104F70001D821E821F8218868A818F708A834FEF5E
:104F800050E060E070E0B4CFA114B10409F405CFA3
:104F9000F50180858F7009F400CFC50119821A824E
:104FA0001B821C821D821E821F8218862A812F70FE
:104FB0002A83FC01418552856385748599CFE1146C
:104FC000F10409F476CFF70180858F7009F071CF75
:104FD00019821A821B821C828A818F708A8349817E
:104FE0005A816B817C8180E090E0DC0195CF0F934A
:104FF0001F93CF93DF938C01FC01C081D1816FE2BD
:1050000070E0CE010F94942C0097E9F0FC0111920E
:10501000CF010E94D917EC016BEE79E089ED90E1A8
:105020000F94A6124AE050E0BE0189ED90E10F9482
:10503000971189ED90E10F945510CE01DF91CF913A
:105040001F910F910895CE010E94D917EC01892B71
:10505000A1F3F80111821082F0CFDC01ED91FC91F7
:10506000309729F090859F7081E0953009F080E0BD
:105070000895EF92FF920F931F93CF93DF93EC016C
:105080007B018E819F81892BA9F4888199810E945F
:1050900052F9082F10E00530110564F40E946FFCEE
:1050A0009F838E83BC01888199810E94BFFB0F5F23
:1050B0001F4FF1CFEE81FF813097D9F08085982F77
:1050C0009F70A9F4807F82608087EE81FF811186C6
:1050D000128613861486EE81FF81F782E682C7016D
:1050E000DF91CF911F910F91FF90EF900895923033
:1050F00061F3F12CE12CF3CFCF92DF92EF92FF928C
:105100000F931F93CF93DF93EC016A017B018E8194
:105110009F81892BA9F4888199810E9452F9082FD7
:1051200010E00530110564F40E946FFC9F838E83AC
:10513000BC01888199810E94BFFB0F5F1F4FF1CF97
:10514000EE81FF81309749F18085982F9F7019F586
:10515000807F82608087EE81FF81C186D286E38670
:10516000F4866FED79E089ED90E10F94A6122AE0C4
:1051700030E0B701A60189ED90E10F944F1189ED60
:1051800090E1DF91CF911F910F91FF90EF90DF9011
:10519000CF900D9455109230F1F2DF91CF911F9185
:1051A0000F91FF90EF90DF90CF900895FC018681E2
:1051B0009781009799F0FC0120852F70223029F407
:1051C00061857285838594850895253039F460E082
:1051D0000E94C0F8009711F0FC01F2CF60E070E08F
:1051E000CB0108950F931F93CF93DF93FC01C281EE
:1051F000D3812097C9F18B0188858F70853021F587
:10520000CE010E9452F98017110671F16CF1602FE6
:10521000CE010E94C0F8FC01892B31F180858F708E
:10522000823039F461857285838594850F943026A8
:1052300006C08330C9F46185728583859485DF91CA
:10524000CF911F910F910895672B71F4823029F44B
:1052500069857A858B859C85E9CF833029F46985BA
:105260007A858B859C85EBCF60E070E0CB01E7CF42
:105270000F931F93CF93DF93FC01C281D3812097BB
:10528000F9F088858F70823049F4672BC9F48985DD
:105290009A85DF91CF911F910F910895853081F408
:1052A0008B01CE010E9452F98017110649F044F09B
:1052B000602FCE010E94C0F8FC0181859285E9CF64
:1052C00090E080E0E6CF0F931F93CF93DF93EC0144
:1052D0008B017B836A838CE592E09983888370E0FD
:1052E00060E0C8010E94382997FD0CC09D838C8323
:1052F000C8010E94AA179F838E83DF91CF911F91CF
:105300000F910895919581959109F0CF8F929F9279
:10531000AF92BF92CF92DF92EF92FF920F931F93C3
:10532000CF93DF93EC01888199810E9452F9082F75
:1053300010E00430110554F40E946FFCBC01888118
:1053400099810E94BFFB0F5F1F4FF3CF60E0888100
:1053500099810E94C0F87C01009769F1DC011896E0
:105360008C9118978F70843041F51996CD90DC9010
:10537000C114D10401F1F60180818823E1F082E4B7
:10538000882E8FE0982EB12CA12C1A2DC4010F94D9
:105390006920AC01B401C6010F948220892B09F465
:1053A0006BC1FFEFAF1ABF0A89E0880E911CA7E11D
:1053B000AA16B10451F71FEF04C08230E1F7F701DC
:1053C00011851887C880D98061E0C6010E94C0F8A5
:1053D0007C019B838A8362E0C6010E94C0F89D83A2
:1053E0008C8364E0C6010E94C0F89F838E831531D0
:1053F00008F031C0E12FF0E08827EE5FF54D8F4FC8
:105400000D94EA27382A382A382A172A2B2A2B2AD9
:105410002B2A2B2A2B2A2B2A572A462A8D2AB42AB2
:105420009F2A2B2ABF2A382A132B2B2A2E2B8AE0BD
:1054300090E00F941D1D8C01BE010E9463298CE534
:1054400093E0D80111969C938E9319961C921E920C
:1054500018971A870987DF91CF911F910F91FF90BD
:10546000EF90DF90CF90BF90AF909F908F90089576
:1054700088E090E00F941D1D8C01BE010E946329FD
:1054800084E393E0F80191838083E3CF8DE090E0A3
:105490000F941D1D8C01BE010E9463298CE093E0D6
:1054A000D8018D939C93C8010E94FCDED2CF89E085
:1054B00090E00F941D1D8C01FC01D383C28386EE06
:1054C00092E091838083CE010E941216D801159636
:1054D0009C938E93149784EE9DE018969C938E93E4
:1054E0001797CE010E94AA17892B09F4B2CF70E05A
:1054F00060E0CE010E943829F8018683882341F0BC
:10550000833009F0A6CF87E49DE090878783A1CF01
:105510008CE390E1908787839CCF8EE090E00F949E
:105520001D1D8C01DC011396DC93CE93129786EF40
:1055300093E08D939C93C8010E9475DF8ACF86E02B
:1055400090E00F941D1D8C01FC01D383C28380EC7D
:1055500092E091838083CE010E941216D8011596A5
:105560009C938E93149775CF86E090E00F941D1D49
:105570008C01FC01D383C2838AE992E0EACF8BE0FD
:1055800090E00F941D1D8C01FC01D383C28380ED3C
:1055900093E091838083168270E060E0CE010E94E8
:1055A000382997FD2DC0D80115969C938E9314979A
:1055B000D80114968D919C91009719F0863491052D
:1055C0002CF080E290E0F8019583848361E070E044
:1055D000CE010E94F22820E030E04AE754E40F9424
:1055E0008F260F940229611571058105910589F0B7
:1055F000D80117966D937D938D939C931A9729CF1D
:10560000919581959109F8019583848381E0868342
:10561000CFCF88E893E1A0E0B0E0F80187839087DE
:10562000A187B28716CF86E090E00F941D1DFC0184
:10563000D383C2838AEA93E09183808315821482A4
:10564000E114F10441F0D70118968C918F708630E7
:1056500011F4F582E482FA87E987FDCE84E090E0D8
:105660000F941D1DFC01D383C28324E833E03183F2
:1056700020839A878987EFCEC6010E94CCBE8A2DEF
:1056800090E0B0E0A0E0F70181879287A387B4871C
:105690008085807F8260808794CECF92DF92EF9268
:1056A000FF926A017B0163E0FC01808191810E948D
:1056B000C0F8FC01892BA9F080858D7091F4C0940D
:1056C000D094E094F094CC24CA9481859285A385EB
:1056D000B4858C219D21AE21BF2181879287A3872C
:1056E000B487FF90EF90DF90CF900895CF92DF9234
:1056F000EF92FF926A017B0163E0FC01808191815E
:105700000E94C0F8FC01892BA9F09085892F8D702B
:1057100089F4907F92609087CC24FF244185528544
:10572000638574854C295D296E297F2941875287BD
:1057300063877487FF90EF90DF90CF900895CF92AA
:10574000DF92EF92FF926A017B0163E0FC018081AE
:1057500091810E94C0F8009791F0FC0120852F7084
:10576000223069F461857285838594856C217D2161
:105770008E219F21FF90EF90DF90CF90089560E001
:1057800070E0CB01F7CFAF92BF92CF92DF92EF9252
:10579000FF920F931F93CF93DF93CDB7DEB7CD5614
:1057A000D1090FB6F894DEBF0FBECDBF5C01A7963E
:1057B0000FAFA797A8961FAFA897A9962FAFA99745
:1057C000AA963FAFAA97AB964FAFAB97AC965FAF99
:1057D000AC97AD966FAFAD97AE967FAFAE97239671
:1057E0001FAE1EAE2397FE01ED5BFF4F82E1DF018E
:1057F0001D928A95E9F772961192119287E0DF0166
:105800001D928A95E9F7CE018A599F4F0E94D822AE
:10581000F0FE2CC0A796EFADA797E83108F050C175
:10582000F0E08827E95EF34D8F4F0D94EA27662D4F
:105830002F2C5D2D602D602D5D2D2F2C602D602D6A
:10584000602D602D602D602D602D2F2C2F2C602D54
:10585000602D602D2F2C2F2C2F2C602D662D6BECA6
:105860007EE0CE018B5A9F4F0F9462200E942CF84D
:10587000882309F407C18091C40B811103C1C114AD
:10588000D10409F05EC030E020E043E050E060E485
:10589000CE0101960E9495DBD501ED91FC916081CE
:1058A00071814FE350E0CE0101960F94672CF1FE19
:1058B00010C1A7968FADA797823009F40AC1853031
:1058C00009F407C1A8968FADA89782958F709FE0C5
:1058D000980F9F70923018F0883009F0FAC001E0FC
:1058E00020E032E044E150E0BE016F5B7F4FCE012B
:1058F0008A599F4F0E94B720BE016F5B7F4FCE0138
:1059000001960F94E30463EB7EE089ED90E10F9440
:10591000A612BE016F5F7F4F89ED90E10F94B01129
:1059200060EB7EE089ED90E10F94A612BE016F5B03
:105930007F4F89ED90E10F94B01189ED90E10F94C4
:105940005510A8968FADA897807F87010027107209
:10595000882311F0F1FC04C00115110509F4F5C00C
:1059600030E020E043E050E060E4CE0101960E9488
:1059700095DBD501ED91FC91608171814FE350E0A1
:10598000CE0101960F94672CC114D10469F061E433
:1059900079E0CE0101960F94412C4FE350E0B6011F
:1059A000CE0101960F94672C61E479E0CE01019657
:1059B0000F94412C4FE350E063EA7EE0011511059E
:1059C00011F46FE97EE0CE0101960F947220A89643
:1059D0008FADA89782958F708450823008F09FC059
:1059E00067E1CE018A599F4F0E94011B6F962FAF2E
:1059F0006F97A0963FAFA097A1964FAFA197A296A1
:105A00005FAFA297A3966FAFA397A4967FAFA4971B
:105A1000A5968FAFA597A6969FAFA69700E020E02A
:105A200033E044E150E0BE016F5B7F4FCE018A5905
:105A30009F4F0E94B72069E97EE089ED90E10F94C5
:105A4000A612BE016F5F7F4F89ED90E10F94B011F8
:105A500066E97EE089ED90E10F94A612BE016F5BCE
:105A60007F4F89ED90E10F94B01189ED90E10F9493
:105A700055100E942CF8882329F08091C40B8823AC
:105A800009F455C0A701FF0C660B770BC5010E94F6
:105A9000762B90E080E0C359DF4F0FB6F894DEBF5D
:105AA0000FBECDBFDF91CF911F910F91FF90EF906F
:105AB000DF90CF90BF90AF90089567EC7EE0D1CE9D
:105AC00069EB7EE089ED90E10F94A612E894F0F87E
:105AD000CDCEF0FE36CF66968FAD6697882309F45B
:105AE00030CFBE016B5A7F4FCE0101960F94E30475
:105AF0006AEA7EE089ED90E10F94A612BE016F5F25
:105B00007F4F89ED90E10F94B01167EA7EE089ED57
:105B100090E10F94A612BE016B5A7F4F0ACF20E08E
:105B200032E0012B11F020E033E000E07ACFBE013B
:105B30006F5B7F4FCE0101960F94E30440E052E08B
:105B400060E070E0C5010E944D2BF0FE90C0A7966A
:105B5000EFADA797E150E53118F5F0E08827EC5458
:105B6000F24D8F4F0D94EA27BF2ED02DD02DD02D82
:105B7000D02DBF2ED02DD02DD02DD02DD02DD02D4D
:105B8000D02DC42EBC2ED02DD02DD02DC92DB62E6B
:105B9000B92E6CE87EE0CE018B5A9F4F0F946220A5
:105BA00030E020E043E050E060E4CE0101960E9446
:105BB00095DBD501ED91FC91608171814FE350E05F
:105BC000CE0101960F94672CC114D10469F061E4F1
:105BD00079E0CE0101960F94412C4FE350E0B601DD
:105BE000CE0101960F94672C61E479E0CE01019615
:105BF0000F94412C4FE350E066E77EE0CE01019622
:105C00000F94722060E77EE089ED90E10F94A61278
:105C1000BE016F5F7F4F89ED90E10F94B0116DE68B
:105C20007EE089ED90E10F94A612BE016B5A7F4F82
:105C300089ED90E10F94B01189ED90E10F9455102A
:105C40000E942CF8882309F41DCF8091C40B811188
:105C500019CFBE016B5A7F4FCE0101960F94E3041A
:105C600040E051E060E070E0C5010E944D2BF2FE83
:105C70007AC040E050E061E070E0C5010E949F2BD7
:105C8000672B682B692B09F482C065E67EE0CE01A4
:105C90008B5A9F4F0F94622030E020E043E050E0A9
:105CA00060E4CE0101960E9495DBD501ED91FC9157
:105CB000608171814FE350E0CE0101960F94672C13
:105CC000C114D10469F061E479E0CE0101960F942A
:105CD000412C4FE350E0B601CE0101960F94672CA2
:105CE00061E479E0CE0101960F94412C4FE350E03E
:105CF00062E57EE0CE0101960F9472206CE47EE0B6
:105D000089ED90E10F94A612BE016F5F7F4F89ED80
:105D100090E10F94B01169E47EE089ED90E10F9479
:105D2000A612BE016B5A7F4F89ED90E10F94B0111E
:105D300089ED90E10F9455100E942CF8882309F406
:105D4000A1CE8091C40B81119DCEBE016B5A7F4FB5
:105D5000CE0101960F94E30440E054E060E070E06F
:105D6000C5010E944D2B81E090E095CE67E87EE072
:105D700012CF63E87EE00FCF6AE77EE00CCFF5013B
:105D80008085853009F00CCF61E97EE004CF40E0EA
:105D900050E062E070E0C5010E949F2B672B682BEA
:105DA000692B19F06EE57EE072CF67E57EE06FCF7C
:105DB000AF92BF92CF92EF920F931F93CF93DF9347
:105DC000CDB7DEB7C856D1090FB6F894DEBF0FBE07
:105DD000CDBF5C01A2960FAFA297A3961FAFA3976A
:105DE000A4962FAFA497A5963FAFA597A6964FAFC1
:105DF000A697A7965FAFA797A8966FAFA897A99603
:105E00007FAFA9979E2D28E0FE01EF59FF4FDE01DD
:105E1000A75ABF4F01900D922A95E1F7A296EFADD8
:105E2000A297E150ED3008F0F2C0EC2CF0E08827AA
:105E3000E35EF04D8F4F0D94EA27942F9D2FFB2F9B
:105E40000530F12F2A2F8B2F07300730A62FB82FC0
:105E5000DE2FCB2F992331F0C5010E94C117009787
:105E600009F449C067E0CE01875A9F4F0E94011B89
:105E700062E07AE089ED90E10F94A6124AE050E0EA
:105E80006A966FAD6A9789ED90E10F94701067EF95
:105E900079E089ED90E10F94A612CE01875A9F4FC9
:105EA0000E94511FAB01BC012AE030E089ED90E176
:105EB0000F944F1189ED90E10F9455106A960FAD34
:105EC0006A976B961FAD6B976C962FAD6C976D961E
:105ED0003FAD6D976E964FAD6E976F965FAD6F97B6
:105EE000A0966FADA097A1967FADA197C5010E9426
:105EF000961F81E090E0C859DF4F0FB6F894DEBFDF
:105F00000FBECDBFDF91CF911F910F91EF90CF903A
:105F1000BF90AF900895911105C0C5010E94C117AF
:105F2000009749F366E09FCF992329F0C5010E94AD
:105F3000C117009701F362E096CF911105C0C5012A
:105F40000E94C1170097B9F261E08DCF40E050E0A8
:105F500061E070E0C5010E949F2B672B682B692BC5
:105F600029F4C5010E94C117009729F26BE07BCF8D
:105F700040E050E061E070E0C5010E949F2B672B7C
:105F8000682B692B31F0C5010E94C117009709F4F5
:105F9000B2CF6AE068CF40E050E062E070E0C50157
:105FA0000E949F2B672B682B692B31F0C5010E9443
:105FB000C117009709F49FCF6CE055CF40E050E047
:105FC00062E070E0C5010E949F2B672B682B692B54
:105FD00031F4C5010E94C117009709F48CCF6DE020
:105FE00042CF911106C0C5010E94C117009709F464
:105FF00082CF63E038CF992331F0C5010E94C117E9
:10600000009709F478CF65E02ECF64E02CCF90E0C4
:1060100080E071CFCF93C62F63E0FC018081918136
:106020000E94C0F8FC01892B21F19085892F8D7089
:1060300001F5907F9260908781859285A385B485D4
:106040008827BB278C2B81879287A387B48767ED2E
:1060500079E089ED90E10F94A6124AE050E06C2FB0
:1060600089ED90E10F94701089ED90E1CF910D943E
:106070005510CF910895CF92DF92FF920F931F9307
:10608000CF93DF93F12C6115710509F499C06A0172
:10609000EB018C01CB010E942D28F82E882309F4F6
:1060A0008FC0D2FE09C0D8018C918B3009F44BC04F
:1060B000E8F58A3009F44CC0D0FE09C0F8016081CF
:1060C00086EF860F843018F0CE010E940A30D1FE90
:1060D0006EC0D80114964D915D916D917C9117978A
:1060E00011968C9182958F70873038F0893008F442
:1060F0003EC08A50823008F46CC0CE010E94221645
:10610000EC81FD81309709F452C080858F709EEF3D
:10611000980F923010F081114AC0D80111969C91CD
:10612000907F80858F70892B808741C08C30B9F03B
:1061300040E050E062E070E08D3009F0BDCFCE016C
:106140000E94762BB9CF40E050E061E070E0F7CFDD
:1061500040E050E061E070E0CE010E944D2B40E055
:1061600050E062E070E0CE010E944D2BA5CFEC81A3
:10617000FD813097E1F080858F709EEF980F92300F
:1061800010F0811114C04187528763877487EC81B6
:10619000FD818085807F83608087EC81FD818085A3
:1061A000982F907F8F708067903609F4BDCF68EA92
:1061B00070E189ED90E10F94A612C8010E94D822E7
:1061C0008F2DDF91CF911F910F91FF90DF90CF9096
:1061D0000895CE010E942216EACF63E0FC0180817F
:1061E00091810E94C0F8009719F0FC018185089503
:1061F0008FEF0895AF92BF92CF92DF92EF92FF920E
:106200000F931F93CF93DF9300D000D01F921F9264
:10621000CDB7DEB76115710509F461C05A016B0194
:106220007C01CB010E942D28082F882379F1D6010B
:1062300014968D919C91009709F445C0FC0110853E
:10624000212F2F703EEF320F323010F0211130C06D
:1062500012951F70B0FE5BC0C6010E94ED30F701C1
:106260008083112391F11295107F81818F70182BFB
:106270001183D6011496ED91FC9181859285A385B9
:10628000B485F70184839583A683B783802F2896EE
:106290000FB6F894DEBF0FBECDBFDF91CF911F9137
:1062A0000F91FF90EF90DF90CF90BF90AF90089547
:1062B000253049F460E00E94C0F8009721F0DC012D
:1062C00018961C91C5CF10E0C5CFD6011496ED915C
:1062D000FC9180858F70823021F0833051F000E096
:1062E000D5CF4185528563857485C7010E94671D9E
:1062F000CDCF4185528563857485F70181818F708B
:10630000806781834483558366837783BFCF11235E
:10631000E1F21295107FF701A8CFAF92BF92CF9212
:10632000DF92EF92FF920F931F93CF93DF9300D0F2
:1063300000D01F921F92CDB7DEB75C017B0160FFDA
:1063400003C0E894E0F8F4F8F4FC0DC00E9416DDF8
:10635000663971058105910530F08091D90C9091D5
:10636000DA0C059719F5A70144275770052E000C84
:10637000660B770BC5010E94762B68E37EE089ED02
:1063800090E10F94A6128FEF9FEF28960FB6F89426
:10639000DEBF0FBECDBFDF91CF911F910F91FF9058
:1063A000EF90DF90CF90BF90AF90089519821A823E
:1063B0001B821C821D821E821F8218868A818F701A
:1063C0008A8340E053E0B501CE0101960E94FA3085
:1063D00040E057E060E070E0C5010E949F2BE62A94
:1063E000F72AD12CC12C09811A812B813C814D8146
:1063F0005E816F817885C5010E94C32BC6CFCF9384
:10640000DF93EC0140E053E060E070E00E949F2BDE
:10641000611571058105910599F02091D90C309194
:10642000DA0C2630310561F4CE010E948D3140E056
:1064300053E060E070E0CE01DF91CF910C944D2BE2
:10644000DF91CF9108958F929F92AF92CF92EF926A
:10645000FF920F931F93CF93DF9300D000D01F9232
:106460001F92CDB7DEB74C0109831A832B833C837F
:106470004D835E836F8378876EEF78E089ED90E1DE
:106480000F94A612CE0101960E94D8228981811113
:1064900030C00A810F70013089F140F1023019F0EB
:1064A00010E00530F1F5D401ED91FC9102A0F3A1CB
:1064B000E02D09811A812B813C814D815E816F81A4
:1064C0007885C401199581E090E028960FB6F8947C
:1064D000DEBF0FBECDBFDF91CF911F910F91FF9017
:1064E000EF90CF90AF909F908F900895CC24C3945D
:1064F000DACF813071F1823009F451C061EF78E078
:1065000089ED90E10F94A6124AE050E0698189ED8F
:1065100090E10F94701089ED90E10F94551001E017
:1065200010E061EE78E089ED90E10F94A6124AE068
:1065300050E0B80189ED90E10F94971189ED90E159
:106540000F945510CE0101960E94D82290E080E071
:10655000BCCFCE0101960E94CFF84497B8F46EE10B
:1065600070E0CE0101960E94B61EF4016281738133
:1065700040E052E0CE0101960E943B3060E072E1C3
:10658000D40112968D919C910E948D31D401ED9190
:10659000FC9102A0F3A1E02DCC24C3948ACF1D82EC
:1065A0001E821F821886D401ED91FC9102A0F3A1F6
:1065B000E02DCC24C39402E01A812B813C8140E081
:1065C0007DCF8F929F92AF92BF92CF92DF92EF9248
:1065D000FF920F931F93CF93DF93CDB7DEB76097F2
:1065E0000FB6F894DEBF0FBECDBF8C017B0140E03B
:1065F00058E060E070E00E949F2B672B682B692BAE
:1066000009F0A9C062E070E0C8010E9438296C015D
:1066100019861A861B861C861D861E861F86188A6A
:106620008A858F708A87D7FC96C040E052E0B80117
:10663000CE0109960E94FA3063E070E0C8010E9422
:106640003829AC011816190614F04FE350E081E028
:10665000C816D10429F4EF2CFF0CFF08FF2404C056
:1066600082E0C816D104D4F32FEF30E0D7010F94A5
:1066700001289A01550F440B550B0F94952749019A
:106680006901C8010E94ED30E82EF12C60E0CE01D6
:1066900009960E94E91D88169906F9F4CD2841F063
:1066A00082E0E816F10419F185E0E816F104F9F04A
:1066B00081E090E060960FB6F894DEBF0FBECDBFCC
:1066C000DF91CF911F910F91FF90EF90DF90CF90CE
:1066D000BF90AF909F908F900895CD2859F186E09C
:1066E000E816F10441F081E0E816F10421F061E0E0
:1066F000C8010E940A30B401CE0109960E94901D83
:1067000040E052E0B801CE0109960E943B3082E0A1
:10671000E816F10421F085E0E816F10429F460E0C0
:1067200071E0C8010E948D3160E072E0C8010E94F2
:106730008D31BECF85E0E816F10409F4B9CF82E0CF
:10674000E816F10409F4B4CF62E0C8010E940A30EF
:1067500060E071E0EBCF90E080E0ACCF81E090E0D2
:1067600008950F931F93CF93DF9300D000D01F9213
:106770001F92CDB7DEB719821A821B821C821D823E
:106780001E821F8218862A812F702A83FC010281B3
:106790001381C8010E94ED30813041F020F0823039
:1067A00011F0853081F490E080E002C081E090E05B
:1067B00028960FB6F894DEBF0FBECDBFDF91CF9104
:1067C0001F910F91089540E052E0B801CE0101966B
:1067D0000E94FA3060E0CE0101960E94E91DE8CFE8
:1067E0008F929F92AF92BF92CF92DF92EF92FF92E1
:1067F0000F931F93CF93DF93CDB7DEB767970FB695
:10680000F894DEBF0FBECDBF8C017B014C018BE045
:10681000880E911C9F8A8E8AF80112861186138633
:10682000148E138E672B09F463C0A090DB0CB0901C
:10683000DC0CA114B10409F45BC06FE270E0C70185
:106840000F944C2C6C01892B09F44AC0F701DE012E
:10685000119690E080E0BD012191222341F02F327A
:1068600031F08431910519F02D930196F5CF860F03
:10687000971FFC011082C5010E940EF8F801918358
:106880008083B6016F5F7F4F4FE050E0C4010F94EB
:10689000852CCE0146960E94F727F801948F838FAE
:1068A0008E899F89892B09F41386C8010E942D289F
:1068B000882319F0C8010E94862967960FB6F894BC
:1068C000DEBF0FBECDBFDF91CF911F910F91FF9023
:1068D000EF90DF90CF90BF90AF909F908F900895F2
:1068E000B701C5010E940EF8F80191838083DDCFC6
:1068F000F80111821082D9CFDC0119968D919C91FB
:10690000009739F0DC01ED91FC910280F381E02DDC
:1069100019940895CF93DF93EC01798368831A86E5
:1069200019861B861C8E1B8E0E942D28882329F019
:10693000CE01DF91CF910C948629DF91CF910895FC
:10694000CF93DF93EC01FB0124813581408151819C
:10695000628173810F944F11CE01DF91CF91089521
:10696000EF92FF920F931F93CF93DF9300D000D04D
:10697000CDB7DEB77C018B0167ED7EE089ED90E15C
:106980000F94A612D701ED91FC916081718189ED80
:1069900090E10F94B0116EEC7EE089ED90E10F94E0
:1069A000A612012E000C220B330B09831A832B83B2
:1069B0003C8380E190E09E838D83BE016F5F7F4FBB
:1069C00089ED90E10E94A0340F94551040E058E00A
:1069D00060E070E0C7010E94762B26960FB6F8940F
:1069E000DEBF0FBECDBFDF91CF911F910F91FF9002
:1069F000EF9008953F924F925F926F927F928F92A5
:106A00009F92AF92BF92CF92DF92EF92FF920F933D
:106A10001F93CF93DF93CDB7DEB72C970FB6F894C3
:106A2000DEBF0FBECDBF5C01362E972E3A01690145
:106A300068E37FE089ED90E10F94A6124AE050E010
:106A4000632D792D89ED90E10F94971160E37FE03C
:106A500089ED90E10F94A612C301B0E0A0E08F830E
:106A60009887A987BA8730E1432E512C5C864B86E4
:106A7000BE01695F7F4F89ED90E10E94A0344C0117
:106A80006CE27FE00F94A6124AE050E0B601C40128
:106A90000F94971164E27FE0C4010F94A612C7011E
:106AA000B0E0A0E089839A83AB83BC835E824D8291
:106AB000BE016F5F7F4FC4010E94A0340F94551038
:106AC0008091330B9091340B70E060E0892B09F0DA
:106AD00047C081E090E09093340B8093330B26E025
:106AE00040E855E260E070E087E49DE00E9493BBDF
:106AF0003092DE0E87E49DE09093DD0E8093DC0EF5
:106B00001092E90F1092EB0F1092EA0F013011056D
:106B100009F44EC00CF041C0012B09F44EC0C11461
:106B2000D10409F457C082E0C816D10409F062C04C
:106B30007092640F6092630F1092660F1092650F4F
:106B4000F092680FE092670F86E00F947006109243
:106B5000340B1092330B882309F456C0682F70E071
:106B6000C5010E94B03490E080E02C960FB6F894F6
:106B7000DEBF0FBECDBFDF91CF911F910F91FF9070
:106B8000EF90DF90CF90BF90AF909F908F907F90CD
:106B90006F905F904F903F9008950330110581F002
:106BA0000430110509F0BBCFFE24EF24FE24B7CF3B
:106BB000FE2CEE24EE24EA94B2CFFF24FA94AFCF59
:106BC000EF2821F492E0E92EF12CEECFEE24E394AD
:106BD000F12CEACF7092640F6092630F90E080E036
:106BE000EE2011F080E09FEF9093660F8093650F89
:106BF00085E0ABCF68E07FE089ED90E10F94A612CD
:106C00001092340B1092330B81E090E0AECF2F92B4
:106C10003F924F925F926F927F928F929F92AF922C
:106C2000BF92CF92DF92EF92FF920F931F93CF9379
:106C3000DF93CDB7DEB72C970FB6F894DEBF0FBE4B
:106C4000CDBF5C0109831A832B833C834D835E8314
:106C50006F837887CE0101960E94CFF81C01023025
:106C600011F0053011F4312C212CF5010281138132
:106C7000F80180858F70853009F07FC0C8010E94BF
:106C800052F9E82EF12CF2E0EF16F1040CF475C085
:106C900060E0C8010E94C0F8FC01818592859C8754
:106CA0008B8761E0C8010E94C0F8FC0141845284D6
:106CB0006384748488248A94982CF2E0EF16F1049B
:106CC00059F062E0C8010E94C0F8FC0181849284FE
:106CD000F3E0EF16F104A1F48FE390E09A8789873F
:106CE00092E0C92ED12C29853A85D1010F94F9273C
:106CF00024E630E040E050E00F94952779011CC075
:106D000063E0C8010E94C0F8FC01818592859A87E2
:106D1000898782E0C82ED12CF4E0EF16F10439F017
:106D200064E0C8010E94C0F8FC01C184D284898556
:106D30009A857101892BB9F684019601A2016B85B0
:106D40007C85C5010E94FA342C960FB6F894DEBFFC
:106D50000FBECDBFDF91CF911F910F91FF90EF90AC
:106D6000DF90CF90BF90AF909F908F907F906F906B
:106D70005F904F903F902F90089590E080E0E4CF97
:106D80008F929F92AF92BF92DF92EF92FF920F93FA
:106D90001F93CF93DF93CDB7DEB7A5970FB6F894C7
:106DA000DEBF0FBECDBF7C010E8F1F8F28A339A37E
:106DB0004AA35BA36CA37DA3CE014E960E940A1F3B
:106DC0004B015C01D7011296ED91FC9180858F708B
:106DD000843009F0E9C0102F61857285CE010196DB
:106DE0000E94F033CE0101960E942D28882309F4D9
:106DF0004AC08985893009F046C070E060E0CE0164
:106E000001960E943829082FD92E6BEF7EE089ED7C
:106E100090E10F94A6124AE050E0602F7D2D89ED9D
:106E200090E10F94971169EF7EE089ED90E10F9466
:106E3000A612B501A40189ED90E10F947E1063EFD5
:106E40007EE089ED90E10F94A612612F70E04AE098
:106E500050E089ED90E10F94971189ED90E10F9446
:106E600055108091330B9091340B892B29F140E020
:106E700053E0B701CE014E960E943B3070E060E0D7
:106E8000C7010E94B03410E000E0CE0101960E94DC
:106E90007C34C801A5960FB6F894DEBF0FBECDBFF7
:106EA000DF91CF911F910F91FF90EF90DF90BF90F6
:106EB000AF909F908F90089581E090E09093340B75
:106EC0008093330B26E040E855E260E070E087E411
:106ED0009DE00E9493BB0093DE0E87E49DE09093BB
:106EE000DD0E8093DC0E1092E90F1092EB0F1092E2
:106EF000EA0FE981FA81153021F01F3011F01230CC
:106F000011F580858F70808770E060E083ED97E0F9
:106F10009093640F8093630F1092660F1092650F29
:106F20007093680F6093670F86E00F94700610925D
:106F3000340B1092330B01E010E0882309F4A5CF45
:106F4000682F70E09DCF80858F708061808722E5FB
:106F500038EB42E152E4C501B4010F941D2820E052
:106F600030E040E251E40F948F262DEE3EE94CE3F1
:106F70005EE30F9489284B015C0120E030E0A90119
:106F80000F94312920E030E040E05FE387FD07C047
:106F9000C501B4010F941D280F94FB28B7CFC5017C
:106FA000B4010F941C28F8CF10E000E072CFCF920C
:106FB000DF92EF92FF920F931F93CF93DF9300D056
:106FC00000D01F921F92CDB7DEB77C0109831A83D0
:106FD0002B833C834D835E836F837887CE0101963C
:106FE0000E94CFF88C018981882359F09A819F7083
:106FF000923008F0BAC0823011F0853011F410E000
:1070000000E070E060E0C7010E943829D82EC92E48
:107010006BEE7EE089ED90E10F94A6124AE050E01D
:107020006D2D7C2D89ED90E10F94971169EE7EE036
:1070300089ED90E10F94A6124AE050E0B80189ED85
:1070400090E10F94971189ED90E10F945510809184
:10705000330B9091340B892BE9F040E053E0B701FA
:10706000CE0101960E943B3070E060E0C7010E94B3
:10707000B03490E080E028960FB6F894DEBF0FBEE3
:10708000CDBFDF91CF911F910F91FF90EF90DF90D7
:10709000CF90089581E090E09093340B8093330B70
:1070A00026E040E855E260E070E087E49DE00E9461
:1070B00093BBD092DE0E87E49DE09093DD0E80932B
:1070C000DC0E1092E90F1092EB0F1092EA0F80ED98
:1070D00097E09093640F8093630F1092660F109265
:1070E000650F01151105E1F185E090E09093680FBF
:1070F0008093670F86E00F947006D82E64E670E0E8
:1071000080E090E00F944602D1100AC062EE7EE06B
:1071100089ED90E10F94A61289ED90E10F9455103E
:1071200082ED97E09093640F8093630F1092660F47
:107130001092650F24E6209FC001219F900D11241D
:107140009093680F8093670F86E00F9470061092FB
:10715000340B1092330B882359F0682F70E086CFE0
:107160001092680F1092670FC5CF8FEF9FEF83CFFC
:1071700081E090E080CFEF92FF920F931F93CF9327
:10718000DF93EC018B011D821C821A821B82E88036
:10719000F980E114F10409F45DC080912E0B909107
:1071A0002F0B892B09F456C0672B09F48701F801CE
:1071B00080858F708630A9F46CE178E0C8010E9468
:1071C0000EF8009719F0FC0181858A836BE379E062
:1071D000C8010E940EF8009709F443C0FC018185A4
:1071E0008B836EE176E0C7010E940EF8009779F577
:1071F0006DE079E089ED90E10F94A6124AE050E04D
:107200006B8189ED90E10F9470106BE079E089ED6E
:1072100090E10F94A6124AE050E06A8189ED90E176
:107220000F94701089ED90E10F94551020E030E03C
:10723000A9016EE176E0888199810E94DDFB6EE113
:1072400076E0888199810E940EF8009719F00996DE
:107250009D838C83DF91CF911F910F91FF90EF90D1
:107260000895F801808191810F94ED1FB9CFAF92FD
:10727000BF92CF92DF92EF92FF920F931F93CF9323
:10728000DF9364E070E041E050E00091E70A109184
:10729000E80A2091E90A3091EA0ACA01052E000C99
:1072A000AA0BBB0B80239123A223B323892B8A2B08
:1072B0008B2BD9F0C090E70AD090E80AE090E90A59
:1072C000F090EA0ACA0180959095092E000CAA0B4D
:1072D000BB0B8C219D21AE21BF218093E70A9093A7
:1072E000E80AA093E90AB093EA0A440F551F6150D7
:1072F000710959F68091E30A9091E40AA091E50A98
:10730000B091E60A892B8A2B8B2B09F47DC00F9450
:1073100046049B01AC016091E30A7091E40A8091FC
:10732000E50A9091E60AA12CB12C65011CE2E12E40
:10733000FF24F39400E010E00E94B8D5882309F4FC
:1073400063C01092E30A1092E40A1092E50A1092C8
:10735000E60A8091240B9091250B892B09F183E09B
:10736000E82EF12CD0E0C0E0E091240BF091250B49
:10737000EE0DFF1D008110E0DF0111972C9130E030
:1073800011974C9150E03397608170E0CE010E94DC
:10739000FA1984E0E80EF11C2196C430D10521F7DA
:1073A000C1E0D0E080912E0290912F028C179D07B2
:1073B00048F580912E0290912F02E091D80BF09128
:1073C000D90BE80FF91F4AE050E0608189ED90E1A8
:1073D0000F94701061E276E089ED90E10F94B011A6
:1073E0002196C131D105F1F689ED90E1DF91CF9180
:1073F0001F910F91FF90EF90DF90CF90BF90AF90D3
:107400000D945510CE01D9CFDF91CF911F910F91DF
:10741000FF90EF90DF90CF90BF90AF9008954F9284
:107420005F926F927F92AF92BF92CF92DF92EF9274
:10743000FF920F931F93CF93DF93CDB7DEB76D9776
:107440000FB6F894DEBF0FBECDBF20912E0B30914A
:107450002F0BFF24F394232B09F41EC1811149C083
:10746000FF24F39461ED71E189ED90E10F94A61290
:1074700089ED90E10F9455108091220B8F5F8093DE
:10748000220BE091DB0CF091DC0C309709F48DC0FD
:10749000068117810115110509F491C0D8011896CC
:1074A0008C918F70853009F5C8010E9452F98823AC
:1074B000E1F0F80160817181CE0101960E94F03304
:1074C000CE0101960E942D28882359F08A859B853C
:1074D000009739F0DC01ED91FC910284F385E02DF9
:1074E0001995CE0101960E947C34F8010281138126
:1074F000D1CF6AE072E189ED90E10F94A61289ED97
:1075000090E10F9455100F9446042B013C0180919B
:10751000D50C882381F10F9446049B01AC01A12C6A
:10752000B12C650110E1E12E17E2F12E00E010E030
:10753000C301B2010E94B8D581111DC00E9478BE5E
:107540008091DF0C811128C00E9437398091D90CBD
:107550009091DA0C059741F08091DB0C9091DC0C56
:10756000892B11F00E9447860E94138782E090E0E9
:107570000E941E82CCCF8091D50C882309F470CF55
:1075800067EE71E184E390E10F94A61284E390E149
:107590000F945510F12C66CF8091DD0C9091DE0C8C
:1075A000892B91F20E947EE2CFCF61EC71E189EDEF
:1075B00090E10F94A61289ED90E10F94551010926E
:1075C0002D0B10922C0B69EB71E189ED90E10F947A
:1075D000A61289ED90E10F94551064E670E080E00A
:1075E00090E00F94460210922B0B61EA71E189ED55
:1075F00090E10F94A6120E9416DDAB01BC012AE0B7
:1076000030E089ED90E10F94531080912E0B909112
:107610002F0B009711F00E9480FD10922F0B1092FB
:107620002E0B1092D80C1092D70C1092DC0C1092EA
:10763000DB0C1092C30B1092C20B1092290B10920C
:10764000280B1092C10B1092C00B1092270B1092B6
:10765000260B1092DE0C1092DD0C1092320B109261
:10766000310B6CE971E189ED90E10F94A6120E9453
:1076700016DDAB01BC012AE030E089ED90E10F940A
:10768000531089ED90E10F94551010922A0B8091C0
:10769000220B81508093220B8F2D6D960FB6F8949C
:1076A000DEBF0FBECDBFDF91CF911F910F91FF9035
:1076B000EF90DF90CF90BF90AF907F906F905F90F2
:1076C0004F900895FC016115710519F4848195812D
:1076D000089586819781681779072CF084819581B8
:1076E000860F971F0895828193810C943829EF9219
:1076F000FF920F931F93CF93DF93DC011296ED91CE
:10770000FC91309709F17A018B01EC016DED75E088
:10771000808191810E940EF80097B1F0FC012085D4
:107720002F70243089F461857285E881F98104889D
:10773000F589E02D9701A801CE01DF91CF911F912E
:107740000F91FF90EF90199490E080E0DF91CF913E
:107750001F910F91FF90EF900895EF92FF920F937A
:107760001F93CF93DF93CDB7DEB760970FB6F89432
:10777000DEBF0FBECDBF8C017901CE0101960E9404
:10778000BDDCA701BE016F5F7F4FC8010E94773B40
:1077900060960FB6F894DEBF0FBECDBFDF91CF91DC
:1077A0001F910F91FF90EF9008952F923F924F926B
:1077B0005F926F927F928F929F92AF92BF92CF9281
:1077C000DF92EF92FF920F931F93CF93DF93CDB78A
:1077D000DEB7A6970FB6F894DEBF0FBECDBF1C0173
:1077E0000F8B188F298F3A8F4B8F5C8F6D8F7E8F09
:1077F00022E1E216F10408F035C0F701EE50FB4F2C
:1078000030813F8FCE0147960E94952097FD04C09E
:10781000BC01C1010E942623988D892F8F70D10150
:107820001196EC911197E07FE82B1196EC9311974C
:107830008F898C93E295EF70EC3008F063C0F0E034
:107840008827EA5DF34C8F4F0D94EA27293E4F3C81
:107850004F3CC73D343C553E903DD13DD13DD13D9F
:10786000903D903D1F8ECECFB12C92959F709D3054
:1078700008F0CDC4E92FF0E08827EE5BF34C8F4F82
:107880000D94EA27823C8F3EAF3E8F3E583E583ED5
:107890008F3E8F3E074107418F3E8F3E5C3D929564
:1078A0009F709D3008F018C1E92FF0E08827E45A56
:1078B000F34C8F4F0D94EA27823C3A3D2D3DF03C2E
:1078C0006C3C693C113D3C3D6C3D6C3DFB3CFB3CE4
:1078D0005C3D8E8DF10187838D8DD10116968C9341
:1078E00016978C8D15968C9315978B8D14968C937B
:1078F00014979295907F11968C9111978F70982B79
:1079000011969C93BF8DBB2309F467C0F10181815F
:1079100082958F702B2F30E08217130609F45DC01B
:1079200066E170E189ED90E10F94A612D101119604
:107930006C9162956F704AE050E089ED90E10F9490
:10794000701063E170E189ED90E10F94A6124AE0B6
:1079500050E06F8D89ED90E10F94701061E170E15E
:1079600089ED90E10F94A612F101008119821A822B
:107970001B821C821D821E821F8218868F8D82951B
:10798000807F9A819F70892B8A830983EE24EA94F1
:10799000FE2C11812281338144815581668177815A
:1079A000CE0101960E94D53BD1012C9311963C93B8
:1079B000119712964C93129713965C931397149603
:1079C0006C93149715967C93159716968C9316972F
:1079D00017969C93C1010E94D82288E0F10178C1DA
:1079E0008D8D9E8DF1018683878190FB80F9878341
:1079F0008C8D858387CF8B8D9C8DAD8DBE8DB7FD96
:107A00000EC08F3F9105A105B10529F024F08FEF3D
:107A100090E0A0E0B0E0D10114968C9373CF80E0A9
:107A2000FACF6B8D7C8D8D8D9E8D20E06D39BFEFF3
:107A30007B078B079B076CF02FEF6115E4E67E0751
:107A40008105910534F424E630E040E050E00F94E5
:107A50009527D10114962C9355CF8D8D9E8DF101D4
:107A60008683878190FB80F987838C8D85838B8DBE
:107A7000848348CF8B8DCFCFCB8CDC8CED8CFE8C70
:107A800020E030E0A901C701B6010F94292660E08B
:107A900087FD0FC020E030E04FE753E4C701B60197
:107AA0000F9431296FEF181624F0C701B6010F9417
:107AB0000229F101648326CFD10111968C9111978F
:107AC0008F70806C11968C9311978B8D9C8D159671
:107AD0009C938E93149716CF66E970E189ED90E13F
:107AE0000F94A612688D62956F704AE050E089EDA0
:107AF00090E10F94701063E970E189ED90E10F94CB
:107B0000A612F101618162956F704AE050E089ED43
:107B100090E10F94701089ED90E10F945510F2CE22
:107B200092959F70933091F09C3031F24B8D5C8D2B
:107B30006D8D7E8DF10144835583668377839295A5
:107B4000907F81818F70982B9183DCCE60E0C101A2
:107B50000E94E91DD10114968C9314978D8D9E8DF2
:107B600016968C93169717968C91179790FB80F921
:107B700017968C9317978C8D15968C931597119655
:107B80008C9111978F70806211968C93BBCE60E0C0
:107B9000CE0147960E94E91DD10114968C9314974B
:107BA000EECF92959F709D3008F066C0E92FF0E00F
:107BB0008827E252F24C8F4F0D94EA27823CF93D20
:107BC000283EA63D283E283EEB3D183E183E183E76
:107BD000073E133E5C3D8B8D9C8DAD8DBE8DF101BE
:107BE00084839583A683B78381818F708066818328
:107BF00089CE6B8D70E090E080E00F942E26D1014D
:107C000014966D937D938D939C9317977BCE6B8D7C
:107C10007C8D8D8D9E8D0F943026F101648375834C
:107C2000868397836FCE6B8D7C8D8D8D9E8DE5CFFA
:107C30009295907FF10181818F70982B91838B8D2C
:107C40009C8DAD8DBE8D84839583A683B7835ACEDC
:107C50009295907FD10111968C9111978F70982BEE
:107C600011969C938B8D9C8DAD8DBE8DF10184837F
:107C70009583A683B78346CE61E870E189ED90E1F4
:107C80000F94A612688D62956F704AE050E089EDFE
:107C900090E10F9470106EE770E189ED90E10F9420
:107CA000A612D10111966C912ECFBB24B394DDCDD9
:107CB0004B8D5C8D6D8D7E8DF10144835583668384
:107CC00077839295907F81818F70982B918388E044
:107CD000DE01119601900D928A95E1F729813A8192
:107CE0004B815C816D817E818F819885A6960FB6D0
:107CF000F894DEBF0FBECDBFDF91CF911F910F91E2
:107D0000FF90EF90DF90CF90BF90AF909F908F90BB
:107D10007F906F905F904F903F902F900895963096
:107D200009F442C148F46B8D913071F06FEF70E04F
:107D3000933051F060E008C0973009F441C19A5087
:107D40006B8D7C8D9230B0F784E68D8F8E8D8E7F1B
:107D50008E8F1C8E888D8F708062888F6B8F2C8D9C
:107D600030E0AFEFB0E00F94C727C12CD12C7601E3
:107D7000CA946115F4E67F078105910544F424E671
:107D800030E040E050E00F94952769017A018601C8
:107D90002B8D28A3622E712CBB2009F475C08E8D0B
:107DA0008695A82FA150BB0B2D01BFEF4B165B068C
:107DB00009F027C1003811050CF009C18FE790E0E8
:107DC0008C199D09869DD001879DB00D969DB00DA3
:107DD00011242FEF30E00F94012821E83EE740E026
:107DE00050E00F949527F1012783ABE9B0E0A7019C
:107DF00096010F94B427EFE78E2E912CA12CB12C75
:107E0000A50194010F94952789019A010C591F4FE0
:107E10002F4F3F4FAEEFB1E0A70196010F94B4276B
:107E2000A50194010F949527D3010F94B4272FEF48
:107E300030E040E050E00F94952739012FEF6216B3
:107E4000710421F01CF066246A94712C61E770E1E2
:107E500089ED90E10F94A6124AE050E0B80189ED57
:107E600090E10F94971163E670E189ED90E10F9432
:107E7000A6124AE050E0B30189ED90E10F9497110A
:107E800089ED90E10F94551030E020E050E040E0A3
:107E900070E060E0CE0101960E94F5BBF02E2D8DC2
:107EA0003E8D3170AFEFBFEF0F94C7272DE631E065
:107EB00040E050E00F94952744275527AAEFB5E0FE
:107EC0000F94B427DC01CB019058AF4FBF4FCD01C9
:107ED000BB2797FDB095AB2F8E3FE1E09E0708F0E2
:107EE0006FC1382F8F3F910508F48CC14EEF481BAE
:107EF00050E03FEFF301319611270F5F1F4FF094D1
:107F0000EF2CF12C309FC001319F900D1124292FAF
:107F100033272E0D3F1DDF010F9401284B015C011B
:107F20008824AA24BB24509F9001519F300D112416
:107F3000232F33272E0D3F1D0F940128BB27A92F78
:107F4000982F872F882A992AAA2A409F9001419F1B
:107F5000300D1124232F33272E0D3F1DDF010F94E9
:107F60000128B82FA72F962F882788279927BB2766
:107F700088299929AA29F101A6839583848367E337
:107F800070E189ED90E10F94A612C1010E94D82200
:107F90008A859B850F94B91D8F81988597FDB2CCFA
:107FA00060E00F940100AECC6B8D7C8D8D8D9E8D2D
:107FB00024E630E040E050E00F949527B901C4CEAC
:107FC0006B8D7C8D8D8D9E8D0F94FB28BDCEA70172
:107FD00096012058310941095109ABE9B0E00F94ED
:107FE000B4272FE730E040E050E00F949527890157
:107FF0009A010C591F4F2F4F3F4FD10117961C92DA
:1080000025CF9201AAEBBFEF0F94F92744E6842E07
:10801000912CA12CB12CA50194010F949527DA0184
:10802000C9018C599F4FAF4FBF4F89A39AA3ABA3F0
:10803000BCA326E430E0D2010F940128A5019401ED
:108040000F94952749015A019EE1890E911CA11CAC
:10805000B11C003811050CF099C08FE790E08C1925
:108060009D09869DD001879DB00D969DB00D112470
:10807000A50194010F94BF279B01AC01AFEFB0E0C5
:108080000F94B42724E63AE640E050E00F94952799
:10809000D10117962C9329A13AA14BA15CA12C0DDB
:1080A0003D1D4E1D5F1DAEEFB1E00F94B42723EED2
:1080B00030E040E050E00F94952729013A013EA3BB
:1080C0002DA3AFEFB0E0A70196010F94B4272FE7DF
:1080D00030E040E050E00F9495278901E8A1AE2FF1
:1080E000B0E0A30192010F94B4272FEF30E040E0FD
:1080F00050E00F94952739012F3F310521F01CF0F6
:1081000066246A94712C6DE570E189ED90E10F941D
:10811000A6122AE030E049A15AA16BA17CA189ED09
:1081200090E10F944F1167E570E189ED90E10F94B4
:10813000A6122AE030E0B501A40189ED90E10F9488
:108140004F116FE470E189ED90E10F94A6124AE0BF
:1081500050E0B80189ED90E10F94971167E470E168
:1081600089ED90E10F94A6124AE050E0B30189ED49
:1081700090E10F9497116EE370E189ED90E10F9417
:10818000A6124AE050E06DA17EA176CEA70196012D
:108190002058310941095109ABE9B0E00F94B427E7
:1081A0002FE730E040E050E00F94952789019A01D5
:1081B0000C591F4F2F4F3F4FD10117961C92A3CF41
:1081C0008C3FF3E09F0768F48D3F22E0920728F48C
:1081D00052E0580F3FEF40E08DCE3CEF381B5FEF91
:1081E000FACF8A3F35E0930781F08B3FE4E09E07AA
:1081F00028F444E0480F5FEF30E07CCE5AEF581B84
:1082000030E001C050E04FEF75CE50E0F9CF65E2AD
:1082100070E189ED90E10F94A612688D62956F7000
:108220004AE050E089ED90E10F94701062E270E155
:1082300034CD2F923F924F925F926F927F928F92A6
:108240009F92AF92BF92CF92DF92EF92FF920F93E5
:108250001F93CF93DF93CDB7DEB7C45CD1090FB6C0
:10826000F894DEBF0FBECDBF1C01C755DF4F08839A
:10827000C95AD040C655DF4F1883CA5AD040C55599
:10828000DF4F2883CB5AD040C455DF4F3883CC5AB8
:10829000D040C355DF4F4883CD5AD040C255DF4F41
:1082A0005883CE5AD040C155DF4F6883CF5AD04053
:1082B000C055DF4F7883C05BD040CF54DF4FF98289
:1082C000E882C15BD040C554DF4FC882CB5BD04051
:1082D000C454DF4FA882CC5BD0400E9416DD6B01F6
:1082E000C354DF4F79836883CD5BD040683C710510
:1082F000B4F46BE87CE084E390E10F94A6124AE0CA
:1083000050E0B60184E390E10F94971184E390E18B
:108310000F945510AA24AA94BA2C0C942A4B0F94AB
:108320004604CF53DF4F688379838A839B83C15C84
:10833000D040C655DF4F8881CA5AD0408F70282F51
:1083400030E0C954DF4F39832883C75BD040809128
:10835000D90C9091DA0CC154DF4F99838883CF5B9D
:10836000D040CF54DF4FE881F981C15BD0403097D6
:1083700021F0808181110C946D50D1011B968C915C
:10838000882341F0C1010B96CF54DF4F9983888336
:10839000C15BD040C954DF4FE881F981C75BD04051
:1083A000EF2B11F00C94C950CF54DF4FE881F981C5
:1083B000C15BD040309711F00C947650D1015B96A0
:1083C0000D90BC91A02DC954DF4FB983A883C75B22
:1083D000D040AB2B11F40C94C950C655DF4F8881A7
:1083E000CA5AD0408F7011F00C94C950C954DF4F55
:1083F0006881C75BD040CE0187559F4F0E94DA1A33
:10840000C756DF4F2883C959D040C656DF4F38833F
:10841000CA59D040C556DF4F4883CB59D040C456C7
:10842000DF4F5883CC59D040C356DF4F6883CD59B6
:10843000D040C256DF4F7883CE59D040C156DF4F6F
:108440008883CF59D040C056DF4F9883C05AD04060
:108450000C94C950D1018D919C91892B09F45ACF6C
:10846000C954DF4F08811981C75BD0400430110522
:1084700099F5C454DF4FE880CC5BD040C755DF4F3F
:108480000881C95AD040C655DF4F1881CA5AD0401A
:10849000C555DF4F2881CB5AD040C455DF4F3881B6
:1084A000CC5AD040C355DF4F4881CD5AD040C25539
:1084B000DF4F5881CE5AD040C155DF4F6881CF5A27
:1084C000D040C055DF4F7881C05BD040C1010E94D1
:1084D000961F5C010C942A4BC755DF4F1881C95A6F
:1084E000D040143009F410C348F4112309F469C0D2
:1084F000912C812CAA24AA94BA2C8AC388EF810FCC
:108500008230B0F788E0FE01E755FF4FDE0111969B
:1085100001900D928A95E1F7C655DF4F8881CA5ABE
:10852000D040807F09F483C3CE0187559F4F0E94BE
:1085300049204B015C0181149104A104B10409F4A8
:1085400076C3193041F4B094A09490948094811C27
:10855000911CA11CB11CB101CE0187559F4F0F94F6
:10856000D51360E0CE0187559F4F0E94011B6A968C
:108570002FAF6A976B963FAF6B976C964FAF6C9728
:108580006D965FAF6D976E966FAF6E976F967FAF7C
:108590006F97A0968FAFA097A1969FAFA197C95450
:1085A000DF4FA881B981C75BD040A230B10509F483
:1085B00098C30CF042C3AB2B09F4D1C3912C812C8E
:1085C00056C519821A821B821C821D821E821F823E
:1085D00018868A818F708A83C655DF4F8881CA5A70
:1085E000D040807F09F484CFC954DF4F288139817E
:1085F000C75BD0402A30310509F43EC254F421153E
:10860000310569F12230310509F4E0C0912C812C4B
:108610002AC2C954DF4F88819981C75BD0408B3013
:10862000910509F4D1C10C9789F7B101CE010196EA
:108630000F94D513CE0187559F4F0E949520BC0102
:10864000CE0101960E94262388E0FE013196DE01CC
:10865000A755BF4F01900D928A95E1F701C2EF2B0C
:1086600059F068E47CE089ED90E10F94A61289ED61
:1086700090E10F945510CACFC1010E94E5518C01C1
:1086800061E070E01816190614F070E060E04AE04E
:1086900050E089ED90E10F9497116CEC76E089ED54
:1086A00090E10F94B011CE0187559F4F0E94511F4A
:1086B000AB01BC012AE030E089ED90E10F944F114D
:1086C00089ED90E10F945510CE0187559F4F1016FC
:1086D000110614F00C945B500E94511F672B682BFD
:1086E000692B09F068C162E0CE0187559F4F0E9457
:1086F000011BCF56DF4F2883C159D040CE56DF4FE4
:108700003883C259D040CD56DF4F4883C359D0403B
:10871000CC56DF4F5883C459D040CB56DF4F6883C7
:10872000C559D040CA56DF4F7883C659D040C95684
:10873000DF4F8883C759D040C856DF4F9883C85948
:10874000D04088248394982C91E0CD54DF4F9883B7
:10875000C35BD0405524539442C061E0CE0187559D
:108760009F4F0E94011BC757DF4F2883C958D04035
:10877000C657DF4F3883CA58D040C557DF4F4883AC
:10878000CB58D040C457DF4F5883CC58D040C35744
:10879000DF4F6883CD58D040C257DF4F7883CE5823
:1087A000D040C157DF4F8883CF58D040C057DF4FEC
:1087B0009883C059D04088248394982CA1E0CD544C
:1087C000DF4FA883C35BD040512C09C0912C812C72
:1087D000CD54DF4F1882C35BD04055245A94B10169
:1087E000CE0101960F94D5138A81982F92959F7090
:1087F000945F9F70923060F4C655DF4F9881CA5ADB
:10880000D04092959F70923019F48F7080628A8365
:10881000F1019085973071F4C655DF4F8881CA5AAF
:10882000D040807E803211F0803421F48A818F70B4
:1088300080628A83F101A185B285892F90E010972B
:1088400041F0ED91FC911197068CF78DE02DCD0153
:1088500019957C01C755DF4F0881C95AD040C655CC
:10886000DF4F1881CA5AD040C555DF4F2881CB5AF7
:10887000D040C455DF4F3881CC5AD040C355DF4F6C
:108880004881CD5AD040C255DF4F5881CE5AD04092
:10889000C155DF4F6881CF5AD040C055DF4F788136
:1088A000C05BD040CE0101960E94D53BCF57DF4F31
:1088B0002883C158D040CE57DF4F3883C258D040AC
:1088C000CD57DF4F4883C358D040CC57DF4F588334
:1088D000C458D040CB57DF4F6883C558D040CA57E3
:1088E000DF4F7883C658D040C957DF4F8883C758B9
:1088F000D040C857DF4F9883C858D040CE0101966A
:108900000E94D822CD54DF4FF881C35BD040FF23B3
:1089100051F1C655DF4F8881CA5AD04082958F7079
:108920009FE0980F9F70923020F08A5F8F708230A6
:10893000D0F48A8182958F7081508230A0F42D818D
:1089400030E0AFEFB0E00F94C7272FEF611504E6DA
:1089500070078105910534F424E630E040E050E0F2
:108960000F9495272D8388E0FE013196DE01A755EF
:10897000BF4F01900D928A95E1F712E1912AF12CF7
:10898000AA24AA94BA2CD10118968C9118978730F2
:1089900009F089C5C354DF4FE881F981CD5BD04030
:1089A000EE35F1400CF090C364E07CE084E390E1AC
:1089B0000F94A612ABCC912C812CB1E0CD54DF4F9B
:1089C000B883C35BD040C6CEB101CE0101960F94EF
:1089D000D513C255DF4F8881CE5AD0409A819295E7
:1089E0009F7039F0923049F0912C812CFF24F39440
:1089F0003BC09A819F7090629A8390E08536910582
:108A000014F084E690E08E8388E0FE013196DE016A
:108A1000A755BF4F01900D928A95E1F762E0CE0114
:108A200087559F4F0E94DA1AEA962FAFEA97EB9686
:108A30003FAFEB97EC964FAFEC97ED965FAFED97AE
:108A4000EE966FAFEE97EF967FAFEF97C158DF4F7F
:108A50008883CF57D040C058DF4F9883C058D0404C
:108A6000812CF2E19F2EF12CCD54DF4F1882C35B95
:108A7000D04055245A9484CFB101CE0101960F9471
:108A8000D513C155DF4F6881CF5AD040C055DF4F55
:108A90007881C05BD0407170CE0101960E94612345
:108AA000CD54DF4F8883C35BD040912C812CFF24B1
:108AB000F3948823F1F288E0FE013196DE01A75598
:108AC000BF4F01900D928A95E1F762E0CE01875584
:108AD0009F4F0E94DA1AE2962FAFE297E3963FAFDC
:108AE000E397E4964FAFE497E5965FAFE597E69698
:108AF0006FAFE697E7967FAFE797E8968FAFE89777
:108B0000E9969FAFE997ACCFC954DF4F28813981EF
:108B1000C75BD0402930310509F461C0C1010E9412
:108B2000E5511816190674F562E0CE0187559F4F7E
:108B30000E94011BAA962FAFAA97AB963FAFAB97A7
:108B4000AC964FAFAC97AD965FAFAD97AE966FAFAB
:108B5000AE97AF967FAFAF97E0968FAFE097E19675
:108B60009FAFE19788248394982CAA24AA94BA2CC6
:108B7000F12C31E0CD54DF4F3883C35BD040552416
:108B8000539401CF61E0CE0187559F4F0E94011B96
:108B9000A2962FAFA297A3963FAFA397A4964FAFED
:108BA000A497A5965FAFA597A6966FAFA697A79631
:108BB0007FAFA797A8968FAFA897A9969FAFA997C1
:108BC00088248394982CAA24AA94BA2CF12C81E0AE
:108BD000CD54DF4F8883C35BD040512CD4CE40E0CE
:108BE00050E061E070E0C1010E949F2B672B682B71
:108BF000692BA9F040E050E061E070E0C1010E9403
:108C00004D2B8824839424E0922EAA24A394B12C83
:108C1000F12CCD54DF4F1882C35BD040DDC040E063
:108C200050E061E070E0C1010E94762BEACF95E050
:108C3000892E912CA12CB12C84CCC954DF4FE88112
:108C4000F981C75BD040EA30F10509F4B3C13B9725
:108C500009F0B4CCC655DF4F8881CA5AD0408295FE
:108C60008F70823009F023C2C501B40124E630E0E0
:108C700040E050E00F949527C255DF4F8881CE5ACF
:108C8000D04090E0280F391F37FF02C030E020E0CD
:108C90002536310514F024E630E0C255DF4F288335
:108CA000CE5AD04062E0CE0187559F4F0E94DA1A1B
:108CB0002A962FAF2A972B963FAF2B972C964FAF24
:108CC0002C972D965FAF2D972E966FAF2E972F96E0
:108CD0007FAF2F9760968FAF609761969FAF619738
:108CE000C3C1CD54DF4F1882C35BD040D101199668
:108CF0008D919C911A97009709F038C018968C9125
:108D000090E000E5402E512C612C712C85309105AE
:108D100049F0412C512C3201449721F0412C512C27
:108D200032014A94C655DF4FE881CA5AD040E295D5
:108D3000EF70E150EB3008F02EC1F0E08827EC55E1
:108D4000F94B8F4F0D94EA27BE46BE46CB47CB4723
:108D5000CB4798475E475E475E47EF46EF46F1E0F8
:108D6000CD54DF4FF883C35BD040C0CFDC01ED9121
:108D7000FC91068CF78DE02D1995C3CFC355DF4FBD
:108D80001881CD5AD040C501B40124E630E040E05E
:108D900050E00F949527DA01C901810F911DA11DA3
:108DA000B11DB7FF03C080E090E0DC018F3F91056B
:108DB000A105B10529F024F08FEF90E0A0E0B0E02C
:108DC000C355DF4F8883CD5AD040812C12E1912EBC
:108DD000F12CAA24AA94BA2C55245A94D4CDC35564
:108DE000DF4FC880D980EA80FB80CD5AD040B4E6FE
:108DF0008B169104A104B104DCF5A4E6B0E0A70150
:108E000096010F94B427860E971EA81EB91E411412
:108E1000510461047104B9F0A30192010F94B427C5
:108E2000362F272FB501A40177FF03C040E050E0A3
:108E3000BA01832E922E5C01481559056A057B05FF
:108E400014F44A015B01C355DF4F88829982AA82DC
:108E5000BB82CD5AD040C655DF4F8881CA5AD04018
:108E60008F708066C655DF4F8883CA5AD040ADCF19
:108E7000C501B40124E630E040E050E00F949527AE
:108E8000C20ED31EE41EF51E411451046104710488
:108E900061F0F7FE03C0C12CD12C76014C145D04A7
:108EA0006E047F0414F473016201C355DF4FC8825E
:108EB000D982EA82FB82CD5AD04087CFC355DF4F9B
:108EC000688179818A819B81CD5AD0400F94FB289B
:108ED0006B017C01C501B40124E630E040E050E0C4
:108EE0000F949527CA01B9016C0D7D1D8E1D9F1D24
:108EF000411451046104710481F06B017C01F7FE9F
:108F000003C0C12CD12C7601C701B6014616570605
:108F10006806790614F4C301B2010F943026C355D4
:108F2000DF4F688379838A839B83CD5AD0404DCFAE
:108F3000C355DF4F88819981AA81BB81CD5AD0402A
:108F4000880E991EAA1EBB1E4114510461047104AF
:108F5000C9F0A4E6B0E0A30192010F94B427362F24
:108F6000272FB501A40177FF03C040E050E0BA010C
:108F7000832E922E5C01481559056A057B0514F471
:108F80004A015B01C355DF4F88829982AA82BB8266
:108F9000CD5AD0401ACF88E0FE013196DE01A755A8
:108FA000BF4F01900D928A95E1F7912C812CFF24FF
:108FB000F3940FCFC655DF4F8881CA5AD0408295AF
:108FC0008F70823009F055C0C501B40124E630E04D
:108FD00040E050E00F949527C155DF4F8881CF5A6C
:108FE000D040C055DF4F6881C05BD040962F917054
:108FF000280F391F2E36E1E03E072CF437FF05C05D
:109000002DE631E002C030E020E0C155DF4F28837B
:10901000CF5AD040C055DF4F8881C05BD04030FB75
:1090200080F9C055DF4F8883C05BD04062E0CE013D
:1090300087559F4F0E94DA1A62962FAF6297639608
:109040003FAF639764964FAF649765965FAF659740
:1090500066966FAF669767967FAF679768968FAF94
:10906000689769969FAF6997812CB2E19B2EF12C8E
:1090700018C088E0FE013196DE01A755BF4F019070
:109080000D928A95E1F76CE37CE084E390E10F9424
:10909000A61284E390E10F945510912C812CFF24AB
:1090A000F394CD54DF4F1882C35BD04092CE88E05A
:1090B000FE013196DE01A755BF4F01900D928A95B2
:1090C000E1F760E37CE0E1CFC554DF4F1881CB5B73
:1090D000D040112309F46BC01296ED91FC9180856C
:1090E0008F70853009F070C0C154DF4FE881F9817D
:1090F000CF5BD040359709F467C0C1010E94E551AC
:1091000021E0181619060CF020E0522ECF54DF4F44
:1091100048815981C15BD040C454DF4F2881CC5B6A
:10912000D040BE0167557F4FD10112968D919C9121
:109130000E941E51C954DF4FE881F981C75BD040BE
:10914000319709F041C0C655DF4F1881CA5AD04047
:10915000812F807FC9F1C454DF4FC880CC5BD040E1
:10916000E52CC755DF4F0881C95AD040C555DF4FA0
:109170002881CB5AD040C455DF4F3881CC5AD040DB
:10918000C355DF4F4881CD5AD040C255DF4F58817B
:10919000CE5AD040C155DF4F6881CF5AD040C0551C
:1091A000DF4F7881C05BD040C1010E94D82EC755E7
:1091B000DF4F8881C95AD040853009F445C150F449
:1091C0008330B9F1D12CC3C0C554DF4F1882CB5BBB
:1091D000D040EDCF863009F482C0873099F7C101C5
:1091E0000E94ED30182F863009F066C068ED7BE0F4
:1091F00089ED90E10F94A6124AE050E066E070E03D
:1092000089ED90E10F94971189ED90E10F9455103D
:1092100062E0CE0187559F4F0E94011B29AF3AAFF4
:109220004BAF5CAF6DAF7EAF8FAF21969FAF2197F5
:109230003FC0C1010E94ED30853021F093E0A92E9E
:10924000B12C08C26FEE7BE089ED90E10F94A6127D
:109250004AE050E065E070E089ED90E10F949711ED
:1092600089ED90E10F945510B101CE0187559F4FC4
:109270000F94D51361E0CE0187559F4F0E94011BCB
:1092800022962FAF229723963FAF239724964FAF76
:10929000249725965FAF259726966FAF269727963A
:1092A0007FAF279728968FAF289729969FAF29974A
:1092B000689480F890F886CF6AEB7BE089ED90E1C6
:1092C0000F94A612612F70E04AE050E089ED90E122
:1092D0000F94971189ED90E10F945510AFCF40E0B6
:1092E00050E061E070E0C1010E949F2B672B682B6A
:1092F000692B09F0A6C0FFEF5F120EC0C1010E94EA
:10930000E551512C181619064CF460EA7BE089ED02
:1093100090E10F94A61292CF5110F7CFB101CE0178
:1093200087559F4F0F94D51361E0CE0187559F4F0E
:109330000E94011B29AB3AAB4BAB5CAB6DAB7EAB78
:109340008FAB98AF689480F890F8E6E0DE2E840149
:109350000160C655DF4F8881CA5AD040982F9F7050
:10936000923050F4C755DF4F9881C95AD0409923A5
:1093700019F0840101601160807F09F489C01260D6
:10938000C554DF4F2881CB5BD04021111D7FA80140
:10939000B101CE0187559F4F0E943B304801AA245E
:1093A000A394B12CF11045C7D10119968D919C91D0
:1093B000009709F0A7C340E050E062E070E0C1010F
:1093C0000E949F2B672B682B692B09F4CDC36CE59A
:1093D0007AE084E390E10F94A61284E390E10F9485
:1093E000551092FC53C661E47AE089ED90E10F9448
:1093F000A6124AE050E0B50189ED90E10F94971173
:109400006AE37AE089ED90E10F94A6120F94460486
:10941000AB01BC01CF53DF4F088119812A813B8109
:10942000C15CD040401B510B620B730B2AE030E053
:1094300089ED90E10F94531089ED90E10F94551050
:1094400009C16BE87BE063CF0FEF50120BC0C10185
:109450000E94E55155245394181619062CF06EE617
:109460007BE055CF5520D9F362E0CE0187559F4F61
:109470000E94011B29A73AA74BA75CA76DA77EA74F
:109480008FA798AB689480F890F875E0D72E5FCFDF
:1094900040E052E0B101CE0187559F4F0E94FA3063
:1094A00081116DCF6DCF3FEF53129DC0C1010E945E
:1094B000E55155245394181619060CF497C0512CF5
:1094C00060E67BE089ED90E10F94A612052D052C56
:1094D000000C110BC354DF4F19830883CD5BD040C0
:1094E0004AE050E0B80189ED90E10F94971169E5E9
:1094F0007BE089ED90E10F94A612CD54DF4F1881E7
:10950000C35BD040612F70E04AE050E089ED90E10C
:109510000F94971189ED90E10F945510CF54DF4FC0
:1095200008811981C15BD0400115110509F4B7C04C
:109530006BEC7EE0C8010F945920CC24C394D12C4D
:10954000892B09F45DC067EC7EE0C8010F945920B7
:1095500042E0C42ED12C892B09F452C065E37AE095
:10956000C8010F94592035E0C32ED12C892B09F462
:1095700047C061E37AE0C8010F94592026E0C22E6B
:10958000D12C892BE9F16CE87EE0C8010F945920B9
:10959000892B99F167E87EE0C8010F945920892B47
:1095A00009F473C061E97EE0C8010F945920BEE060
:1095B000CB2ED12C892B21F16AE77EE0C8010F94D4
:1095C0005920AFE0CA2ED12C892BD1F063E87EE080
:1095D000C8010F945920D12CC12C892B89F4F5E1B5
:1095E000CF2ED12C0DC0552009F46ACF81E0CD5487
:1095F000DF4F8883C35BD04063CF93E1C92ED12C6A
:10960000C1010E94ED30682E712C6114710431F497
:10961000C354DF4F68807980CD5BD040C114D10442
:1096200009F486C06C147D04A1F16DE37BE089ED43
:1096300090E10F94A6124AE050E0B30189ED90E169
:109640000F94971189ED90E10F945510EDEFAE2E28
:10965000BB24BA94C501CC53DF4F0FB6F894DEBFDC
:109660000FBECDBFDF91CF911F910F91FF90EF9073
:10967000DF90CF90BF90AF909F908F907F906F9032
:109680005F904F903F902F90089584E1C82ED12C89
:10969000B7CFCF54DF4F19821882C15BD040C95475
:1096A000DF4FE881F981C75BD0403197A9F4C554F9
:1096B000DF4FF881CB5BD040FF2399F0C655DF4FD9
:1096C0008881CA5AD040807F01E0C554DF4F0883AB
:1096D000CB5BD040811105C0C554DF4F1882CB5BF6
:1096E000D040C755DF4FD880C95AD04015E11D156D
:1096F00008F4E7C1ED2DF0E08827EE57F44B8F4FCB
:109700000D94EA27DB4B134DF94C1A4CDB4BDA4C2A
:10971000A04C654CDB4BDB4B4D4D574D754D754D9E
:109720002D4D2D4D614D614D614D2D4D2D4D2D4DCD
:10973000D10119968D919C91009709F4B0CFDC016D
:10974000ED91FC910688F789E02DC454DF4FA88085
:10975000CC5BD040CD54DF4FC880C35BD040780194
:10976000C755DF4F0881C95AD040C655DF4F188111
:10977000CA5AD040C555DF4F2881CB5AD040C45576
:10978000DF4F3881CC5AD040C355DF4F4881CD5A86
:10979000D040C255DF4F5881CE5AD040C155DF4F1F
:1097A0006881CF5AD040C055DF4F7881C05BD04030
:1097B00019950C946942D12CC554DF4F8881CB5B3D
:1097C000D040882309F4EECDC454DF4FC880CC5B71
:1097D000D040952D9170E92EC755DF4F0881C95AA9
:1097E000D040C655DF4F1881CA5AD040C555DF4F0B
:1097F0002881CB5AD040C455DF4F3881CC5AD04055
:10980000C355DF4F4881CD5AD040C255DF4F5881F4
:10981000CE5AD040C155DF4F6881CF5AD040C05595
:10982000DF4F7881C05BD040C1010E94D82EE89400
:1098300091F8B8CDC1010E94ED30853009F0FECC21
:1098400068E27BE089ED90E10F94A6124AE050E0D7
:1098500065E070E089ED90E10F94971189ED90E15A
:109860000F945510B101CE0187559F4F0F94D5131A
:10987000D10118968C918530C9F46EE0CE018755E0
:109880009F4F0E94011B29A33AA34BA35CA36DA386
:109890007EA38FA398A7689480F890F8D12CB1E0AC
:1098A000CD54DF4FB883C35BD04086CF61E0CE019B
:1098B00087559F4F0E94011B298F3A8F4B8F5C8FDA
:1098C0006D8F7E8F8F8F98A3E6CFC1010E94ED3000
:1098D000182F863091F561E17BE089ED90E10F94DE
:1098E000A6124AE050E066E070E089ED90E10F9446
:1098F000971189ED90E10F94551062E0CE018755E4
:109900009F4F0E94011B298B3A8B4B8B5C8B6D8B7D
:109910007E8B8F8B988F40E050E068E070E0C10153
:109920000E944D2B689480F890F8D12CE1E0CD5442
:10993000DF4FE883C35BD0403FCF63EF7AE0BECC1C
:1099400040E050E061E070E0C1010E949F2B672B76
:10995000682B692B61F5511027C0B101CE018755E5
:109960009F4F0F94D51361E0CE0187559F4F0E9402
:10997000011B29873A874B875C876D877E878F8796
:10998000988B40E050E068E070E0C1010E94762BC7
:10999000689480F890F876E0D72EF1E0CD54DF4F50
:1099A000F883C35BD04008CF69ED7AE0B0CC64ECBB
:1099B0007AE0ADCC5520D1F062E0CE0187559F4FC3
:1099C0000E94011B29833A834B835C836D837E83D2
:1099D0008F839887689480F890F865E0D62E01E030
:1099E000CD54DF4F0883C35BD040E6CE67EA7AE010
:1099F0008ECCC655DF4F8881CA5AD0408F70D12C8B
:109A0000823068F7C1010E94ED30689480F890F8C8
:109A1000853009F413CCD12C11E0CD54DF4F1883DD
:109A2000C35BD040C9CEC655DF4F8881CA5AD040EB
:109A30008F70823080F7552081F06EE87AE089EDF2
:109A400090E10F94A61261E0C1010E940A3060E02B
:109A500071E1C1010E948D31F1CBC655DF4F888184
:109A6000CA5AD040982F9F70923008F043C0DD2032
:109A700069F0807F31F4B101CE0187559F4F0F947B
:109A8000D513689480F823E0922AD12C31E0CD548C
:109A9000DF4F3883C35BD0408FCE689492F8D12CCF
:109AA00081E0CD54DF4F8883C35BD04085CE68947E
:109AB00092F8D12C91E0CD54DF4F9883C35BD04016
:109AC0007BCEC655DF4F8881CA5AD040807F51F483
:109AD000689490F8D12CA1E0CD54DF4FA883C35BEC
:109AE000D0406ACEB3E09B2A20CFD12C812C54E009
:109AF000952E53CFD12C21E0CD54DF4F2883C35B6B
:109B0000D0405ACEDC01ED91FC91028CF38DE02D1A
:109B1000C755DF4F0881C95AD040C655DF4F18815D
:109B2000CA5AD040C555DF4F2881CB5AD040C455C2
:109B3000DF4F3881CC5AD040C355DF4F4881CD5AD2
:109B4000D040C255DF4F5881CE5AD040C155DF4F6B
:109B50006881CF5AD040C055DF4F7881C05BD0407C
:109B60001995811128CC33CCF10181859285892BFF
:109B700009F473C08114910439F0A401B101CE013C
:109B800087559F4F0E943B30D10119968D919C9132
:109B9000CF54DF4FE880F980C15BD040DC01ED910C
:109BA000FC910688F789E02DC454DF4FA880CC5B78
:109BB000D040CD54DF4FC880C35BD040C755DF4F86
:109BC0000881C95AD040C655DF4F1881CA5AD040C3
:109BD000C555DF4F2881CB5AD040C455DF4F38815F
:109BE000CC5AD040C355DF4F4881CD5AD040C255E2
:109BF000DF4F5881CE5AD040C155DF4F6881CF5AD0
:109C0000D040C055DF4F7881C05BD04019955C01D2
:109C1000F10181859285DC01ED91FC91068CF78D37
:109C2000E02D1995059711F4689480F892FC73C1A2
:109C3000DD2021F06D2DC1010E940A30C154DF4F9B
:109C400008811981CF5BD040B4010530110509F4BA
:109C5000CACBC1010E948D31C6CB8085863009F404
:109C600077C008F5843009F45EC1853009F78114A6
:109C7000910439F0A401B101CE0187559F4F0E9494
:109C80003B30C954DF4F08811981C75BD040023097
:109C9000110509F444C10330110509F4D2C00130A3
:109CA000110531F6CAC0883009F4A1C1893009F024
:109CB000BFCF8114910439F0A401B101CE018755C1
:109CC0009F4F0E943B30CD54DF4FE881C35BD040B3
:109CD000EE2309F4ADCF552079F0C755DF4F8881C9
:109CE000C95AD040813041F4C655DF4F8881CA5AE5
:109CF000D040807F09F49CCFC755DF4F0881C95AF7
:109D0000D040C655DF4F1881CA5AD040C555DF4FE5
:109D10002881CB5AD040C455DF4F3881CC5AD0402F
:109D2000C355DF4F4881CD5AD040C255DF4F5881CF
:109D3000CE5AD040C155DF4F6881CF5AD040C05570
:109D4000DF4F7881C05BD040C1010E94D73739C155
:109D5000C755DF4FF880C95AD040FF2009F487CF9C
:109D600070E060E0C1010E9438298C0181149104E7
:109D700039F0A401B101CE0187559F4F0E943B30BD
:109D80000115110509F454CF712C612C17FF06C081
:109D900011950195110966246394712CC8010197EE
:109DA0008634910508F044CFE02E61E0802F0F94B7
:109DB0000100EFEFEF0DE53110F5F0E08827EC51F1
:109DC000F14B8F4F0D94EA27F94EFB4EFF4EFF4E9D
:109DD000FB4EF94EFB4EFF4EFF4EFF4EFF4EFF4E29
:109DE000FF4EF94EF94EFF4EFF4EFF4EFF4EF94E1D
:109DF000F94EF1E06F26662D8E2D0E94D3FF67E5A8
:109E00007AE089ED90E10F94A6124AE050E0B801A3
:109E100089ED90E10F94971165E57AE089ED90E185
:109E20000F94A6124AE050E0B30189ED90E10F943F
:109E3000971189ED90E10F945510689480F890F88F
:109E40006AC0C1010E94D628892B49F4D101ED9145
:109E5000FC916081718183E296E00F94FE04CE0153
:109E600087559F4F0E940A1F20E030E048EC52E4E3
:109E70000F948F260F94FB28C954DF4F6883798392
:109E80008A839B83C75BD040C954DF4F4880598089
:109E9000C75BD04088E00E946DD6CD54DF4F688309
:109EA00079838A839B83C35BD040CD54DF4F688026
:109EB0007980C35BD04061E57AE089ED90E10F9451
:109EC000A6124AE050E0C954DF4F68817981C75B30
:109ED000D04089ED90E10F9497116CE47AE089ED20
:109EE00090E10F94A612CD54DF4F488159816A81C9
:109EF0007B81C35BD040662777272AE089ED90E11C
:109F00000F94071089ED90E10F945510B301A20151
:109F1000C1010E947C28AA24A394B12C89CE689404
:109F200080F891F8F8CF8114910439F0A401B101BF
:109F3000CE0187559F4F0E943B30CD54DF4FB881F3
:109F4000C35BD040BB2309F473CEC755DF4F888174
:109F5000C95AD0405520B9F1813041F4C655DF4F80
:109F60008881CA5AD040807F09F462CEC755DF4F3E
:109F70000881C95AD040C655DF4F1881CA5AD0400F
:109F8000C555DF4F2881CB5AD040C455DF4F3881AB
:109F9000CC5AD040C355DF4F4881CD5AD040C2552E
:109FA000DF4F5881CE5AD040C155DF4F6881CF5A1C
:109FB000D040C055DF4F7881C05BD040C1010E94C6
:109FC00007365C0135CE813089F6CE0187559F4F2B
:109FD0000E94CFF8449750F66EE170E0CE018755AD
:109FE0009F4F0E94B61E689480F891F8BFCF8114ED
:109FF000910439F0A401B101CE0187559F4F0E9411
:10A000003B30CD54DF4FF881C35BD040FF2309F4D0
:10A010000FCE552079F0C755DF4F8881C95AD040FF
:10A02000813041F4C655DF4F8881CA5AD040807FC5
:10A0300009F4FECDC755DF4F0881C95AD040C65537
:10A04000DF4F1881CA5AD040C555DF4F2881CB5AFF
:10A05000D040C455DF4F3881CC5AD040C355DF4F74
:10A060004881CD5AD040C255DF4F5881CE5AD0409A
:10A07000C155DF4F6881CF5AD040C055DF4F78813E
:10A08000C05BD040C1010E94C0369BCFC154DF4F9E
:10A0900028813981CF5BD0402530310509F4A3C92F
:10A0A00040E054E0B101CE0187559F4F0E943B3004
:10A0B00060E074E0CECD0E94511F672B682B692BA6
:10A0C00011F00C94AD43912C812C11E0CD54DF4F55
:10A0D0001883C35BD0400C94E443C954DF4F2881FC
:10A0E0003981C75BD040232B09F053C0808188237E
:10A0F00011F40C94DE41CE018F549F4F0E94F7273C
:10A10000C954DF4F99838883C75BD040C655DF4F62
:10A110008881CA5AD0408F7091F5C954DF4F688149
:10A12000C75BD040CE0187559F4F0E94DA1ACF55AA
:10A13000DF4F2883C15AD040CE55DF4F3883C25AF3
:10A14000D040CD55DF4F4883C35AD040CC55DF4F68
:10A150005883C45AD040CB55DF4F6883C55AD0408E
:10A16000CA55DF4F7883C65AD040C955DF4F888320
:10A17000C75AD040C855DF4F9883C85AD040C954F9
:10A18000DF4FE881F981C75BD040EF2B11F40C94CD
:10A19000DE4160E87CE089ED90E10F94A6124AE090
:10A1A00050E0B60189ED90E10F94971169E77CE0EA
:10A1B00089ED90E10F94A612D101ED91FC9160819F
:10A1C000718189ED90E10F94B01163E77CE089ED36
:10A1D00090E10F94A612CF54DF4F68817981C15B63
:10A1E000D04089ED90E10F94B01161E77CE089EDFA
:10A1F00090E10F94A612CE0187559F4F0E94D8225E
:10A20000CF54DF4FE881F981C15BD040309711F422
:10A210000C942A428081843211F00C942A426DE51C
:10A220007CE089ED90E10F94A61289ED90E10F9406
:10A2300055108CEFA82EBB24BA940CCA2F923F92D3
:10A240004F925F926F927F928F929F92AF92CF9236
:10A25000DF92EF92FF920F931F93CF93DF93CDB7CF
:10A26000DEB76D970FB6F894DEBF0FBECDBF009777
:10A2700009F4A9C0FC0130853F70353009F0A3C056
:10A28000D22E1A014B01668077808091D50C8F5FAA
:10A290008093D50C6114710409F490C0F30180859A
:10A2A0008F70843009F086C0618572858091DB0CE7
:10A2B0009091DC0C0E940EF82C01009709F47AC0F2
:10A2C000FC0180858F70853009F074C0B201CE0129
:10A2D00001960E948A3481149104B1F0CE01019656
:10A2E0000E942D28882381F0AD2CC12C7101F4012E
:10A2F000008111812281338144815581668177817A
:10A30000CE0101960E94194160E0C2010E94C0F88E
:10A310000097E9F1FC0120852F702230C1F581857D
:10A320009285A385B4850797A105B10581F561E004
:10A33000C2010E94C0F82D2DA101B4010E941E513E
:10A340008114910499F5882389F18091D50C81506D
:10A350008093D50CCE0101960E947C3481E06D96ED
:10A360000FB6F894DEBF0FBECDBFDF91CF911F9126
:10A370000F91FF90EF90DF90CF90AF909F908F90D4
:10A380007F906F905F904F903F902F900895811431
:10A39000910461F4CE0101960E942D28882331F0AA
:10A3A000CE0101960E94E551892B79F6CE010196E6
:10A3B0000E947C34F301628073806CCF8091D50C55
:10A3C00081508093D50C80E0CACFDF92EF92FF924C
:10A3D0000F931F93CF93DF9300D000D01F921F9253
:10A3E000CDB7DEB77C0119821A821B821C821D82C6
:10A3F0001E821F8218868A818F708A83D701ED9111
:10A40000FC916081718189ED90E10F94B0116CEC49
:10A410007CE089ED90E10F94A612C7010E942D28DF
:10A4200081111BC063EC7CE089ED90E10F94A612D2
:10A4300089ED90E10F9455100FEF1FEFC80128969A
:10A440000FB6F894DEBF0FBECDBFDF91CF911F9145
:10A450000F91FF90EF90DF900895C7010E94ED30BB
:10A46000D82EF70181859285009791F0DC01ED915E
:10A47000FC91008CF18DE02D19958C0197FD08C0A1
:10A4800081E00115110509F480E00E948917D6CFFB
:10A49000F7018085873009F42EC0EFEFED0DE43130
:10A4A00050F5F0E08827E85AFD4A8F4F0D94EA27CF
:10A4B0006C5275527B527B5275526C527B527B525E
:10A4C0007B527B527B527B527B526C527B527B5233
:10A4D0007B527B526C526C5264EA7CE089ED90E1D5
:10A4E0000F94A61201E010E0A9CF80E00E94891726
:10A4F00010E000E0A3CF40E052E0B701CE010196AA
:10A500000E94FA30D70118968C911897873089F1FC
:10A5100060F4833009F457C0843061F064EB7CE070
:10A5200089ED90E10F94A612E3CF883009F44BC077
:10A530008930A1F760E0CE0101960E94E91D8C01EF
:10A5400069EA7CE089ED90E10F94A6124AE050E0C0
:10A55000B80189ED90E10F94971189ED90E10F9486
:10A56000551091E080E0012B09F490E0092F182F9D
:10A5700065CF1296ED91FC9180858F7010E000E020
:10A580008530F1F661EC7CE089ED90E10F94A61244
:10A5900020E050E040E070E060E0F70182819381CC
:10A5A0000E941E51F82E082F10E06EEB7CE089ED22
:10A5B00090E10F94A6128F2D0E94891789ED90E1EA
:10A5C0000F9455103BCFCE0101960E94511F8B0175
:10A5D000B7CFAF92CF92EF92FF920F931F93CF938B
:10A5E000DF9300D000D01F921F92CDB7DEB7198243
:10A5F0001A821B821C821D821E821F8218861A816B
:10A600001F70A12CCC24C394F12CE12C02E02B81EF
:10A610003C8140E05E816F8178850E9419412896D7
:10A620000FB6F894DEBF0FBECDBFDF91CF911F9163
:10A630000F91FF90EF90CF90AF9008952F923F929F
:10A640004F925F926F927F928F929F92AF92BF9242
:10A65000CF92DF92EF92FF920F931F93CF93DF93EE
:10A66000CDB7DEB7CA55D1090FB6F894DEBF0FBE1D
:10A67000CDBF4C013B0140E058E060E070E00E943B
:10A680009F2B672B682B692B09F45CC019821A82F7
:10A690001B821C821D821E821F8218868A818F70F7
:10A6A0008A8340E053E0B401CE0101960E94FA3063
:10A6B000D40119968D919C91892B09F41AC140E01F
:10A6C00058E060E070E0C4010E944D2B69E17DE03C
:10A6D00089ED90E10F94A612F40181859285DC0149
:10A6E000ED91FC910688F789E02DA12CCC24C39430
:10A6F000F12CE12C09811A812B813C814D815E81F5
:10A700006F8178851995D401ED91FC918F3F980761
:10A71000C9F060817181892B09F055C189ED90E103
:10A720000F94B0116CED7CE089ED90E10F94A612CE
:10A7300064ED7CE089ED90E10F94A61289ED90E143
:10A740000F94551065E0F401808191810E94C0F85A
:10A750005C01009709F46FC1DC011896BC91699601
:10A76000BFAF6997B295BF706896BFAF6897FC019D
:10A7700021843284438454840F9446046896FFAD48
:10A780006897FF2309F457C1261A370A480A590A5D
:10A7900019A21AA21BA21CA21DA21EA21FA218A6C9
:10A7A0008AA18F70806B8AA3F9A3B201A101CE01A7
:10A7B00081960E94671D2F962FAF2F9760963FAF0F
:10A7C000609761964FAF619762965FAF62976396AD
:10A7D0006FAF639764967FAF649765968FAF659709
:10A7E00066969FAF669724E06216710451F5D12CEE
:10A7F000C12CE12C50E2F52E09A11AA12BA13CA1FC
:10A800004DA15EA16FA178A5C4010E94C32BC20116
:10A81000B10128EE33E040E050E00F949527BA01F3
:10A82000A9012AE030E089ED90E10F944F1169E22F
:10A830007EE089ED90E10F94A61289ED90E10F94EE
:10A84000551057FEF8C082E028163104410480E814
:10A8500058060CF4F0C00E9416DD1B016B967FAF0A
:10A860006EAF6B97D12CC12CE12C40E2F42E09A1E4
:10A870001AA12BA13CA14DA15EA16FA178A5C40195
:10A880000E94C32B6B96AEADBFAD6B97A83CB105D4
:10A890000CF0A6C060E17EE084E390E10F94A61284
:10A8A0004AE050E0B10184E390E10F94971184E312
:10A8B00090E10F94551066246A94762CC301C65A11
:10A8C000DF4F0FB6F894DEBF0FBECDBFDF91CF9143
:10A8D0001F910F91FF90EF90DF90CF90BF90AF90BE
:10A8E0009F908F907F906F905F904F903F902F90B0
:10A8F0000895F4018085883009F445C0893019F144
:10A90000843009F01FCF8091330B9091340B892B49
:10A9100009F018CF40E058E060E070E0C4010E9408
:10A920004D2B64E07DE089ED90E10F94A612098142
:10A930001A812B813C814D815E816F817885C401B4
:10A940000E940736E0CE8091330B9091340B892B17
:10A9500009F0F8CE40E058E060E070E0C4010E94E9
:10A960004D2B63EF7CE089ED90E10F94A6120981F5
:10A970001A812B813C814D815E816F817885C40174
:10A980000E94D737C0CE8091330B9091340B892B26
:10A9900009F0D8CE40E058E060E070E0C4010E94C9
:10A9A0004D2B6EED7CE089ED90E10F94A6120981AC
:10A9B0001A812B813C814D815E816F817885C40134
:10A9C0000E94C036A0CE89ED90E10F94B01162EDE7
:10A9D0007CE089ED90E10F94A6126EEC7CE0AACEAB
:10A9E000F50180858F70808719821A821B821C82F4
:10A9F0001D821E821F8218868A818F708A836896C4
:10AA0000FFAD6897F98369968FAD69978F70AA2417
:10AA1000A394873009F0A12CCC24C394F12CE12C11
:10AA200009811A812B813C814D815E816F817885FE
:10AA3000C4010E94194121E06216710459F4D40145
:10AA400018968C91843079F0893009F470C1C40172
:10AA50000E94FF31F40181859285009709F0A0C41E
:10AA6000712C612C2BCF8091330B9091340B892B5F
:10AA7000B9F4F40142805380D20118968C918F7002
:10AA8000853041F4C2010E9452F9082F10E00230D3
:10AA9000110554F468E77DE089ED90E10F94A6126A
:10AAA000C4010E94FF310ACF7092340B6092330BC5
:10AAB00070E060E0C4010E9438291C0161E070E090
:10AAC000C4010E9438295C01053011050CF440C016
:10AAD00064E0C2010E94C0F8FC010185128526E0F5
:10AAE00040E855E260E070E087E49DE00E9493BB9F
:10AAF0002092DE0E87E49DE09093DD0E8093DC0EC5
:10AB00001092E90F1092EB0F1092EA0F64E67DE0CD
:10AB100089ED90E10F94A612D401ED91FC91608132
:10AB2000718189ED90E10F94B01189ED90E10F945E
:10AB300055100130110509F4C2C06CF4012B09F461
:10AB4000B3C068E47DE089ED90E10F94A61225C0C2
:10AB500002E010E0C4CF0230110579F00330110596
:10AB600081F7B092E00EA092DF0E81E090E090932A
:10AB7000E20E8093E10E84E00BC0B092E00EA09252
:10AB8000DF0E81E090E09093E20E8093E10E83E08F
:10AB90000F94700667968FAF67976796BFAD6797FC
:10ABA000B11197C00091E30E1091E40E63E47DE0D3
:10ABB00089ED90E10F94A612D401ED91FC91608192
:10ABC000718189ED90E10F94B0116CE37DE089ED26
:10ABD00090E10F94A612C801012E000CAA0BBB0B2A
:10ABE00089839A83AB83BC8380E190E09E838D83CD
:10ABF000BE016F5F7F4F89ED90E10E94A0340F94FA
:10AC00005510B801C4010E94E132E0912C0BF09183
:10AC10002D0B62817381CE0101960E948A3480914E
:10AC20002C0B90912D0B892BB1F1CE0101960E9436
:10AC30002D28882381F18985843069F570E060E0F2
:10AC4000CE0101960E9438292816390621F561E0C7
:10AC500070E0CE0101960E943829A816B906D9F4F1
:10AC6000B801CE0101960E94E132E0912C0BF091E7
:10AC70002D0B8281938190932D0B80932C0B892B2C
:10AC800051F4E091DB0CF091DC0C8681978190937C
:10AC90002D0B80932C0BCE0101960E947C341092D8
:10ACA000340B1092330BFCCEB092E00EA092DF0E6C
:10ACB00081E090E09093E20E8093E10E69CFB09234
:10ACC000E00EA092DF0E1093E20E0093E10E82E000
:10ACD0005FCF6FE27DE089ED90E10F94A612D40181
:10ACE000ED91FC916081718189ED90E10F94B0113B
:10ACF00067E27DE089ED90E10F94A6126796EFADD3
:10AD000067978E2F90E0B0E0A0E089839A83AB83B1
:10AD1000BC8380E190E09E838D83BE016F5F7F4F97
:10AD200089ED90E10E94A0340F945510B8CF809126
:10AD3000330B9091340B892B09F0B2CE7092340B07
:10AD40006092330B0E944EC12C01009741F0DC0150
:10AD500018968C911897807F866018968C93F201D4
:10AD600080858F70808730E020E043E050E060E233
:10AD7000CE0101960E9495DBD401ED91FC9160819A
:10AD800071814FE150E0CE0101960F94672C62E390
:10AD900076E0CE0101960F94412C26E040E855E282
:10ADA00060E070E087E49DE00E9493BB70E060E0AB
:10ADB000C4010E9438298093DE0E87E49DE09093C1
:10ADC000DD0E8093DC0E1092E90F1092EB0F1092C3
:10ADD000EA0F60E07EE089ED90E10F94A612D401C5
:10ADE000ED91FC916081718189ED90E10F94B0113A
:10ADF00089ED90E10F94551062E370E080E090E0FF
:10AE00000F94460284E398E09093E00E8093DF0E67
:10AE10008AE090E09093E20E8093E10E83E00F943D
:10AE20007006182F811154C263EF7DE089ED90E127
:10AE30000F94A61203EE1EE097EF292E9EE0392E06
:10AE400020E1A22EB12CF801819191918F01092E60
:10AE5000000CAA0BBB0B89A39AA3ABA3BCA3BEA2F5
:10AE6000ADA2BE016F5D7F4F89ED90E10E94A034DD
:10AE700061EF7DE00F94A6122016310621F789EDCF
:10AE800090E10F9455106091E70E7091E80E90E0FC
:10AE900080E00F94302620E030E048EC52E40F943C
:10AEA00089289B01AC016DEA78E0C2010E94ACFDEB
:10AEB000C090EB0ED090EC0EF12CE12CA701960186
:10AEC00068E376E0C2010E94DDFB6091ED0E7091B7
:10AED000EE0E90E080E00F94302620E030E048EC69
:10AEE00052E40F9489289B01AC016CE376E0C20127
:10AEF0000E94ACFD6091EF0E7091F00E90E080E04A
:10AF00000F94302620E030E040E251E40F9489288D
:10AF10009B01AC016AE376E0C2010E94ACFD209186
:10AF2000E30E3091E40E50E040E06EE376E0C201C3
:10AF30000E94DDFBCD28CE28CF2809F47AC0D401A9
:10AF40001296ED91FC9190859F70953009F071C03B
:10AF500061E0CF010E94C0F8009709F46AC0FC01CB
:10AF600020852F70243009F064C061857285CE0180
:10AF700081960E94F033CE0181960E942D2888236D
:10AF800009F453C022961CAE1DAE1EAE1FAE229712
:10AF900026961CAE1DAE1EAE1FAE26978FAD8F70CF
:10AFA00080618FAF8FEF23968FAF239724965FAD8D
:10AFB000249725963FAD259726962FAD26979EADD3
:10AFC0007FAD21966FAD219722964FAD2297092F25
:10AFD00027969FAF279728967FAF289729966FAF20
:10AFE00029972A964FAF2A97482F2B968FAF2B97EA
:10AFF0002C965FAF2C972D963FAF2D972E962FAFA7
:10B000002E97A12CCC24C394F12CE12C172F262FA2
:10B010002A963FAD2A972D966FAD2D972E967FAD30
:10B020002E97CE0181960E941941CE0181960E94F1
:10B030007C348091E30E83FF76C166EC7DE089ED80
:10B0400090E10F94A612D401ED91FC916081718181
:10B0500089ED90E10F94B01189ED90E10F945510B6
:10B0600062E370E080E090E00F9446028EE398E0A7
:10B070009093E00E8093DF0E81E090E09093E20EDB
:10B080008093E10E83E00F94700681110BC0209134
:10B09000E30E3091E40E50E040E061E476E0C2015E
:10B0A0000E94DDFB1092340B1092330BC4010E94FE
:10B0B000E551181619061CF4C4010E94E95281E0FA
:10B0C00090E09093340B8093330B66EB7DE089ED39
:10B0D00090E10F94A612D401ED91FC9160817181F1
:10B0E00089ED90E10F94B01189ED90E10F94551026
:10B0F00062E370E080E090E00F94460283E190E02C
:10B100009093E00E8093DF0E84E090E09093E20E47
:10B110008093E10E83E00F947006182F811115C102
:10B1200069EA7DE089ED90E10F94A61203EE1EE03E
:10B130008BEEE82E8EE0F82EF801619171918F016F
:10B140004AE050E089ED90E10F94971167EA7DE0C5
:10B1500089ED90E10F94A612E016F10669F789EDEA
:10B1600090E10F9455100091E30E1091E40E01153B
:10B170001105D1F0B801012E000C880B990B0F942A
:10B1800030262DEE3EE94CE35EE30F948F2622E558
:10B1900038EB42E152E40F941C289B01AC0164EEB1
:10B1A00076E0C2010E94ACFD6091E50E7091E60E62
:10B1B000072E000C880B990B0F9430262DEE3EE9DC
:10B1C0004CE35EE30F948F2622E538EB42E152E434
:10B1D0000F941C286B017C01AC019B0166E376E0B7
:10B1E000C2010E94ACFD6091E90E7091EA0E161644
:10B1F00017060CF0A1C0072E000C880B990B0F94BA
:10B20000302620E030E040E251E40F9489289B0191
:10B21000AC0165E476E0C2010E94ACFD20E030E0C4
:10B2200040E252E4C701B6010F9431291816B4F474
:10B23000012BA1F00E942CF8882369F08091C40BA7
:10B24000811109C0D401ED91FC916081718189E483
:10B2500096E00F94FE04C4010E94E95280E091E060
:10B260000F941D1D8C01892BD9F01CA21BA21EA2BC
:10B270001DA28FEF9FEF98A78FA384E892E09AA377
:10B2800089A31AA619A61CA70BA780E091E098AB8A
:10B290008FA71EA61DA6B201CE0181960E943EBFB9
:10B2A0000E942CF8882349F08091C40B811105C0BD
:10B2B000B801CE0101960F94FE04C8010F94B91D88
:10B2C0004114510409F4EBCCC2010E9480FDE7CC8B
:10B2D00064EE7DE089ED90E10F94A612D401ED912A
:10B2E000FC916081718189ED90E10F94B0116CED5A
:10B2F0007DE089ED90E10F94A612812F90E0B0E0FF
:10B30000A0E089A39AA3ABA3BCA380E190E09EA395
:10B310008DA3BE016F5D7F4F89ED90E10E94A03447
:10B320000F94551086CE20E030E0A90161E476E06C
:10B33000C2010E94DDFBC9CE20E030E0A90165E436
:10B3400076E0C2010E94DDFB69CF67E97DE089ED0F
:10B3500090E10F94A612D401ED91FC91608171816E
:10B3600089ED90E10F94B0116FE87DE089ED90E1F7
:10B370000F94A612812F90E0B0E0A0E089A39AA3D9
:10B38000ABA3BCA380E190E09EA38DA3BE016F5D43
:10B390007F4F89ED90E10E94A0340F9455105ECF4D
:10B3A000DC01ED91FC910484F585E02D1995892B44
:10B3B00009F456CBF40181859285DC01ED91FC9175
:10B3C0000480F581E02DB30119953C0177CA2F92D5
:10B3D0003F924F925F926F927F928F929F92AF9225
:10B3E000BF92CF92DF92EF92FF920F931F93CF9372
:10B3F000DF93CDB7DEB7CE57D1090FB6F894DEBFD5
:10B400000FBECDBFDC0114962D913C911597232BD7
:10B4100011F40C9427643B014C01AA969FAF8EAFA8
:10B42000AA978BE794E0A8969FAF8EAFA897AE96A9
:10B43000BFAFAEAFAE9781E694E0AC969FAF8EAF54
:10B44000AC97FD0182819B012250310922303105E8
:10B4500008F017C6803409F4F7C208F04AC08430F7
:10B4600008F085C28091EB0A8F5F8093EB0AA301FD
:10B470006FEFC4010E94231BD40112960C91129706
:10B480000695017013961C9113978AEC810F8031F9
:10B4900008F043C066E576E08D919C910E940EF81D
:10B4A0007C010097D1F1FC0180858F708530A9F572
:10B4B0008091E710181324C08091E810803401F5C2
:10B4C0008091E9109091EA105C01990FCC08DD0899
:10B4D00060E0C7010E94C0F8FC0181859285A385C8
:10B4E000B485A816B906CA06DB060CF065C0512C57
:10B4F0003EC0823409F4A8C208F439C28058AFCFE4
:10B500001093E71080E48093E810812F0F941401CA
:10B510009093EA108093E910D7CF212F30E0F90102
:10B52000E75AF54D8491F901E754F54D1491F9016D
:10B53000E150F54DF490FF2009F43BC081110E94C9
:10B540006CFFEF2DF0E0EE0FFF1FEF52F64DA591CF
:10B55000B491EC911E2331E020E009F430E0832F18
:10B56000922F552453940817190609F0C0CFF3E021
:10B570006F16710409F488C0D4011496ED91FC9102
:10B58000E181EF70E150EC3008F07EC0F0E08827F8
:10B59000E353F54A8F4F0D94EA27EE5A6A5C245B19
:10B5A0005A5B6A5C735B6A5CA75BD45BED5B2F5C88
:10B5B000515C90E080E0D5CF61E0C7010E94C0F807
:10B5C00055245394FC0181859285A385B4858A1501
:10B5D0009B05AC05BD050CF0CACF89CF0F9446047E
:10B5E0009B01AC0144275527D4011496ED91FC91A1
:10B5F0006281738190E080E0AA24AA94BA2CC12CC5
:10B60000D12C18EEE12E13E0F12E00E010E00E94A4
:10B61000B8D58823C9F1F4010081118163EB75E08D
:10B62000C8010E940EF8892B41F468EB75E0C8014F
:10B630000E940EF8892B09F40EC142E050E063E04D
:10B64000C4010E94231B20C00F9446049B01AC013F
:10B6500044275527D4011496ED91FC9162817381A2
:10B6600090E080E0AA24AA94BA2CC12CD12C1CE230
:10B67000E12EFF24F39400E010E00E94B8D542E0F0
:10B6800050E064E0811184C0D4011496ED91FC91E6
:10B69000808183FB992790F9951509F4D2C1982FE1
:10B6A000907E09F439C1982F907E90528F71892B2A
:10B6B000808358C10F9446049B01AC014427552751
:10B6C000D4011496ED91FC916281738190E080E049
:10B6D000AA24AA94BA2CC12CD12C16E9E12EF12C63
:10B6E00000E010E0CACF0F9446049B01AC01442750
:10B6F0005527D4011496ED91FC916281738190E0FD
:10B7000080E0AA24AA94BA2CC12CD12C18EEE12EE8
:10B7100013E0F12E00E010E00E94B8D5882309F470
:10B72000B3CFF401008111816EEB75E0C8010E9476
:10B730000EF8892B41F464EC75E0C8010E940EF804
:10B74000892B09F488C042E050E068E079CF0F947B
:10B7500046049B01AC0144275527D4011496ED9172
:10B76000FC916281738190E080E0AA24AA94BA2CB3
:10B77000C12CD12C1CE2E12EFF24F39400E010E058
:10B780000E94B8D542E050E069E0882309F47CCFFC
:10B79000C4010E94231B0F944604D4011496ED911A
:10B7A000FC917383628370CF0F9446049B01AC01BC
:10B7B00044275527D4011496ED91FC916281738141
:10B7C00090E080E0AA24AA94BA2CC12CD12C16E9CE
:10B7D000E12EF12C00E010E0D3CF0F9446049B0142
:10B7E000AC0144275527D4011496ED91FC91628158
:10B7F000738190E080E0AA24AA94BA2CC12CD12CA9
:10B8000018EEE12E13E0F12E00E010E00E94B8D512
:10B81000882309F439CFF401008111816BEC75E0C4
:10B82000C8010E940EF8892B39F461ED75E0C8015A
:10B830000E940EF8892B21F042E050E06BE000CF2F
:10B840006DEA75E0C8010E940EF842E050E066E043
:10B85000892B09F4F5CE42E050E06DE0F1CE0F9473
:10B8600046049B01AC0144275527D4011496ED9161
:10B87000FC916281738190E080E0AA24AA94BA2CA2
:10B88000C12CD12C1CE2E12EFF24F39400E010E047
:10B890000E94B8D5882309F4F7CE42E050E06CE06E
:10B8A00077CF0F9446049B01AC0144275527D40160
:10B8B0001496ED91FC916281738190E080E0AA245E
:10B8C000AA94BA2CC12CD12C16E9E12EF12C00E05F
:10B8D00010E0DECF0F9446049B01AC0144275527AE
:10B8E000D4011496ED91FC916281738190E080E027
:10B8F000AA24AA94BA2CC12CD12C18E5E12E12E06E
:10B90000F12E00E010E00E94B8D5882309F4BCCEE7
:10B9100042E050E060E094CE0F944604D4011496C7
:10B92000ED91FC91159773836283E181EF7055204F
:10B9300009F445C0E230F1F050F4EE23E9F1D4010E
:10B940001496ED91FC91808150FA83F9B1CEE530E7
:10B9500089F0A3016AE0E73091F7C4010E94231B3C
:10B960008111EDCF8091EB0A81508093EB0A90E03A
:10B9700080E06FC7F4010081118167EA75E0C801BA
:10B980000E940EF8892BA9F46EEB75E0C8010E94A5
:10B990000EF8892B71F464EC75E0C8010E940EF872
:10B9A000892B39F46FE875E0C8010E940EF8892BE5
:10B9B00019F0A30166E0D1CFA30161E0CECFE15041
:10B9C000ED3008F0BCCFF0E08827E651F34A8F4F06
:10B9D0000D94EA27F75C9F5CFA5CFA5C9F5CFD5C67
:10B9E0009F5C1E5D1E5D1E5D1E5D1E5DFA5CA301FB
:10B9F00062E0B3CFA30165E0B0CF0D911C9167EA7F
:10BA000075E0C8010E940EF8892BA9F46EEB75E071
:10BA1000C8010E940EF8892B71F464EC75E0C8012E
:10BA20000E940EF8892B39F46FE875E0C8010E9476
:10BA30000EF8892B19F0A30167E08FCFA30160E016
:10BA40008CCF8F71806434CEB3E06B16710409F42F
:10BA50008ECF66E576E0F401808191810E940EF838
:10BA60008C01D40113968C919091E7108913E5C055
:10BA70009091E810903409F0E0C08091E910909125
:10BA8000EA103C010115110509F404C1F8012085F3
:10BA90002F70253009F0FEC0C8010E9452F9AF9600
:10BAA0008FAFAF97843008F4D4C063E0C8010E9420
:10BAB000C0F8DC0119968D919C912AE0F22EF89E37
:10BAC0001001F99E300C112462E0C8010E94C0F8F8
:10BAD000FC0181859285F89E5001F99EB00C1124DD
:10BAE00065010B2C000CEE08FF08EF96CCAEDDAE26
:10BAF000EEAEFFAEEF9761E0C8010E94C0F82C01E6
:10BB000060E0C8010E94C0F8DC011996CD90DD907C
:10BB1000ED90FC901C97E396CCAEDDAEEEAEFFAEA2
:10BB2000E3979301072C000C440B550B2C193D098E
:10BB30004E095F09B101032C000C880B990BEF969D
:10BB4000CCACDDACEEACFFACEF976C197D098E0987
:10BB50009F090F946327D20119962D913D914D9124
:10BB60005C911C97E396CCACDDACEEACFFACE397FC
:10BB70002C193D094E095F09E3962CAF3DAF4EAF3E
:10BB80005FAFE3970F949527EF96CCACDDACEEACAE
:10BB9000FFACEF97C20ED31EE41EF51EAF962FAD7D
:10BBA000AF97253009F465C081E090E0A101032C36
:10BBB000000C660B770B4C155D056E057F050CF4CC
:10BBC00061C0B701A60165010B2C000CEE08FF084F
:10BBD0004C155D056E057F050CF459C06A017B01AB
:10BBE000AF96BFADAF97B23009F065C06301770C77
:10BBF000EE08FF0860E0C8010E94C0F8FC018185E2
:10BC00009285A385B485C816D906EA06FB060CF40E
:10BC10003AC661E0C8010E94C0F8FC0181859285A6
:10BC2000A385B4858C159D05AE05BF050CF09FCE90
:10BC300081E090E0A0E0B0E029C68093E71090E4B6
:10BC40009093E8100F9414019093EA108093E910F8
:10BC500018CF8AE0869D6001879DD00C11240D2CA1
:10BC6000000CEE08FF08B12CA12C212C88E2382E04
:10BC70009BCF64E0C8010E94C0F8DC0119968D9149
:10BC80009C9194CF66246A94B3E07B2E9CCF712C58
:10BC9000612CA6CF2AE0289F6001299FD00C112497
:10BCA0000D2C000CEE08FF08B12CA12C212CA8E2D1
:10BCB0003A2E81E090E0D4011496ED91FC916281DE
:10BCC0007381A301461B570B57FF03C05195419544
:10BCD0005109841795070CF4C0C08081982F929564
:10BCE00096959770963008F0BBC09F5F9295990F1C
:10BCF000907E8F71892BB3C0F20161857285DB0163
:10BD00008C91811154C60115110509F457C0D80151
:10BD100018968C9118978F70843009F04FC019963F
:10BD20006D917C91CE0101960E94F033CE01019677
:10BD30000E942D288823F1F12114310409F460C0F8
:10BD40004114510431F0F20180858F70843009F480
:10BD50004CC025961CAE1DAE1EAE1FAE2597299673
:10BD60001CAE1DAE1EAE1FAE299723961FAD2397A6
:10BD70001F7023961FAF239781E022968FAF2297E3
:10BD8000A12CCC24C394F12CE12C01E024962FADFE
:10BD9000249725963FAD259740E027965FAD2797DE
:10BDA00028966FAD289729967FAD2997CE010196E9
:10BDB0000E941941CE0101960E947C34D401149650
:10BDC000ED91FC9133822282D2CD6114710429F06D
:10BDD000F30180858F70843019F06FE27AE0E7C557
:10BDE00061857285FB0180818CCF61857285FB0145
:10BDF00080818823F9F2CE0101960F946C14DACF7A
:10BE00006114710431F0D30118968C918F708430D5
:10BE1000F1F025961CAE1DAE1EAE1FAE25972996DD
:10BE20001CAE1DAE1EAE1FAE299723961FAD2397E5
:10BE30001F7023961FAF239782E022968FAF229721
:10BE4000A12CCC24C394F12CE12C02E09FCFF30170
:10BE500061857285DB018C91CCCF80818F7180836D
:10BE60008081803A98F0C501BB0CAA0BBB0B8C15E6
:10BE70009D05AE05BF0551F0C101330CAA0BBB0BEC
:10BE80008C159D05AE05BF0509F071CD66157705CA
:10BE900009F46DCDA2961CAE1DAE1EAE1FAEA297CC
:10BEA000A0968FADA0978F708066A0968FAFA09759
:10BEB000A2968CAD9DADAEADBFADA29768968CAF8E
:10BEC0009DAFAEAFBFAF6897AAE0B0E0A701960103
:10BED0000F94B4276C966CAF7DAF8EAF9FAF6C970D
:10BEE00064E179E089ED90E10F94A6124AE050E018
:10BEF000F401638189ED90E10F94701062E179E0C3
:10BF000089ED90E10F94A612CE018C5A9F4F0E94AA
:10BF1000D8226AE576E0D4018D919C910E940EF8BA
:10BF2000B12CA12CD12CC12C6596EFAC65976696EF
:10BF3000FFAC669767960FAD679768961FAD6897D9
:10BF400069962FAD69976A963FAD6A976B964FAD2C
:10BF50006B976C965FAD6C976FEF0E9423E0F401D6
:10BF60000081118168ED75E0C8010E940EF87C0126
:10BF70006DED75E0C8010E940EF88C010097F1F19B
:10BF8000DC0118968C9118978F708430B9F519964A
:10BF90006D917C9140E450E0CE0101960F94852C88
:10BFA0006FE270E0CE0101960F944C2C892B51F476
:10BFB000F8012185328543E050E060E4CE0101962E
:10BFC0000E9495DB00E020E032E040E150E0BE015D
:10BFD0006F5B7F4FCE018C5A9F4F0E94B7200E940B
:10BFE0002CF8882359F08091C40B811107C0BE0141
:10BFF0006F5B7F4FCE0101960F94E304E114F104CF
:10C00000C9F1D70118968C9118978F70843091F5EB
:10C0100019966D917C91CE0101960E94F033CE016C
:10C0200001960E942D28882309F1A12CCC24C394C9
:10C03000F12CE12C65960FAD659766961FAD66975E
:10C0400067962FAD679768963FAD689769964FAD35
:10C0500069976A965FAD6A976B966FAD6B976C96B2
:10C060007FAD6C97CE0101960E941941CE010196D9
:10C070000E947C34D4011496ED91FC91738262820B
:10C0800076CC863009F456C070F4843009F45AC076
:10C09000853009F06CCC61E070E0CE018A599F4F89
:10C0A0000E948E7464CC883009F4E1C2803109F0BA
:10C0B0005ECC0F9446042B013C01C4010E947F1604
:10C0C000A12CB12C650110E3E12E15E7F12E00E063
:10C0D00010E0A30192010E94B8D5882309F447CC4F
:10C0E0006DED75E0D4018D919C910E940EF88C014C
:10C0F000009709F497C2FC0180858F70843009F0A5
:10C1000091C20F9446042AE0AE014F5F5F4F0F9437
:10C11000F2200E942CF8882309F484C28091C40B79
:10C12000811180C2BE016F5F7F4FD80119968D913A
:10C130009C9176C261E070E0CE0186599F4F0E94CB
:10C14000387615CC0F9446042B013C01C4010E94A3
:10C150007F16A12CB12C650118E9E12E1AE3F12E0E
:10C1600000E010E0A30192010E94B8D5882309F4F1
:10C17000FECBF401838127968FAF279796E128960F
:10C180009FAF2897282F30E0F901E754F54DE4914F
:10C190002996EFAF2997F901E150F54DE4912A96E0
:10C1A000EFAF2A9740E85EE360E070E062964CAF44
:10C1B0005DAF6EAF7FAF629762E00F9401000F94A6
:10C1C0004604605D7740810991092E966CAF7DAF82
:10C1D0008EAF9FAF2E9787E364968FAF6497CE01A3
:10C1E0008F5B9F4F0F946C05882349F028968FAD85
:10C1F00028978C3009F46FC048F48B3011F1412C32
:10C20000512C60EC662E6FE7762E47C08551823048
:10C21000B0F724961FAD2497612F70E0762F662724
:10C2200066277F7725968FAD2597682B90E080E075
:10C230000F942E262DEC3CEC4CEC5DE30F948F26F6
:10C2400068C024966FAD249770E090E080E00F9472
:10C250002E266B017C0125961FAD259717FF0AC07E
:10C26000AC019B0160E070E080E89FEB0F941C281C
:10C270006B017C011F70612F70E090E080E00F94F3
:10C2800030262DEC3CEC4CEC5DE30F948F26A7019F
:10C2900096010F941D282B013C01CE018F5B9F4F0F
:10C2A0000F946C05882309F4D7C128968FAD289781
:10C2B0008B3030F08D30B0F18551823008F4BAC146
:10C2C000312C212C30ECAF963FAFAF974FE7E09683
:10C2D0004FAFE0974DC024961FAD2497612F70E0BB
:10C2E00090E080E00F942E266B017C0125966FADC7
:10C2F00025976F7070E090E080E00F9430262DEC71
:10C300003CEC4CEC5DE30F948F26A70196010F9453
:10C310001D282B013C0117FFC0CF77FA709477F8E6
:10C320007094BBCF23966FAD239770E090E080E0D0
:10C330000F9430262DEC3CEC4CEC5DE30F948F26F3
:10C340006B017C0122966FAD229770E090E080E057
:10C350000F9430269B01AC01C701B6010F941D2834
:10C36000362E272EAF968FAFAF97E0969FAFE09710
:10C370006EE379E089ED90E10F94A6124AE050E077
:10C38000D40113966C9189ED90E10F9470106EE2D8
:10C3900079E089ED90E10F94A612B301A20189ED35
:10C3A00090E10F947E1067E279E089ED90E10F94BF
:10C3B000A612432D522DAF966FADAF97E0967FAD8D
:10C3C000E09789ED90E10F947E1065E279E089EDC8
:10C3D00090E10F94A61289ED90E10F945510F401AD
:10C3E0000081118160E277E0C8010E940EF8E596B5
:10C3F0009FAF8EAFE5976EE576E0C8010E940EF81C
:10C40000E7969FAF8EAFE797A3019201C301B201F8
:10C410000F94912981111FC019821A821B821C82DC
:10C420008A818F708067F82E8A83242D4D825E82E8
:10C430006F827886B12CA12CD12CC12CE9800B8184
:10C440001C813E814F8158856FEFE5968EAD9FAD83
:10C45000E5970E9423E0232D322DAF964FADAF9785
:10C46000E0965FADE097632D722DAF968FADAF97DD
:10C47000E0969FADE0970F949129811127C0198212
:10C480001A821B821C828A818F708067F82E8A83B1
:10C49000232D832D922DAF96AFADAF97E096BFAD14
:10C4A000E0978D839E83AF83B887B12CA12CD12CCC
:10C4B000C12CE9800B811C813E814F8158856FEF33
:10C4C000E7968EAD9FADE7970E9423E06DED75E096
:10C4D000D4018D919C910E940EF87C01009709F483
:10C4E000A1C0FC0180858F70843009F09BC020E0E2
:10C4F00030E0A901C301B2010F942926882309F471
:10C5000091C020E030E0A901632D722DAF968FAD70
:10C51000AF97E0969FADE0970F942926882309F402
:10C5200081C0A3019201C301B2010F942926811198
:10C5300079C0232D322DAF964FADAF97E0965FAD0A
:10C54000E097632D722DAF968FADAF97E0969FADBC
:10C55000E0970F942926811165C01A821982FE0185
:10C5600033968EE3DF011D928A95E9F7F701618525
:10C57000728540E450E08E010F5F1F4FC8010F9499
:10C58000852C6FE270E0C8010F944C2C892B51F47C
:10C59000D70119962D913C9143E050E060E4C80129
:10C5A0000E9495DB6CE178E0C8010F94412CB30147
:10C5B000A201CE018C5A9F4F0E94BDDC0E942CF834
:10C5C000882351F08091C40B811106C0BE016C5AC2
:10C5D0007F4FC8010F94FE04F80101900020E9F795
:10C5E0003197E01BF10BEC0FFD1F88E48083432D96
:10C5F000522DAF966FADAF97E0967FADE097CE012D
:10C600008C5A9F4F0E94BDDC0E942CF8882351F069
:10C610008091C40B811106C0BE016C5A7F4FC801C6
:10C620000F94FE040F944604AB01BC01C4010E94A8
:10C6300058169DC923966EAD7FAD23977627672741
:10C64000762790E080E00F942E262DEC3CEC4CEC0D
:10C650005DE30F948F2684CE312C212CF0ECAF9625
:10C66000FFAFAF972FE7E0962FAFE09781CE0F9403
:10C6700046042B013C01C4010E947F16A12CB12C61
:10C68000650118E9E12E1AE3F12E00E010E0A301A4
:10C6900092010E94B8D5882309F469C9D40114967F
:10C6A000ED91FC911597818113961C91811157C0D2
:10C6B000163008F03FC08CE0ECE4F2E0DE011196A9
:10C6C00001900D928A95E1F7E12FF0E0EE0FFF1F48
:10C6D000CC24C394D12CCC0EDD1EEC0DFD1D60E0EE
:10C6E00080810F9401006FEC76E183E01330C9F094
:10C6F00070F467ED76E181E0113099F063ED76E159
:10C7000082E0123071F06BED76E180E00AC06BECF4
:10C7100076E184E0143029F067EC76E185E01530AD
:10C7200091F70E941AFCD4011496ED91FC9181E0DE
:10C7300081831DC966E979E089ED90E10F94A61225
:10C740004AE050E0F401638189ED90E10F947010AC
:10C7500069E679E089ED90E10F94A61208C924E01A
:10C76000129FF0011124E451F54FC080D180E28086
:10C77000F38065E679E089ED90E10F94A6124AE036
:10C7800050E0D40113966C9189ED90E10F947010F4
:10C7900061E579E089ED90E10F94A6122AE030E09E
:10C7A000B701A60189ED90E10F944F116DED75E091
:10C7B000F401808191810E940EF88C01009709F4A8
:10C7C00043C0DC0118968C9118978F708430E1F586
:10C7D00019966D917C9140E450E0CE0101960F9442
:10C7E000852C6FE270E0CE0101960F944C2C892BC2
:10C7F00051F4F8012185328543E050E060E4CE0138
:10C8000001960E9495DBFF92EF92DF92CF9289EE24
:10C8100095E09F938F938E010F5B1F4F1F930F9394
:10C820000F94DC2C0E942CF80FB6F894DEBF0FBEDC
:10C83000CDBF882309F4F6CE8091C40B8111F2CECE
:10C84000B801CE010196ECCE62E479E083CF8FEFA0
:10C850009FEFC258DF4F0FB6F894DEBF0FBECDBFBB
:10C86000DF91CF911F910F91FF90EF90DF90CF90CC
:10C87000BF90AF909F908F907F906F905F904F9000
:10C880003F902F90089580E090E0DC01F401248136
:10C890003581F90142815381052E000C660B770B1F
:10C8A000481759076A077B0709F461C81C01D401BE
:10C8B0006D907C9068ED75E0C3010E940EF88C01CC
:10C8C0006DED75E0C3010E940EF87C0101151105A4
:10C8D00019F4892B09F472CA62EA75E0C3010E9457
:10C8E0000EF82C016DE975E0C3010E940EF83C01C1
:10C8F0006AE179E089ED90E10F94A6124AE050E0F8
:10C90000F401638189ED90E10F94701068E179E0A2
:10C9100089ED90E10F94A6124AE050E0B10189ED53
:10C9200090E10F94971189ED90E10F945510E11467
:10C93000F10409F4E8C9D70118968C9118978F7003
:10C94000843009F0E0C919966D917C9140E450E083
:10C95000CE0101960F94852C0E942CF8882309F4AF
:10C96000D2C98091C40B8111CEC96FE270E0CE01B3
:10C9700001960F944C2C892B51F4F70121853285B7
:10C9800043E050E060E4CE0101960E9495DB211463
:10C99000310409F41ACA4114510439F0D20118962D
:10C9A0008C918F70843009F4A7C964E27AE0CE01DB
:10C9B00001960F94E304A7C9AF92BF92DF92EF9262
:10C9C000FF920F931F93CF93DF9300D000D0CDB78A
:10C9D000DEB78C017B01D42EFB0184819581892BEC
:10C9E000F9F0A080B1806FE370E0C5010F944C2C8A
:10C9F0000097B1F09C012A193B0937FD11C050E0A6
:10CA000040E0B701CE0101960F94810DBE016F5F2A
:10CA10007F4FC7010F94B70CCE0101960F945F0DA5
:10CA2000F70184819581892BD9F1E080F18062E65C
:10CA300076E0C7010F94572C892B01F5F801128A73
:10CA4000118A80E090E19587848784E890E0948B58
:10CA5000838B81E08687D58A81E090E026960FB6A9
:10CA6000F894DEBF0FBECDBFDF91CF911F910F9124
:10CA7000FF90EF90DF90BF90AF9008956FE676E063
:10CA8000C7010F94572C892B59F4F801128A118A87
:10CA9000148A138A84E890E0958784871686DBCF12
:10CAA00090E080E0DBCFDC011296ED91FC911397D2
:10CAB0003097B9F016968D919C918430910541F094
:10CAC0008530910541F0039749F482E090E00895A4
:10CAD00081E090E0089581E190E00895808590E004
:10CAE000089590E080E00895089584E190E008952D
:10CAF000DC01ED91FC910684F785E02D60E019954D
:10CB000081E090E00895DC011496ED91FC9180E0C5
:10CB1000309711F085A1817090E00895E5E0F1E093
:10CB200080818F7980830895E5E0F1E080818066DF
:10CB3000808308958FE090E09093DA0C8093D90C75
:10CB400088EC90E00895009789F0FC0120852F7013
:10CB5000253061F40E94C0F8009741F0FC01208567
:10CB60002F70243019F481859285089590E080E03B
:10CB7000089567EC7BE1811102C069EC7BE18CE2F6
:10CB800090E10D94A61264EC78E18CE290E10F94B0
:10CB9000A612F0E0E0E0199584EF91E00895CF93BC
:10CBA000DF93EC016CEC71E289ED90E10F94A61239
:10CBB000EA81FB810190F081E02D6081718189ED36
:10CBC00090E10F94B01189ED90E10F945510E88138
:10CBD000F9810684F785E02D60E0CE01199581E0AA
:10CBE00090E0DF91CF910895CF93DF93EC01EC813A
:10CBF000FD8140815181052E000C660B770B22814F
:10CC000087E49DE00E9493BB70E060E08A819B8195
:10CC10000E943829ECEDFEE0828387E49DE0918359
:10CC200080831092E90F1092EB0F1092EA0FDF91C0
:10CC3000CF910895AF92BF92CF92DF92EF92FF9281
:10CC40000F931F93CF93DF9300D000D01F921F92BA
:10CC5000CDB7DEB7E982FA820B831C832D833E8336
:10CC60004F835887DC011296ED91FC91309781F14A
:10CC7000028113810115110559F1F80180858F702A
:10CC8000853031F57B01C8010E9452F9823000F1F4
:10CC900061E0C8010E94C0F80097D1F0DC0118964D
:10CCA0002C912F702630A1F4B7010E940EF8009746
:10CCB00079F0B12CA12CD12CC12CE980FA800B8108
:10CCC0001C812D813E814F8158856FEF0E9423E0AA
:10CCD00028960FB6F894DEBF0FBECDBFDF91CF917F
:10CCE0001F910F91FF90EF90DF90CF90BF90AF908A
:10CCF00008951F93CF93DF9300D000D0CDB7DEB758
:10CD00006230710591F06330710509F459C06130EA
:10CD1000710509F04BC09093E00E8093DF0E5093A5
:10CD2000E20E4093E10E82E009C09093E00E809302
:10CD3000DF0E5093E20E4093E10E83E00F947006F5
:10CD4000182F80E00E946DD66093BA0B7093BB0BD6
:10CD50008093BC0B9093BD0B1123D9F06AE173E271
:10CD600084E390E10F94A612812F90E0B0E0A0E060
:10CD700089839A83AB83BC8380E190E09E838D831B
:10CD8000BE016F5F7F4F84E390E10E94A0340F9457
:10CD9000551081E0111180E026960FB6F894DEBFA1
:10CDA0000FBECDBFDF91CF911F9108959093E00EFC
:10CDB0008093DF0E5093E20E4093E10E81E0BECFF0
:10CDC0009093E00E8093DF0E55275093E20E409330
:10CDD000E10E84E0B3CFCF93DF93EC016BE776E015
:10CDE00089ED90E10F94B011EA81FB810190F0810F
:10CDF000E02D6081718189ED90E10F9459108C8153
:10CE00009D81009711F00F94B91D70E060E08A8158
:10CE10009B810E9439281D821C8281E090E0DF9175
:10CE2000CF9108950D94B91D0D94B91D0D94B91DA0
:10CE3000CF93DF93EC016DEB71E289ED90E10F94FC
:10CE4000A612EA81FB810190F081E02D6081718161
:10CE500089ED90E10F94B01189ED90E10F94551098
:10CE6000E881F9810684F785E02D62E0CE0119950D
:10CE700081E090E0DF91CF910895DC01ED91FC918C
:10CE80000684F785E02D62E0199581E090E0089531
:10CE9000AF92BF92CF92DF92EF92FF920F931F93C8
:10CEA000CF93DF93EC018C819D81892B61F40A8102
:10CEB0001B8184E190E00F941D1DBC01C8010E94FC
:10CEC00039289D838C830C811D810115110569F41E
:10CED00066E073E284E390E10F94A61284E390E1AC
:10CEE0000F94551090E080E0A0C180E00E946DD6C4
:10CEF000D80116966D937D938D939C931997CC8052
:10CF0000DD80C114D104D9F0EA81FB813097B9F0FA
:10CF1000028113810115110591F0F80180858F7050
:10CF2000853069F4C8010E9452F9823040F0E090E7
:10CF3000310BF090320BE114F10409F086C069EC7A
:10CF400072E284E390E10F94A61261E070E08C81BC
:10CF50009D81892B11F470E060E04AE050E084E3A9
:10CF600090E10F94971167EC72E284E390E10F94E3
:10CF7000A61261E070E08A819B81892B11F470E038
:10CF800060E04AE050E084E390E10F94971165EC93
:10CF900072E284E390E10F94A612EA81FB8161E0E2
:10CFA00070E082819381892B11F470E060E04AE0A7
:10CFB00050E084E390E10F94971163EC72E284E314
:10CFC00090E10F94A612EA81FB810280F381E02DAB
:10CFD00080858F7061E070E0853011F470E060E072
:10CFE0004AE050E084E390E10F94971161EC72E223
:10CFF00084E390E10F94A612EA81FB818281938100
:10D000000E9452F961E070E0823010F070E060E060
:10D010004AE050E084E390E10F94971184E390E1BB
:10D020000F9455106EED72E284E390E10F94A61216
:10D0300084E390E10F945510E881F9810684F78527
:10D04000E02D61E0CE0119954DCF61E0C8010E944D
:10D05000C0F88C01DC0118968C9118978F70843081
:10D0600031F419966D917C916115710539F469EA75
:10D0700072E284E390E10F94A612D0CFC7010E9420
:10D080000EF87C01009771F467E872E284E390E1A6
:10D090000F94A612F8016185728584E390E10F94E4
:10D0A000B011BCCF6AE876E00E940EF8009709F450
:10D0B000DAC0DC0118962C9118972F70243009F0F3
:10D0C000D2C01996AD90BC9010E000E0A114B1045C
:10D0D00009F4BCC0B801615C7D4DC5010F945920B5
:10D0E000892B09F0ADC0F801ED5BFD4D2591349120
:10D0F000922F832FF6019283838361E976E0C70143
:10D100000E940EF8EC81FD81009709F4B4C0DC01A7
:10D1100018962C9118972F70223009F0ACC01996F0
:10D120004D915D916D917C911C9741155105610563
:10D13000710509F4A0C05183408340815181052EBF
:10D14000000C660B770B228187E49DE00E9493BB65
:10D1500066E976E0C7010E940EF86C010C811D8122
:10D16000009709F495C0FC0180858F70863009F026
:10D170008FC06BE976E0C6010E940EF8D8011B96BD
:10D180009C938E931A9760EA76E0C6010E940EF88F
:10D19000F8019587848764EA76E0C6010E940EF85C
:10D1A000D8011F969C938E931E976AEA76E0C6017B
:10D1B0000E940EF8F801918B808B6FEA76E0C60131
:10D1C0000E940EF8009709F45BC0DC0119968D915E
:10D1D0009C91F8019583848365EB76E0C7010E94FA
:10D1E0000EF8D80153969C938E93529761EF72E29A
:10D1F0008CE290E10F94A612EA81FB810190F0810C
:10D20000E02D608171818CE290E10F94B0118CE28D
:10D2100090E10F945510E881F9810684F785E02D9F
:10D2200062E0CE01199581E090E0DF91CF911F91EE
:10D230000F91FF90EF90DF90CF90BF90AF90089547
:10D240000A5F1F4F0834110509F040CF62E272E215
:10D2500089ED90E10F94A61289ED90E10F9455109D
:10D2600096E080E047CF86E090E0D60113969C934D
:10D270008E93129742CF80E895E2918380835DCFB1
:10D2800088EE93E0D80115969C938E931497A4CFC3
:10D29000F8011386128688EE93E0958384831586C1
:10D2A00014869ACF4F925F926F927F928F929F9245
:10D2B000AF92BF92CF92DF92EF92FF920F931F93A4
:10D2C000CF93DF93CDB7DEB768970FB6F894DEBF84
:10D2D0000FBECDBF098B1A8B2B8B3C8B4D8B5E8B7E
:10D2E0006F8B788FDC0112962D913C911397232B35
:10D2F00009F4E0C0CC2009F4DDC06C01ED91FC9193
:10D30000068CF78DE02D19955C0165EE71E289EDD3
:10D3100090E10F94A612CE0141960E94D822A1144A
:10D32000B10471F460E0CE0141960E94E91D682FBE
:10D33000F601848195810E94B9D081E090E0BCC063
:10D34000CE0141960E9495204C0184E0F2E0AF1698
:10D35000B10459F081E1A816B10409F447C081E095
:10D36000A1E0AA16B10409F485E019861A861B8685
:10D370001C861D861E861F86188A8295807F9A8548
:10D380009F70892B8A87EE24EA94FE2C09891A89DA
:10D390002B893C894D895E896F89788DCE010996EC
:10D3A0000E94D53B6BED71E289ED90E10F94A612DE
:10D3B000CE0109960E94D822B2E0AB16B10489F0E2
:10D3C000E1E1AE16B104B1F0AA94AB2809F0B5CFF3
:10D3D000188963E070E0C6010E94623B612F0E94E1
:10D3E000B9D06F85F6018481958151C0888D817097
:10D3F000888FBACF0FE710E08FEF88169806A9F054
:10D40000092C000CAA08BB08A5019401295931096F
:10D4100041095109AFEFB0E00F94B4272BE531E09B
:10D4200040E050E00F949527890163E070E0C60169
:10D430000E94623B5C01288930E0D8010F940128EA
:10D44000412C512C32014A94A30192010F9495274B
:10D45000622FC5010E94B9D064E070E0C6010E944D
:10D46000623B5C01AFEFB0E0A01BB10B288930E05C
:10D470000F940128A30192010F949527622FC501F3
:10D480000E94B9D06F85D60114968D919C910E940F
:10D49000B9D01E8561E070E0C6010E94623B612F39
:10D4A0000E94B9D01D8562E070E0C6010E94623B17
:10D4B000612F41CF90E080E068960FB6F894DEBF10
:10D4C0000FBECDBFDF91CF911F910F91FF90EF90D5
:10D4D000DF90CF90BF90AF909F908F907F906F9094
:10D4E0005F904F900895CF93DF93FC0122813381A9
:10D4F000232B59F1EC0162E271E289ED90E10F9486
:10D50000A6124AE050E06E8189ED90E10F94701010
:10D5100089ED90E10F9455108C819D810F94B91D78
:10D5200070E060E08A819B810E9439281D821C8204
:10D53000E881F9810684F785E02D60E0CE01199538
:10D5400081E090E0DF91CF91089590E080E0FACF04
:10D550006F927F928F929F92AF92BF92CF92DF9203
:10D56000EF92FF920F931F93CF93DF93EC018C8187
:10D570009D81892B09F4A8C08A819B81892B09F49C
:10D58000A3C03A014B01E881F9810484F585E02DBF
:10D59000CE011995039701F5EC81FD8180A591A538
:10D5A000A2A5B3A5892B8A2B8B2BB1F00F9446042F
:10D5B0009B01AC01EC81FD8160A571A582A593A5BD
:10D5C000A12CB12C650116E9E12EF12C00E010E050
:10D5D0000E94B8D5882301F38F81988521E0621AD3
:10D5E0007108DC01ED91FC910280F381E02DA30133
:10D5F000B40119958F819885DC01ED91FC91019022
:10D60000F081E02DD401129660E09D0128193909BE
:10D610002615370518F42D91620FF7CF19950C8157
:10D620001D8180E00E946DD6F80160A771A782A7D6
:10D6300093A767EC70E289ED90E10F94A6124AE09F
:10D6400050E06E8189ED90E10F94701063EC70E210
:10D6500089ED90E10F94A6128401C80188199909F7
:10D6600086159705B8F4D8016C9140E150E06A3016
:10D6700050F469EB76E089ED90E10F94B01140E150
:10D6800050E0F801608189ED90E10F9470100F5F18
:10D690001F4FE3CF89ED90E10F945510E881F98198
:10D6A0000684F785E02D63E0CE01DF91CF911F91D5
:10D6B0000F91FF90EF90DF90CF90BF90AF909F9031
:10D6C0008F907F906F901994DF91CF911F910F9160
:10D6D000FF90EF90DF90CF90BF90AF909F908F9092
:10D6E0007F906F900895CF92EF92FF920F931F93C8
:10D6F000CF93DF9300D000D01F921F92CDB7DEB73B
:10D700007C0109831A832B833C834D835E836F8363
:10D71000788763EB71E289ED90E10F94A612CE0158
:10D7200001960E94D822898181112AC00A810F7036
:10D73000013071F128F010E00230E9F5CC20E9F079
:10D7400060E0CE0101960E94E91DF701028113817C
:10D75000892B69F0C8010E94D628672B682B692B9A
:10D7600061F480E00E946DD6AB01BC0103C040E0D3
:10D7700050E0BA01C8010E947C2881E090E02EC0F0
:10D780008031D0F58E30D8F58130C9F18230D9F1B1
:10D7900066EA71E289ED90E10F94A6124AE050E04A
:10D7A000698189ED90E10F94701089ED90E10F94FB
:10D7B000551001E010E066E971E289ED90E10F9407
:10D7C000A6124AE050E0B80189ED90E10F9497115C
:10D7D00089ED90E10F94551090E080E028960FB607
:10D7E000F894DEBF0FBECDBFDF91CF911F910F9197
:10D7F000FF90EF90CF9008958351833048F6F70162
:10D8000002811381A7CF40E050E0BA01F701828185
:10D810009381B1CF4F925F926F927F928F929F923E
:10D82000AF92BF92CF92DF92EF92FF920F931F932E
:10D83000CF93DF93CDB7DEB72C970FB6F894DEBF4A
:10D840000FBECDBF6D7F6130710509F4C0C0DC0132
:10D850001296ED90FC90E114F10409F4B8C04C016B
:10D86000C7010E94D6282B013C0161E070E0C7018E
:10D870000E94F228411451046104710409F4A7C004
:10D8800020E030E04AE754E40F948F260F940229F9
:10D8900069877A878B879C87672B682B692B09F4AC
:10D8A00096C00F9446049B01AC01A12CB12C6501DC
:10D8B000E984FA840B851C85C301B2010E94B8D5A6
:10D8C000882309F484C0F4016280738070E060E012
:10D8D000C3010E94F22820E030E048EC52E40F94AB
:10D8E0008F260F9402296B017C0180E00E946DD687
:10D8F000AB01BC01C3010E947C2819821A821B82E1
:10D900001C821D821E821F8218868A818F708A83E4
:10D91000D40112966D917C9140E053E0CE010196C6
:10D920000E94FA30CE0101960E9449202B013C0151
:10D930006BEB76E089ED90E10F94B0112AE030E0D6
:10D94000B301A20189ED90E10F9453106AEC76E0E7
:10D9500089ED90E10F94B0112AE030E0B701A60103
:10D9600089ED90E10F94531089ED90E10F945510DB
:10D97000C40CD51CE61CF71C8A818F7080668A83D4
:10D98000CD82DE82EF82F886F4016281738140E00D
:10D9900052E0CE0101960E943B306EEC76E089EDBC
:10D9A00090E10F94B0112AE030E0B701A60189EDB3
:10D9B00090E10F94531089ED90E10F94551060E0C1
:10D9C00072E0D40112968D919C910E948D3190E06D
:10D9D00080E02C960FB6F894DEBF0FBECDBFDF916E
:10D9E000CF911F910F91FF90EF90DF90CF90BF905C
:10D9F000AF909F908F907F906F905F904F90089521
:10DA0000CF92DF92EF92FF920F931F93CF93DF930A
:10DA1000CDB7DEB762970FB6F894DEBF0FBECDBFAD
:10DA20006C010B871C872D873E874F87588B698B2E
:10DA30007A8B61E971E2C7010F945920EEE0F0E0C2
:10DA4000892BF1F06BE871E2C7010F945920E0E1F6
:10DA5000F0E0892BA9F065E871E2C7010F94592025
:10DA6000EFE0F0E0892B61F01F7061E871E2C7011F
:10DA70000F945920E12FF0E0892B11F4EDE0F0E054
:10DA80009B85992341F0309731F4EF2809F461C068
:10DA90008FEF9FEF96C0E131F10508F03CC0882779
:10DAA000EB5AF2498F4F0D94EA27486DA96D666DC8
:10DAB0008B6D8B6D8B6D8B6D346E7C6E8B6D8B6D0A
:10DAC0008B6D8B6D8B6D866ECF6E946ECE010B96CB
:10DAD0000E94511F20EF260F2931D0F6D60114964F
:10DAE000ED91FC91159723A39B01AC0133274427AB
:10DAF00055271296ED91FC9113970190F081E02D3E
:10DB000060817181ED91FC910088F189E02D03EE37
:10DB100016E0C6011995D6011496ED91FC91159762
:10DB2000118A1496ED91FC91159781E081871496E6
:10DB3000ED91FC9115978DE482871496ED91FC91FF
:10DB400015978FE5838714966D917C9145E250E09F
:10DB500033C0F601A481B58191509531E0F6E92FEB
:10DB6000F0E08827E954F2498F4F0D94EA27CC6DF5
:10DB7000F06D8B6D8B6DF06DCC6D8B6D8B6D8B6DDA
:10DB80008B6D8B6D8B6D8B6D016E196E8B6D8B6DCF
:10DB90008B6D156E116E176E95968C9195975D969F
:10DBA0008C93D6011496ED91FC91858D8160858FC3
:10DBB0004DE050E06AE172E0C6010E94A86A81E08F
:10DBC00090E062960FB6F894DEBF0FBECDBFDF9136
:10DBD000CF911F910F91FF90EF90DF90CF9008951C
:10DBE00095968C9195975D968C93D6011496ED91B0
:10DBF000FC91858D8E7F858F4DE050E06DE072E069
:10DC0000DBCF57961C92D6011496ED91FC91159797
:10DC100085A1858F1496ED91FC91858D8160858F0E
:10DC20007ACF81E057968C93EECF82E0FBCF84E0F1
:10DC3000F9CF83E057968C93D6011496ED91FC9121
:10DC4000159785A1858F1496ED91FC911597858D7B
:10DC50008160858F1496ED91FC91818D833009F060
:10DC60005ACF82E0818F57CF1982F6010481158146
:10DC70009031B1F150F49E3091F0CE010B960E949C
:10DC8000511FD80159966C9314C0913171F19231A2
:10DC9000A1F782E0F801818F6CE671E206C083E0B3
:10DCA000D80159968C936CE771E2CE0101960F94DE
:10DCB0006220D6011296ED91FC9113970190F081AC
:10DCC000E02D60817181ED91FC910488F589E02D52
:10DCD00028EE36E0AE014F5F5F4FC60119951BCFAE
:10DCE000F801118E67E771E2E0CF81E0D801599623
:10DCF0008C9360E771E2D9CFCE010B960E94511F41
:10DD0000D6011496ED91FC91678B05CFD601149640
:10DD1000ED91FC91913029F0923009F0FCCE148EF7
:10DD2000FACE80E5848FF7CEF6010481158191301B
:10DD300049F09230F1F0CE010B960E94511FF8018C
:10DD4000638FE9CE83E0D8015B968C93D601028085
:10DD5000F381E02D0190F081E02D60817181ED91E2
:10DD6000FC910488F589E02D2DEE36E044E25AE07E
:10DD7000B4CFF801138ED6011296ED91FC91139752
:10DD80000190F081E02D60817181ED91FC9104881A
:10DD9000F589E02D2DEE36E04FE25AE09ECFD60118
:10DDA0001496ED91FC91913031F0923009F0B3CEA0
:10DDB000858D877F34CF858D886031CFCF93C1E04B
:10DDC00068EE73E080E090E00F9446024AE050E095
:10DDD0006C2F8CE290E10F947010CF5FC43181F70B
:10DDE00084EF91E0CF9108954F925F926F927F926E
:10DDF0008F929F92AF92BF92CF92DF92EF92FF925B
:10DE00000F931F93CF93DF93CDB7DEB7C258D109DD
:10DE10000FB6F894DEBF0FBECDBFDC0114962D9176
:10DE20003C911597232B09F49AC43B014C01ED91C9
:10DE3000FC910484F585E02D199597FD40C0823052
:10DE400091050CF48CC40397D1F5D4011496ED918F
:10DE5000FC9180A591A5A2A5B3A5892B8A2B8B2B1C
:10DE600071F10F9446049B01AC01D4011496ED911D
:10DE7000FC9160A571A582A593A5A12CB12C65018B
:10DE800016E9E12EF12C00E010E00E94B8D58823BD
:10DE9000B1F0D401ED91FC910684F785E02D62E0AC
:10DEA000C4011995F401E480F58080E00E946DD6EC
:10DEB000D70198966D937D938D939C939B9790E05B
:10DEC00080E06A94672809F04CC4D401ED91FC917C
:10DED0000484F585E02DC4011995029731F50F945E
:10DEE00046049B01AC01D4011496ED91FC9160A510
:10DEF00071A582A593A5A12CB12C650118E8E12E8E
:10DF000013E1F12E00E010E00E94B8D5882369F0FB
:10DF100060E671E289ED90E10F9458174DE050E012
:10DF200060E072E0C4010E94A86AF40187819085D4
:10DF3000DC01ED91FC910084F185E02D1995859728
:10DF40000CF427C3F4016481758145E250E08781B8
:10DF500090850F945C0FD40117968D919C91DC01F4
:10DF6000ED91FC910084F185E02D19957C01892BC0
:10DF700089F062E070E080E090E00F944602F401E6
:10DF800087819085DC01ED91FC910284F385E02D81
:10DF90001995E1CF6BE571E289ED90E10F94A6123E
:10DFA0004AE050E0F401668189ED90E10F94701031
:10DFB00066E571E289ED90E10F94A612D401149602
:10DFC000ED91FC91EE0DFF1D608140E150E06A3063
:10DFD00078F469EB76E089ED90E10F94B011D4010B
:10DFE0001496ED91FC91EE0DFF1D40E150E0608133
:10DFF00089ED90E10F947010BFEFEB1AFB0AE4E299
:10E00000EE16F104D9F6D4011496ED91FC91159712
:10E0100084A197A1891709F4B8C287A31496ED913A
:10E02000FC91EF961CAE1DAE1EAE1FAEEF97C15811
:10E03000DF4F188219821A821B82CF57D040ED968B
:10E040008FADED978F70ED968FAFED9783A190E038
:10E050006C01B0E1CB0ED11C499708F090C2B58499
:10E06000878986A3118D738CD40114962D913C91D0
:10E07000858DD90195968C93E48CF12C878DF401D4
:10E0800020813181A281B3810D90BC91A02D6D9131
:10E090007C91D9015496ED91FC9124EF36E044E255
:10E0A0005AE080FD02C04FE25AE0C4011995B0E881
:10E0B000EB16F10409F09CC0D4011296ED91FC918D
:10E0C00013970190F081E02D60817181ED91FC91B9
:10E0D0000488F589E02D2BEF36E044E25AE0C401D4
:10E0E000199561E077E089ED90E10F94B011D401CA
:10E0F0001496ED91FC914AE050E065A189ED90E124
:10E100000F94701089ED90E10F945510D40114967E
:10E11000ED91FC91159785A12D913C911197129647
:10E120000D90BC91A02D0D90BC91A02D6D917C9176
:10E13000D9015496ED91FC912CE037E044E25AE08D
:10E1400083FD02C04FE25AE0C4011995D401ED915C
:10E15000FC9111970488F589E02D12968D919C9180
:10E16000DC018D919C91DC016D917C91D401149620
:10E170008D919C91DC0195968C9123E137E044E2EE
:10E180005AE081FD02C04FE25AE0C401199519829C
:10E19000113009F401C208F442C0123009F421C25E
:10E1A000133009F443C26BE471E2CE0101960F947F
:10E1B000622060E0CE0185589F4F0E94011B64964B
:10E1C0002FAF649765963FAF659766964FAF66979A
:10E1D00067965FAF679768966FAF689769967FAFEE
:10E1E00069976A968FAF6A976B969FAF6B973BC0A4
:10E1F000EF2809F076CFD4011296ED91FC91139798
:10E200000190F081E02D60817181ED91FC91048895
:10E21000F589E02D2BEF36E04FE25AE060CF67E75B
:10E2200071E2CE0101960F94622060E1CE01855823
:10E230009F4F0E94011BE4962FAFE497E5963FAFF6
:10E24000E597E6964FAFE697E7965FAFE797E896D4
:10E250006FAFE897E9967FAFE997EA968FAFEA97B5
:10E26000EB969FAFEB97D4011296ED91FC9113972B
:10E270000190F081E02D60817181ED91FC91048825
:10E28000F589E02D28EE36E0AE014F5F5F4FC40107
:10E290001995EC96EFACEC97ED96FFACED97EE96FA
:10E2A0000FADEE97EF961FADEF97C158DF4F288166
:10E2B000CF57D040C058DF4F3881C058D040CF57DB
:10E2C000DF4F4881C158D040CE57DF4F5881C258E8
:10E2D000D04069EE76E0C4010E941A66F4018081A4
:10E2E0009181A281B3810D90BC91A02D6D917C9103
:10E2F000DC015496ED91FC912DEE36E04FE25AE0B0
:10E30000772011F044E25AE0C40119950D2C000C5D
:10E31000EE08FF08D4011296ED91FC91139701903D
:10E32000F081E02D60817181ED91FC910088F1898F
:10E33000E02D03EE16E0A7019601C40119954B2CC0
:10E34000512C712C612CBFEFBB16A9F0D401129691
:10E35000ED91FC9113970190F081E02D6081718126
:10E36000ED91FC910088F189E02D0FE117E0A30108
:10E370009201C40119951B861C861D861E861F8668
:10E38000188A198A1A8A8C858F708C87B701A60122
:10E39000CE010B960E94671D2C962FAF2C972D96C1
:10E3A0003FAF2D972E964FAF2E972F965FAF2F979B
:10E3B00060966FAF609761967FAF619762968FAFFF
:10E3C000629763969FAF639779018A019B01AC01C5
:10E3D00064EE76E0C4010E941A661B861C861D86C8
:10E3E0001E861F86188A198A1A8A8C858F708C87D8
:10E3F000B301A201CE010B960E94671D2B8B3C8BB3
:10E400004D8B5E8B6F8B788F898F9A8F63E0CE01F7
:10E4100043960E94DA1A24962FAF249725963FAF91
:10E42000259726964FAF269727965FAF2797289672
:10E430006FAF289729967FAF29972A968FAF2A9793
:10E440002B969FAF2B9779018A019B01AC0160E26B
:10E4500077E0C4010E941A661982D4011496ED91E6
:10E46000FC9186A1811107C16CE771E2CE01019692
:10E470000F9462206EE0CE0185589F4F0E94011BD1
:10E480002BAF3CAF4DAF5EAF6FAF21967FAF219703
:10E4900022968FAF229723969FAF2397D40114968D
:10E4A000ED91FC91159726A130E050E040E01296E6
:10E4B000ED91FC9113970190F081E02D60817181C5
:10E4C000ED91FC910088F189E02D05E217E0C4018F
:10E4D0001995D4011496ED91FC9185A180FD14C08D
:10E4E00060E371E2CE0101960F94622062E0CE01FA
:10E4F00085589F4F0E94011B2B873C874D875E8765
:10E500006F87788B898B9A8BD4011296ED91FC9151
:10E5100013970190F081E02D60817181ED91FC9164
:10E520000488F589E02D2BE237E0AE014F5F5F4FA5
:10E53000C4011995EC96EFACEC97ED96FFACED9716
:10E54000EE960FADEE97EF961FADEF97C158DF4FE8
:10E550002881CF57D040C058DF4F3881C058D040B5
:10E56000CF57DF4F4881C158D040CE57DF4F588139
:10E57000C258D0406CE277E0C4010E941A666FE492
:10E5800071E289ED90E10F94A61289ED90E10F946C
:10E59000551081E090E0E5C060E771E2CE010196A0
:10E5A0000F94622061E1CE0185589F4F0E94011BAC
:10E5B000AC962FAFAC97AD963FAFAD97AE964FAF41
:10E5C000AE97AF965FAFAF97E0966FAFE097E196EB
:10E5D0007FAFE197E2968FAFE297E3969FAFE39725
:10E5E00042CE6CE671E2CE0101960F94622062E1A8
:10E5F000CE0185589F4F0E94011BA4962FAFA49770
:10E60000A5963FAFA597A6964FAFA697A7965FAFE3
:10E61000A797A8966FAFA897A9967FAFA997AA9634
:10E620008FAFAA97AB969FAFAB971DCE6CE771E209
:10E63000CE0101960F9462206EE0CE0185589F4F67
:10E640000E94011B6C962FAF6C976D963FAF6D9734
:10E650006E964FAF6E976F965FAF6F97A0966FAF46
:10E66000A097A1967FAFA197A2968FAFA297A396EE
:10E670009FAFA397F8CD8130A9F466E471E2CE0193
:10E6800001960F94622064E1CE0185589F4F0E944D
:10E69000011B2BAB3CAB4DAB5EAB6FAB78AF89AF27
:10E6A0009AAFFCCE8230A9F461E471E2CE0101960A
:10E6B0000F94622063E1CE0185589F4F0E94011B99
:10E6C0002BA73CA74DA75EA76FA778AB89AB9AABEA
:10E6D000E5CE8330A9F468E371E2CE0101960F9490
:10E6E00062206FE0CE0185589F4F0E94011B2BA333
:10E6F0003CA34DA35EA36FA378A789A79AA7CECE0C
:10E700008430A9F464E371E2CE0101960F94622093
:10E7100065E1CE0185589F4F0E94011B2B8F3C8FD6
:10E720004D8F5E8F6F8F78A389A39AA3B7CE8D3656
:10E7300009F0B4CE6BE471E2CE0101960F94622031
:10E7400060E0CE0185589F4F0E94011B2B8B3C8BB4
:10E750004D8B5E8B6F8B788F898F9A8F9FCE8FEFCB
:10E760009FEFCE57DF4F0FB6F894DEBF0FBECDBF81
:10E77000DF91CF911F910F91FF90EF90DF90CF909D
:10E78000BF90AF909F908F907F906F905F904F90D1
:10E7900008950F931F93CF93DF93DC0112962D9171
:10E7A0003C91232B81F1EC0167E171E289ED90E16D
:10E7B0000F94A6124AE050E06E8189ED90E10F942B
:10E7C000701089ED90E10F9455108C819D81892BFB
:10E7D00061F40A811B818CE290E00F941D1DBC0145
:10E7E000C8010E9439289D838C83EC81FD8130977C
:10E7F00069F465E071E284E390E10F94A61284E38A
:10E8000090E10F94551090E080E044C085E2DF0174
:10E810001D928A95E9F7EC81FD8116A2EC81FD81BC
:10E8200015A2EC81FD8117A20C811D8180E00E9460
:10E830006DD6F80160A771A782A793A78E81811179
:10E8400016C062E00F9401006CEC70E28CE290E183
:10E850000F94A6128CE290E10F9455108CE390E196
:10E860000E948FAB1092310281E08093C80B26E0AA
:10E8700040E855E260E070E08F8198850E9493BB8C
:10E88000E881F9810684F785E02D62E0CE011995D3
:10E8900081E090E0DF91CF911F910F910895EF9269
:10E8A000FF921F93CF93DF93192F7B01C82FD92F8E
:10E8B000D7FF03C0D195C195D10961E08C2F0F948A
:10E8C000010082E0E816F10499F460E08C2F0E94C8
:10E8D000D3FF65E27FE189ED90E10F94A61289ED07
:10E8E00090E1DF91CF911F91FF90EF900D94551023
:10E8F000612FEF2851F46095661F6627661F8C2FE5
:10E900000E94D3FF61E27FE1E6CF661F6627661FA4
:10E910008C2F0E94D3FF6CE17FE1DDCF2F923F92DD
:10E920004F925F926F927F928F929F92AF92BF921F
:10E93000CF92DF92EF92FF920F931F93CF93DF93CB
:10E94000CDB7DEB766970FB6F894DEBF0FBECDBF6A
:10E950004C018091B90B6CEA70E2882309F47DC107
:10E9600060E083E00E94D3FF61E070E080E090E02F
:10E970000F944602BE016F5F7F4F80E00E9430FD22
:10E98000892B09F068C1898183FF65C144E0BE011C
:10E990006F5F7F4F82E00E94DBFC009791F429813A
:10E9A0003A813227232732273093A90E2093A80ECD
:10E9B0002B813C813227232732273093A70E2093C7
:10E9C000A60E0F947A1260E377E089ED90E10F9440
:10E9D000B0116091A80E7091A90E90E080E00F94A4
:10E9E0002E26362E272E898B492E462F572F682FFD
:10E9F000792F89ED90E10F947E1066E377E089ED41
:10EA000090E10F94B0116091A60E7091A70E90E066
:10EA100080E00F942E26562E7A8B8B8B9C8B462F64
:10EA2000572FBC0189ED90E10F947E106EE377E0E3
:10EA300089ED90E10F94B01142E0BE016F5F7F4F0E
:10EA400081E10E94DBFC49815A81542745275427E4
:10EA5000892B11F050E040E070E060E04093B50B8E
:10EA60005093B60B6093B70B7093B80B2AE030E06D
:10EA700089ED90E10F944F1120E030E44CE156E431
:10EA8000632D722D8989942D0F94292687FF78C0D4
:10EA9000D4011296ED91FC91608071806AE477E078
:10EAA000C3010E940EF89E8B8D8B6EE477E0C3014C
:10EAB0000E940EF83C0119821A821B821C828A81F4
:10EAC0008F708067F82E8A83232D832D922DA9893C
:10EAD000B42D8D839E83AF83B887B12CA12CD12C0C
:10EAE000C12CE9800B811C813E814F8158856FEFDD
:10EAF0008D899E890E9423E019821A821B821C82C2
:10EB00008A818F708067F82E8A83252D852D9A89BA
:10EB1000AB89BC898D839E83AF83B887E9800B81E5
:10EB20001C813E814F8158856FEFC3010E9423E015
:10EB300023E537E0432D522D6989742DC4010E94CD
:10EB4000AD3B28E537E0452D5A896B897C89C401A6
:10EB50000E94AD3B6091B50B7091B60B8091B70BE5
:10EB60009091B80B2AE0AE014F5F5F4F0F94F220F7
:10EB70004EE557E0BE016F5F7F4FC4010E94773BB7
:10EB800064E677E089ED90E10F945910BE016F5F64
:10EB90007F4F80EE0E9430FD892B19F419811F3FB1
:10EBA00029F566E677E089ED90E10F94591061E070
:10EBB00083E00E94D3FF81E090E066960FB6F89460
:10EBC000DEBF0FBECDBFDF91CF911F910F91FF90A0
:10EBD000EF90DF90CF90BF90AF909F908F907F90FD
:10EBE0006F905F904F903F902F90089515FF06C053
:10EBF00067E877E089ED90E10F94B01114FF06C04B
:10EC00006BE977E089ED90E10F94B01113FF06C036
:10EC10006EEA77E089ED90E10F94B01112FF06C023
:10EC200063EC77E089ED90E10F94B01111FF06C01D
:10EC30006AED77E089ED90E10F94B01110FF06C006
:10EC400060EF77E089ED90E10F94B01189ED90E1EC
:10EC50000F945510ACCF61E970E289ED90E10F940B
:10EC6000A61289ED90E10F94551090E080E0A5CFB9
:10EC70002F923F924F925F926F927F928F929F92CC
:10EC8000AF92BF92CF92DF92EF92FF920F931F93BA
:10EC9000CF93DF93CDB7DEB72E970FB6F894DEBFD4
:10ECA0000FBECDBF6130710579F42C018091B40B9A
:10ECB000811125C069E770E289ED90E10F94A612F9
:10ECC00089ED90E10F94551090E080E02E960FB6FC
:10ECD000F894DEBF0FBECDBFDF91CF911F910F9192
:10ECE000FF90EF90DF90CF90BF90AF909F908F906C
:10ECF0007F906F905F904F903F902F90089562E0CB
:10ED000078E089ED90E10F94B01182E00F947902E0
:10ED1000892E912C40E150E0B40189ED90E10F94EF
:10ED20009E118FEF8816910409F42CC16EE078E0F3
:10ED300089ED90E10F94B01180E00F947902BC014D
:10ED400090E080E00F942E2620E030E040E857E38A
:10ED50000F948F2620E030E045E253E40F948F2695
:10ED600020E030E040E252E40F941C28962E672EFB
:10ED7000782E892E462F572F682F792F89ED90E115
:10ED80000F947E1062E178E089ED90E10F94B0116C
:10ED900081E00F947902BC0190E080E00F942E2670
:10EDA00020E030E040E857E30F948F2620E030E089
:10EDB00048EC52E40F948F26362E272E89879A87A7
:10EDC000462F572FBC0189ED90E10F947E1069E129
:10EDD00078E089ED90E10F945910D2011296ED91EF
:10EDE000FC91E080F18060E277E0C7010E940EF8BC
:10EDF0009C878B876EE576E0C7010E940EF89E87A0
:10EE00008D87292D362D472D582D692D762D872D4F
:10EE1000982D0F94912981113EC019821A821B826C
:10EE20001C828A818F708067F82E8A83292D892D14
:10EE3000962DA72DB82D8D839E83AF83B887B12CD7
:10EE4000A12CD12CC12CE9800B811C813E814F81EA
:10EE500058856FEF8B859C850E9423E019821A826A
:10EE60001B821C828A818F708067F82E8A83232DF3
:10EE7000832D922DA985BA858D839E83AF83B88714
:10EE8000E9800B811C813E814F8158856FEF8D8514
:10EE90009E850E9423E02BE138E0492D562D672DF9
:10EEA000782DC2010E94AD3B2EE138E0432D522D5A
:10EEB00069857A85C2010E94AD3B8091B90B882398
:10EEC00009F45DC020E030E048EC51EC692D762D6E
:10EED000872D982D0F94292687FD51C020E030E022
:10EEE00048E452E4692D762D872D982D0F94312911
:10EEF00018160CF444C020E030E048EC52E4632DD6
:10EF0000722D89859A850F9431291816C4F120E055
:10EF100030E04AE754E4632D722D89859A850F9479
:10EF20008F260F94022966507F4F8F4F9F4F24EFFB
:10EF3000C22EDD24D394E12CF12CA70196010F946D
:10EF4000732729831A8220E030E04AE754E4692DD0
:10EF5000762D872D982D0F948F260F9402296E55AC
:10EF60007D498F4F9F4FA70196010F9473272B83E5
:10EF70001C82BE016F5F7F4F85E00E94A1FC88EE7E
:10EF800093E0A4CE0E941AD6FACFEF92FF920F938D
:10EF90001F93CF93DF93CDB7DEB760970FB6F8948A
:10EFA000DEBF0FBECDBF8091B40B8823C9F06AE5E8
:10EFB00070E289ED90E10F94A61289ED90E10F9433
:10EFC000551090E080E060960FB6F894DEBF0FBE5B
:10EFD000CDBFDF91CF911F910F91FF90EF900895DA
:10EFE00061E278E089ED90E10F9459100E948AFC6B
:10EFF00080E48093B20E0E948AFC10E01B7F809117
:10F00000B20E0E9480FC62E08FE89EE00E9441AE5A
:10F01000612F8FE89EE00E9441AE60E08FE89EE0A5
:10F020000E9441AE8FE89EE00E948CD26AE070E0C0
:10F0300080E090E00F9446026FE278E089ED90E185
:10F040000F94B0118EEF0F947902AC0170E060E084
:10F0500020E189ED90E10F94071089ED90E10F9484
:10F06000551062E478E089ED90E10F94B0118FEFD4
:10F070000F947902AC0170E060E020E189ED90E14D
:10F080000F94071089ED90E10F9455106FE478E02C
:10F0900089ED90E10F94B0118BEF0F947902182F46
:10F0A000092F8CEF0F947902F82EE92E8DEF0F9433
:10F0B00079029F938F93EF92FF920F931F9385E6B0
:10F0C00098E09F938F938E010F5F1F4F1F930F93B5
:10F0D0000F94DC2CB80189ED90E10F94591081E078
:10F0E0008093B40B0FB6F894DEBF0FBECDBF81E0A6
:10F0F00090E069CF0F931F93CF93DF9300D000D0A0
:10F100001F92CDB7DEB78091B90B882369F06CE30D
:10F1100070E284E390E10F94A61284E390E10F94EF
:10F12000551090E080E0BBC061E083E00F940100E7
:10F1300060E083E00E94D3FF64E778E08CE290E136
:10F140000F9459100E948AFC88EC8093B80080913B
:10F15000180490911904A0911A04B0911B0489839A
:10F160009A83AB83BC838FE89EE090939C0E809340
:10F170009B0E1E8280E197E22E812F5F2E830197E6
:10F18000D9F71D82BE016B5F7F4F80E20E9430FD88
:10F190008C01892BF1F48D8101E010E08138C9F4F4
:10F1A000BE016F5F7F4F8FEF0E94A1FC1F8280E83E
:10F1B0009EE32F812F5F2F830197D9F7BE016B5FED
:10F1C0007F4F80E00E9430FD8D8180FF0CC003E006
:10F1D00010E060E878E084E390E10F94B011C8019A
:10F1E0000F947A129ECFBE016B5F7F4F80E00E942A
:10F1F00030FD892B61F78D8184FFE9CF80919D0ED1
:10F200000E9480FC80919B0E90919C0EDC01ED9100
:10F21000FC910190F081E02D64EF199580919B0E97
:10F2200090919C0E0E948CD2882319F002E010E08D
:10F23000D0CFBE016B5F7F4F81E00E9430FD8C011B
:10F24000892B39F61D811F7810611D8380919D0ED9
:10F250000E9480FC80919B0E90919C0EDC01ED91B0
:10F26000FC910190F081E02D61E0199580919B0E59
:10F2700090919C0EDC01ED91FC910190F081E02DCC
:10F28000612F199580919B0E90919C0E0E948CD2BB
:10F290008111CCCF81E08093B90B81E090E027967B
:10F2A0000FB6F894DEBF0FBECDBFDF91CF911F9197
:10F2B0000F910895CF93DF9300D000D01F921F923B
:10F2C000CDB7DEB7E6E1F0E1128A118A80E090E185
:10F2D0009587848784E890E0948B838B81E0868790
:10F2E00087E7858B1C821B828BEA94E09A83898353
:10F2F000FE83ED838FEF9FEF98878F836CEB7FE129
:10F300008CE290E10F94A61260912E0B70912F0B5E
:10F31000CE0101960E943EBF86E190E10E949317C4
:10F320006CEA7FE18CE290E10F94A6128CE290E10E
:10F330000F9455100F944B1328960FB6F894DEBF18
:10F340000FBECDBFDF91CF910895CF93DF93EB0137
:10F350000297B4F164EC7BE18A819B810F943B209E
:10F36000892B29F40F947F0F6F770E945BFB60EC71
:10F370007BE18A819B810F943B20892B29F40F9498
:10F380007F0F60680E945BFB68EC7AE18CE290E1A1
:10F390000F94A6120F947F0F6095661F6627661F55
:10F3A00070E04AE050E08CE290E10F9497118CE21B
:10F3B00090E10F94551088EC90E0DF91CF91089583
:10F3C0000E945A79F8CF892B71F0FB0182819381D9
:10F3D0000F94191260E47BE18CE290E10F94A61285
:10F3E00088EC90E0089590E080E0F2CF892B71F0F6
:10F3F000FB01828193810F94B81169E27BE18CE279
:10F4000090E10F94A61288EC90E0089590E080E0DF
:10F41000F2CFEF92FF920F931F93CF93DF93CDB76D
:10F42000DEB72C970FB6F894DEBF0FBECDBF8C01B0
:10F430007B018DE895E09A8389831B821C821D8263
:10F440001E8298878F8319861A861B861C86053034
:10F450001105ECF0BE01695F7F4FF7018085918552
:10F460000E947FDC892B99F0CE0107960E9420FA3A
:10F47000BE01695F7F4FF701868197810E947FDC23
:10F48000892B61F0CE0107960E94F2FA0EC0CE01E0
:10F4900001960E9420FA0430110554F7CE0101961E
:10F4A0000E94F2FA03301105A4F1BE01695F7F4F9B
:10F4B000F701848195810E947FDC892B51F1CE0177
:10F4C00007960E9489FABE01695F7F4FF70182812A
:10F4D00093810E947FDC892B19F1CE0107960E944F
:10F4E000B7F962E07BE18CE290E10F94A61280E034
:10F4F0000F94D90F88EC90E02C960FB6F894DEBFED
:10F500000FBECDBFDF91CF911F910F91FF90EF9074
:10F510000895CE0101960E9489FA023011059CF6E9
:10F52000CE0101960E94B7F901301105D1F6CE0146
:10F5300001960E94B7F969E07BE18CE290E10F94BB
:10F54000A612CFCF0F931F93CF93DF938C01EB01C4
:10F550000297C4F08A819B810F94ED1F8093310242
:10F5600099270F94E20F0230110549F08C819D819B
:10F570000F94ED1F8093300299270F94EC0FC8EC85
:10F58000D0E002C0C0E9D1E06EEE7AE18CE290E119
:10F590000F94A6124AE050E0609131028CE290E1B3
:10F5A0000F94701069ED7AE18CE290E10F94A6124D
:10F5B0004AE050E0609130028CE290E10F947010CC
:10F5C0008CE290E10F945510CE01DF91CF911F9105
:10F5D0000F910895CF92DF92EF92FF920F931F93B6
:10F5E000CF93DF93CDB7DEB769970FB6F894DEBF40
:10F5F0000FBECDBFE091C50BF091C60B309709F45B
:10F6000083C08091DD0C9091DE0C892B09F47CC0C5
:10F610008FEF8387148613821482158216821782D5
:10F6200010861186128665EE78E18CE290E10F94E7
:10F63000A6128CE290E10F9455108E010F5E1F4FC1
:10F64000BE016E5E7F4F8091C50B9091C60B0E94EC
:10F6500016D518160CF058C0A895DE0111969E011B
:10F660002E5E3F4F7D01F90141919F01842F90E073
:10F6700054E0959587955A95E1F7845B9B4FFC0183
:10F6800080818C93E42FEF70F0E0E45BFB4F80818E
:10F6900011968C9311971296A017B10721F7198A2A
:10F6A000B7018091DD0C9091DE0C0E940EF86C0188
:10F6B00060EE78E18CE290E10F94A612B7018CE243
:10F6C00090E10F94B011C114D104B9F0C6010E94A9
:10F6D000DCDE7C01892B09F4B3CF6BED78E18CE2A1
:10F6E00090E10F94A612B7018CE290E10F94B01153
:10F6F0008CE290E10F945510A3CF66ED78E18CE297
:10F7000090E10F94A612F4CF88EC90E069960FB6C2
:10F71000F894DEBF0FBECDBFDF91CF911F910F9147
:10F72000FF90EF90DF90CF900895CF92DF92EF920D
:10F73000FF920F931F93CF93DF93CDB7DEB7C154E2
:10F74000D1090FB6F894DEBF0FBECDBF6C01AB017F
:10F7500030E020E060E4CE0101967C010E9495DB60
:10F76000F70101900020E9F731978F010E191F0969
:10F77000A801B701C6010F94772C892B11F010E076
:10F7800000E0C801CF5BDF4F0FB6F894DEBF0FBEBD
:10F79000CDBFDF91CF911F910F91FF90EF90DF9040
:10F7A000CF9008950F931F93CF93DF938C01D0E0F8
:10F7B000C0E001151105B1F0BE0160517E4DC801D8
:10F7C0000F945920892B51F4FE01EC50FE4D849189
:10F7D00090E0DF91CF911F910F9108952596C2334C
:10F7E000D10539F781E090E0F4CF2F923F924F920C
:10F7F0005F926F927F928F929F92AF92BF92CF92C1
:10F80000DF92EF92FF920F931F93CF93DF93CDB7C9
:10F81000DEB7CD56D1090FB6F894DEBF0FBECDBF0F
:10F82000A7969FAF8EAFA7972A01AA962FAFAA9748
:10F83000AC961FAF0EAFAC97DC2CA596BFAEAEAEAC
:10F84000A597DC011496ED91FC910288F389E02DD7
:10F8500066807780AB2839F4FE01EE59FF4FA596FC
:10F86000FFAFEEAFA59781E0A596AEADBFADA59772
:10F870008C934B01B12CA12C6114710409F4B2C416
:10F88000AA96BFADAA97B13009F49DC008F493C001
:10F89000B23041F0B33009F48BC0D30112966D90B1
:10F8A0007C90EACF63E978E0C3010E940EF8CC2493
:10F8B000C394009791F3FC0181859285A385B4855B
:10F8C00088159905AA05BB0541F767ED77E0C301E7
:10F8D0000E940EF8A9969FAF8EAFA997A796AEADDE
:10F8E000BFADA7971296ED91FC9162E08281938162
:10F8F0000E94C0F84C01BFE30FEF1FEFB41540F0BA
:10F90000F201FF27EE0FFF1FE452F14F0781108530
:10F91000A2961FAEA2976D961CAE1DAE1EAE1FAE78
:10F920006D97A1961CAE1DAE1EAE1FAEA1976B9635
:10F930008FAD6B978F706B968FAF6B9763EA78E0A4
:10F94000C3010E940EF81C0166E576E0C3010E9427
:10F950000EF85C012114310451F0F10180858F70A3
:10F96000843029F4818592850E94D27BC82E2C2D6B
:10F970000C2C000C330BAE963FAF2EAFAE97EFEFD3
:10F98000EC0DEB3008F0B6C10E2E000CFF0B8827F3
:10F99000E353F3488F4F0D94EA27E67CB17D8E7DCB
:10F9A000D77D7A7E7A7E037EEF7D187E2F7E4D7E18
:10F9B00067E978E079CF6AE978E0C3010E940EF840
:10F9C0004BE0C42E76CF6FE978E0F7CF1801512CC9
:10F9D000412CA801110F660B770BCE01875A9F4F60
:10F9E0000E94671D62962FAF629763963FAF639741
:10F9F00064964FAF649765965FAF659766966FAFF5
:10FA0000669767967FAF679768968FAF6897699696
:10FA10009FAF69976AED73E289ED90E10F94A612AA
:10FA200000E020E033E040E150E0BE016F5F7F4F37
:10FA3000CE01875A9F4F0E94B720BC0189ED90E10B
:10FA40000F94B0116EEC73E289ED90E10F94A61261
:10FA50004AE050E0AE966EAD7FADAE9789ED90E195
:10FA60000F9497116CEC73E289ED90E10F94A6125C
:10FA7000D3016D917C9189ED90E10F94B01189EDE6
:10FA800090E10F945510A114B10409F448C1F50197
:10FA900080858F708550823008F041C1B501CE015C
:10FAA000875A9F4F0E94F9236A962FAF6A976B96E9
:10FAB0003FAF6B976C964FAF6C976D965FAF6D973E
:10FAC0006E966FAF6E976F967FAF6F97A0968FAF62
:10FAD000A097A1969FAFA197211103C0307F09F491
:10FAE0000DC16DEB73E289ED90E10F94A61200E079
:10FAF00020E033E040E150E0BE016F5F7F4FCE0178
:10FB0000875A9F4F0E94B720BC0189ED90E10F9466
:10FB1000B01189ED90E10F94551001C11801512CDD
:10FB2000412CB201A801CE01875A9F4F0E943E1D71
:10FB30002A962FAF2A972B963FAF2B972C964FAF35
:10FB40002C972D965FAF2D972E966FAF2E972F96F1
:10FB50007FAF2F9760968FAF609761969FAF619749
:10FB600059CF1027012710271801512C412CB20121
:10FB7000A101CE01875A9F4F0E94671D22962FAF89
:10FB8000229723963FAF239724964FAF249725962D
:10FB90005FAF259726966FAF269727967FAF27975B
:10FBA00028968FAF289729969FAF299733CF102794
:10FBB000012710271801512C412CB201A101CE01BF
:10FBC000875A9F4F0E943E1D29AF3AAF4BAF5CAFA3
:10FBD0006DAF7EAF8FAF21969FAF21971BCF1127BF
:10FBE0001801512C412CB201A801CE01875A9F4F18
:10FBF0000E943E1D29AB3AAB4BAB5CAB6DAB7EAB11
:10FC00008FAB98AF07CF012F11271801512C412C32
:10FC1000B201A801CE01875A9F4F0E943E1D29A71D
:10FC20003AA74BA75CA76DA77EA78FA798ABF2CE8C
:10FC30001801512C412C6B968FAD6B978F7080669D
:10FC40006B968FAF6B972AE030E0D8010F940128B4
:10FC5000A1966CAF7DAF8EAF9FAFA197DBCE1801A1
:10FC6000512C412C6B968FAD6B978F7080676B9684
:10FC70008FAF6B97B801110F880B990B0F9430263B
:10FC800020E030E048EC52E40F948928A1966CAF54
:10FC90007DAF8EAF9FAFA197BDCEF20194E0F695F8
:10FCA000E7959A95E1F74FEF5FEFE03438F4FF27DF
:10FCB000EE0FFF1FE452F14F478150853FE0432292
:10FCC000552402C0569547954A94E2F7417055274E
:10FCD0001A01512C412CB201CE01875A9F4F0E942C
:10FCE0003E1D29A33AA34BA35CA36DA37EA38FA3C0
:10FCF00098A790CE212C312C21018CCE68EA78E097
:10FD0000C5010E940EF88C01009749F0DC0118969D
:10FD10008C918F70823029F0843009F4DAC010E0C1
:10FD20005DC06EEA73E289ED90E10F94A612F801CE
:10FD300041855285638574852AE030E089ED90E144
:10FD40000F944F1189ED90E10F945510D801199639
:10FD50006D917D918D919C911C97AC96EEADFFAD10
:10FD6000AC978F0130E020E060177107820793079E
:10FD70000CF4A6C0870130E020E00617170728071B
:10FD800039070CF49DC0AB014E1B5F0B9E012F5930
:10FD90003F4F5901C12C8F01AA962FADAA97A79664
:10FDA0008EAD9FADA7970E94F57B6A962FAF6A979D
:10FDB0006B963FAF6B976C964FAF6C976D965FAF3E
:10FDC0006D976E966FAF6E976F967FAF6F97A09699
:10FDD0008FAFA097A1969FAFA19711E0DD2039F0DA
:10FDE000A996EEADFFADA997EF2B09F03DC28114A6
:10FDF0009104D1F1F40180858F708630A9F5D3018B
:10FE00006D917C91C4010E940EF84C01009761F144
:10FE1000FC0180858F70F82C092D853011F4F68057
:10FE200007816EE176E08F2D902F0E940EF8FC0185
:10FE3000892B09F482C19085892F8F70823009F057
:10FE400044C1418552856385748542155305640517
:10FE5000750509F033C1A596AEADBFADA5971C924F
:10FE6000112311F0D11083C188E0FE01E75AFF4F42
:10FE7000DE01519601900D928A95E1F729893A8920
:10FE80004B895C896D897E898F89988DC359DF4F35
:10FE90000FB6F894DEBF0FBECDBFDF91CF911F919B
:10FEA0000F91FF90EF90DF90CF90BF90AF909F9019
:10FEB0008F907F906F905F904F903F902F9008951C
:10FEC0006CE973E284E390E10F94A61284E390E17D
:10FED00022CE6CE873E289ED90E10F94A612D8016E
:10FEE00019966D917C9189ED90E10F94B01189ED97
:10FEF00090E10F9455108114910409F4AAC1F40102
:10FF000080858F70863009F0D5C1D80119966D9122
:10FF10007C91C4010E940EF8009709F4CBC16EE1F8
:10FF200076E00E940EF87C01009709F4C3C1FC0141
:10FF300080858F70823009F0BDC16AE773E289ED78
:10FF400090E10F94A612D70119964D915D916D9194
:10FF50007C911C972AE030E089ED90E10F944F11DD
:10FF600089ED90E10F945510F80161857285A7968F
:10FF7000AEADBFADA7971496ED91FC9182899389A0
:10FF80000E940EF88C01009709F494C163EA78E0AE
:10FF90000E940EF8009749F0FC0120852F70243054
:10FFA00021F4818592850E94D27BD70119964D91CB
:10FFB0005D916D917C911C97CE01875A9F4F0E9455
:10FFC000671D298F3A8F4B8F5C8F6D8F7E8F8F8F40
:10FFD00098A366E576E0C8010E940EF8BC01009780
:10FFE00019F1FC0190859F7095509230E8F4CE0194
:10FFF000875A9F4F0E94F9236A962FAF6A976B9694
:020000021000EC
:100000003FAF6B976C964FAF6C976D965FAF6D97E8
:100010006E966FAF6E976F967FAF6F97A0968FAF0C
:10002000A097A1969FAFA19765E673E289ED90E155
:100030000F94A61200E020E033E040E150E0BE0162
:100040006F5F7F4FCE01875A9F4F0E94B720BC0140
:1000500089ED90E10F94B01189ED90E10F94551066
:10006000D70118968C911897982F92959F7090FDB4
:1000700021C121E0A2962FAFA29791609295907F27
:100080008F70892B18968C9311E0DD2009F4B2CE85
:10009000A9962EAD3FADA997232B09F4ABCEE4C0B2
:1000A000A796EEADFFADA7976281738140E051E066
:1000B000CE01875A9F4F0E943B3099CE21863286CF
:1000C00043865486907E926090871111CBCEA59680
:1000D000EEADFFADA5978081882309F4C5CE6CEA0B
:1000E00078E08F2D902F0E940EF83C01009709F4C4
:1000F00088C0DC0118968C9118978F70823009F0B7
:1001000064C019968D919D910D90BC91A02D821582
:100110009305A405B50509F058C06FE273E289EDB7
:1001200090E10F94A61289ED90E10F945510A596D9
:10013000EEADFFADA597108297CE66E573E289ED2F
:1001400090E10F94A612F3016081718189ED90E135
:100150000F94B01189ED90E10F945510A201910117
:100160006EE176E08F2D902F0E94DDFBAECFA29640
:100170008FADA297811108C0A596AEADBFADA59772
:100180008C91882309F470CEB12CA12CD12CC12CD8
:100190006A96EFAC6A976B96FFAC6B976C960FAD57
:1001A0006C976D961FAD6D976E962FAD6E976F968F
:1001B0003FAD6F97A0964FADA097A1965FADA19769
:1001C0006FEFC4010E9423E04FCED1101DC0D401B7
:1001D00018968C9187FD48CEF3012186328643869E
:1001E000548642CE19821A821B821C828A818F70A9
:1001F0008A831D821E821F82188688E0FE01319646
:1002000037CEDD2009F430CEB12CA12CD12CC12C5D
:100210006A96EFAC6A976B96FFAC6B976C960FADD6
:100220006C976D961FAD6D976E962FAD6E976F960E
:100230003FAD6F97A0964FADA097A1965FADA197E8
:100240006FEFC4010E9423E06114710409F0BFCF75
:100250000BCEDD2009F408CEA996EEADFFADA9972F
:1002600010E0EF2B09F400CEA996AEADBFADA99773
:1002700018968C9118978F70823009F0B8CD199626
:100280008D919D910D90BC91A02D81309105A1057E
:10029000B10509F405CF0297A105B10509F0A7CD75
:1002A000A796AEADBFADA79712966D917C9140E039
:1002B00052E0FECE10E0E9CE2F923F924F925F9235
:1002C0006F927F928F929F92AF92BF92CF92DF9266
:1002D000EF92FF920F931F93CF93DF93CDB7DEB7CB
:1002E00068970FB6F894DEBF0FBECDBF61157105DC
:1002F00009F489C05E8B498B9D8B8C8BFB018680BA
:1003000097808114910409F47EC0F40180858F7078
:10031000823031F0853031F1F40182809380F1CF69
:100320006184728441E050E069897E89C3010E9442
:100330007966882389F3B12CA12CCC24C394730152
:100340008301298950E040E0B3018C899D890E9496
:10035000F57B29873A874B875C876D877E878F87F8
:10036000988BDACFC4010E9452F98230A9F660E07E
:10037000C4010E94C0F8FC01C184D284E384F484E7
:1003800061E0C4010E94C0F8FC01218432844384EE
:100390005484388E2F8ADB8ACA8AA1014C195D09E0
:1003A0004F5F5F4F69897E89C6010E947966882305
:1003B00009F4B2CF89ED90E10F945510712C612CA6
:1003C0006A897B89660D771D8F89988D86179707B7
:1003D0000CF4A2CFB12CA12CCC24C39471010A89B6
:1003E0001B892989A3018C899D890E94F57B29831A
:1003F0003A834B835C836D837E838F8398879FEFE3
:10040000691A790ADDCF68960FB6F894DEBF0FBE81
:10041000CDBFDF91CF911F910F91FF90EF90DF90B3
:10042000CF90BF90AF909F908F907F906F905F9094
:100430004F903F902F900895089508958F929F9226
:10044000AF92BF92CF92DF92EF92FF920F931F93E2
:10045000CF93DF9300D000D0CDB7DEB72091D70C7B
:100460003091D80C232B09F484C02091D60C211193
:1004700080C04C018091D60C8F5F8093D60C809108
:10048000D50C8F5F8093D50C0F9446049B01AC0173
:100490006091A40B7091A50B8091A60B9091A70B76
:1004A000A12CB12C65011BE0E12EF12C00E010E045
:1004B0000E94B8D5882309F452C0E091D70CF0917E
:1004C000D80C0681178101151105B9F1F801808555
:1004D0008F70863071F56AE576E0C8010E940EF8EB
:1004E0000097D1F0FC0120852F702530A9F4E6801B
:1004F000F780E114F104E9F0FA82E982B801CE0153
:1005000001960E94BB38B401CE0101960E94E759C2
:10051000F701E280F380EDCF1A83098370E060E099
:10052000CE0101960E94BB38B401CE0101960E9413
:10053000E759F80102811381C6CFF3E08F169104C9
:1005400051F00F9446046093A40B7093A50B809315
:10055000A60B9093A70B1092E7101092E8108091D1
:10056000D50C81508093D50C8091D60C815080930E
:10057000D60C26960FB6F894DEBF0FBECDBFDF9126
:10058000CF911F910F91FF90EF90DF90CF90BF9090
:10059000AF909F908F900895A89582E090E00C9482
:1005A0001E828091C40B8F5F8093C40BA89583E05B
:1005B00090E00E941E820E9478BE8091C40B815000
:1005C0008093C40B08956AEF7EE18CE290E10F9472
:1005D000A61267EE7EE18CE290E10F94A61269ED1F
:1005E0007EE18CE290E10F94A61261ED7EE18CE257
:1005F00090E10F94A6128CE290E10F94551061ECFB
:100600007EE18CE290E10F94A61265EB7EE18CE234
:1006100090E10F94A6126DE87EE18CE290E10F94D8
:10062000A6126DE77EE18CE290E10F94A61260E7DE
:100630007EE18CE290E10F94A6126BE57EE18CE204
:1006400090E10F94A6126CE47EE18CE290E10F94AD
:10065000A61264E47EE18CE290E10F94A61263E3BB
:100660007EE18CE290E10F94A6126DE07EE18CE2D7
:1006700090E10F94A61260E07EE18CE290E10F948D
:10068000A61266EF7DE18CE290E10F94A61267EE70
:100690007DE18CE290E10F94A6126FED7DE18CE29A
:1006A00090E10F94A61263ED7DE18CE290E10F944E
:1006B000A61269EB7DE18CE290E10F94A6126AE943
:1006C0007DE18CE290E10F94A61265E87DE18CE279
:1006D00090E10F94A6126DE67DE18CE290E10F941B
:1006E000A6126FE57DE18CE290E10F94A61263E51E
:1006F0007DE18CE290E10F94A6126BE47DE18CE247
:1007000090E10F94A61260E47DE18CE290E10F94F9
:10071000A61263E37DE18CE290E10F94A6126BE2F6
:100720007DE18CE290E10F94A61260E27DE18CE223
:1007300090E10F94A61261E17DE18CE290E10F94CB
:10074000A61268E07DE18CE290E10F94A6126AEFB8
:100750007CE18CE290E10F94A6126CEE7CE18CE2DD
:1007600090E10F94A6128CE290E10D9455100F9336
:100770001F93CF93DF9300D000D0CDB7DEB70E9498
:10078000E38260E376E18CE290E10F94A612CE0161
:1007900001960E941AFECE0101960E9429DC0DE806
:1007A00015E01A8309838091890E90918A0EA09199
:1007B0008B0EB0918C0E8B839C83AD83BE83CE0158
:1007C00001960E9429DC1A8309831B821C821D82E8
:1007D0001E8280E590E00E9407FE44E050E0BE01EA
:1007E0006D5F7F4F81E090E00E9437C20E942EC370
:1007F000CE0101960E9429DC1A8309831B821C8288
:100800001D821E8280E590E00E9407FE44E050E0D9
:10081000BE016D5F7F4F85E090E00E9437C20E946D
:100820002EC3CE0101960E9429DC66E576E18CE2BA
:1008300090E10F94A61288EC90E026960FB6F894FB
:10084000DEBF0FBECDBFDF91CF911F910F910895F5
:10085000CF92DF92EF92FF921F93CF93DF9300D05E
:1008600000D0CDB7DEB76BE872E18CE290E10F9477
:10087000A61280E1E82E80E1F82E10E090E1C92E6A
:10088000D12CF70181917F01803130F469EB76E062
:100890008CE290E10F94B011153041F1F7013197DE
:1008A000808190E0B0E0A0E089839A83AB83BC8331
:1008B000DE82CD82BE016F5F7F4F8CE290E10E94AD
:1008C000A03469E872E10F94A6121F5F1630C9F6D2
:1008D00026960FB6F894DEBF0FBECDBFDF91CF9145
:1008E0001F91FF90EF90DF90CF90089580911510A9
:1008F00090E0B0E0A0E089839A83AB83BC83DE8282
:10090000CD82BE016F5F7F4F8CE290E10E94A034E8
:100910000F945510DACFEF92FF920F931F93CF935E
:10092000DF9300D000D01F92CDB7DEB77B01CE01A0
:1009300007969F938F9301979F938F9301979F9310
:100940008F9301979F938F9301979F938F93019715
:100950009F938F938E010F5F1F4F1F930F938FEA0B
:1009600098E09F938F93DB0113968C9113978F934D
:1009700012968C918F930F940C2D0FB6F894DEBFC6
:100980000FBECDBF0697ECF466E57BE184E390E112
:100990000F94A612D70112966D917C9184E390E199
:1009A0000F94B01180E991E027960FB6F894DEBF5E
:1009B0000FBECDBFDF91CF911F910F91FF90EF90B0
:1009C00008958091081090910910892B09F449C06D
:1009D0000E9462F9882309F444C0A0910810B091E4
:1009E000091052961C921E92519754961C921E9278
:1009F000539784E890E01D969C938E931C971E96C7
:100A00001C921E9782E755968C935597ED91FC9119
:100A100011970088F189E02D64E070E0CD0119950F
:100A20008091081090910910DC01ED91FC910280F9
:100A3000F381E02D46E050E0B801199586E0F80119
:100A4000A0E1B0E101900D928A95E1F78091081044
:100A500090910910DC01ED91FC910488F589E02D5D
:100A600019950E94288468E67BE18CE290E10F945E
:100A7000A61288EC90E098CFFF920F931F93CF932C
:100A8000DF9300D000D0CDB7DEB78C01BC01CE0122
:100A900001960F94670DBE016F5F7F4F89ED90E166
:100AA0000F94981289ED90E10F945510CE010196A4
:100AB0000F945F0D1A8219821C821B821E821D8276
:100AC0006BEC7BE1CE0101960F94020DF8012481BD
:100AD00035818D819E81F12C2817390738F0BE01B0
:100AE0006F5F7F4FC8010E940EFFF82ECE01019666
:100AF0000F945F0DFF2069F0B801CE0101960F94AD
:100B0000670DCE0101960F94CA12CE0101960F9483
:100B10005F0D26960FB6F894DEBF0FBECDBFDF91F6
:100B2000CF911F910F91FF9008950F931F93CF9333
:100B3000DF9300D000D0CDB7DEB7A0910810B09100
:100B40000910109709F478C052961C921E92519782
:100B500054961C921E92539784E890E01D969C93A5
:100B60008E931C971E961C921E9787E755968C9322
:100B70005597ED91FC9111970088F189E02D70E077
:100B800060E0CD01199510E000E08091081090918F
:100B90000910DC01ED91FC9111971C962D913C916F
:100BA0000217130740F40190F081E02D60E01995E1
:100BB0000F5F1F4FEACF0088F189E02D70E060E001
:100BC000199504E015E08091081090910910F80142
:100BD00061918F01DC01ED91FC910190F081E02D9C
:100BE0001995B5E008301B0771F7809108109091B6
:100BF0000910DC01ED91FC910488F589E02D19952F
:100C000063EA79E0CE0101960F94700DCE01019652
:100C10000F94CA12CE0101960F945F0D87E090E009
:100C20000F94E20F87E090E00F94EC0F69E17BE115
:100C30008CE290E10F94A6121092281010922710C7
:100C400080E090E1909323108093221084E890E05C
:100C500090932A108093291081E08093241082E7DA
:100C600080932B1086E190E10E941B1786E190E1B2
:100C70000E94931788EC90E026960FB6F894DEBF9A
:100C80000FBECDBFDF91CF911F910F910895AF920D
:100C9000BF92CF92DF92EF92FF920F931F93CF9369
:100CA000DF93CDB7DEB76D970FB6F894DEBF0FBEFA
:100CB000CDBF0F9446049B01AC016091B00B7091C5
:100CC000B10B8091B20B9091B30BA12CB12C6501AB
:100CD00018EEE12E13E0F12E00E010E00E94B8D5EE
:100CE000F82E882351F00F9446046093B00B709354
:100CF000B10B8093B20B9093B30B8091D50C8F5FA7
:100D00008093D50CE091DB0CF091DC0C068117810F
:100D100094E0C92ED12CF11003C082E0C82ED12C52
:100D2000A090DB0CB090DC0CA114B10429F10115EA
:100D3000110511F1F80180858F708530A9F7C80180
:100D40000E9452F9823080F3B801CE0101960E94D0
:100D50008A34CE0101960E942D28882329F0B601FD
:100D6000CE0101960E941E53F80102811381CE012B
:100D700001960E947C34D4CF8091D50C8150809311
:100D8000D50C8091D90C9091DA0C0597D9F1FF2000
:100D9000C9F110E060912C0B70912D0B611571055C
:100DA00089F111112FC0FB0180858F70853091F47E
:100DB000CE0101960E948A3461E070E0CE01019676
:100DC0000E941E5311E0892B09F410E0CE01019618
:100DD0000E947C34E0912C0BF0912D0B309791F018
:100DE0008281938190932D0B80932C0B892B91F60C
:100DF000E091DB0CF091DC0C8681978190932D0BB8
:100E000080932C0B6D960FB6F894DEBF0FBECDBF4E
:100E1000DF91CF911F910F91FF90EF90DF90CF90D6
:100E2000BF90AF9008952F923F924F925F926F9232
:100E30007F928F929F92AF92BF92CF92DF92EF926A
:100E4000FF920F931F93CF93DF93CDB7DEB7C955B2
:100E5000D1090FB6F894DEBF0FBECDBF0F94460484
:100E60009B01AC016091AC0B7091AD0B8091AE0B0E
:100E70009091AF0BA12CB12C650110E3E12E15E789
:100E8000F12E00E010E00E94B8D5882309F42EC2AC
:100E9000E091DB0CF091DC0C309709F427C28091D3
:100EA000D50C8F5F8093D50C2680378010E02114FD
:100EB000310409F43AC1F10180858F708530F9F46D
:100EC00060E0C1010E94C0F8FC0181859285A38584
:100ED000B4850597A105B10591F4B101CE01019644
:100EE0000E948A34CE0101960E942D2866968FAF0B
:100EF0006697811108C0CE0101960E947C34F101F1
:100F000022803380D4CF25961CAE1DAE1EAE1FAE00
:100F1000259729961CAE1DAE1EAE1FAE299740E048
:100F200052E0BE016F5F7F4FCE018F5B9F4F0E94EB
:100F3000FA30CE0101960E94D6286B017C01699699
:100F40006FAF69976A96DFAE6A9770E060E0CE0196
:100F500001960E9438294C01CE018F5B9F4F0E9461
:100F60000A1F65966CAF7DAF8EAF9FAF6597CE01C0
:100F700001960E94ED30182FB601DD0C880B990BFD
:100F80000F94302620E030E048EC52E40F9489289A
:100F90002B013C01CE0101960E94E55168969FAF5E
:100FA0008EAF689766EA7FE189ED90E10F94A61213
:100FB00065964CAD5DAD6EAD7FAD659789ED90E109
:100FC0000F947E1060EA7FE189ED90E10F94A61204
:100FD000B301A20189ED90E10F947E106AE97FE1EF
:100FE00089ED90E10F94A612612F70E04AE050E085
:100FF00089ED90E10F949711E114F10409F48EC08A
:1010000088E00E946DD69B01AC0144275527B701AB
:1010100090E080E0AA24AA94BA2CC12CD12C17E22B
:10102000E12E19E0F12E00E010E00E94B8D58823EF
:1010300071F1F1016081718184E390E10F94B0114D
:101040006AE87FE184E390E10F94A612F1016081E8
:10105000718183EC98E00F94FE0490E080E0BC0185
:1010600069964FAD69976A965FAD6A97CE01019612
:101070000E947C2862E070E0C4010E944F74CE019F
:1010800001960E947C3466961FAD669738CF20E0AB
:1010900030E048E152E4C301B2010F94312918163F
:1010A0003CF4F1016081718189E496E00F94FE04C3
:1010B00068968EAD9FAD6897892B19F461E070E05A
:1010C000DBCF20E030E040E85FE365966CAD7DADBE
:1010D0008EAD9FAD65970F941C289B01AC01C30199
:1010E000B2010F94292670E060E087FDC5CFA3010F
:1010F000920165966CAD7DAD8EAD9FAD65970F94F9
:1011000029261816DCF66BE77FE189ED90E10F9454
:10111000A61289ED90E10F945510B1CF61E77FE100
:1011200089ED90E10F94A612AACF8091D50C815041
:101130008093D50C0F9446046093AC0B7093AD0B69
:101140008093AE0B9093AF0B0E9416DD2B013C01F8
:101150000F9446046B017C010E942CF8882309F44B
:1011600089C08091C40B811185C030E020E041E04E
:1011700050E060E4CE0101960E9495DB4FE350E021
:101180006AE47FE1CE0101960F94722061E479E078
:10119000CE0101960F94412C4FE350E061E47FE1D2
:1011A000CE0101960F9472202AE0AE014F5B5F4F93
:1011B000C301B2010F94F220BE016F5B7F4FCE01DD
:1011C00001960F94E30430E020E041E050E060E459
:1011D000CE0101960E9495DB4FE350E06AE47FE187
:1011E000CE0101960F94722061E479E0CE01019660
:1011F0000F94412C4FE350E06AE37FE1CE0101966A
:101200000F947220C701B60128EE33E040E050E0B1
:101210000F947327CA01B9012AE0AE014F5B5F4FFB
:101220000F94F220BE016F5B7F4FCE0101960F94A9
:10123000E30430E020E041E050E060E4CE010196BC
:101240000E9495DB4FE350E063E37FE1CE0101961E
:101250000F9472204FE050E06DE27FE1CE018F5B92
:101260009F4F0F949020BE016F5B7F4FCE01019680
:101270000F94E304112309F453C06BE67FE189ED79
:1012800090E10F94A6120E9416DDAB01BC012AE08A
:1012900030E089ED90E10F94531063E67FE189ED32
:1012A00090E10F94A6126091D50C062E000C770BDE
:1012B0004AE050E089ED90E10F94971161E57FE1FC
:1012C00089ED90E10F94A6124091A80B5091A90BC3
:1012D0006091AA0B7091AB0B2AE030E089ED90E1B0
:1012E0000F94531089ED90E10F945510C75ADF4FBA
:1012F0000FB6F894DEBF0FBECDBFDF91CF911F9127
:101300000F91FF90EF90DF90CF90BF90AF909F90A4
:101310008F907F906F905F904F903F902F900895A7
:1013200061E67FE189ED90E10F94A6120E9416DD3F
:10133000AB01BC012AE030E089ED90E10F9453103D
:1013400069E57FE1ACCF6F927F928F929F92AF92CF
:10135000BF92CF92DF92EF92FF920F931F93CF93A2
:10136000DF93CDB7DEB7A5970FB6F894DEBF0FBEFB
:10137000CDBF80912E0B90912F0B892B09F414C6B1
:101380008091D50C811110C68091D50C8F5F809310
:10139000D50C68EB7AE18CE290E10F94A6128CE216
:1013A00090E10F94551000912E0B10912F0B6FECC4
:1013B00078E0C8010E940EF89093DC0C8093DB0C5F
:1013C00065ED78E0C8010E940EF89093C30B8093FE
:1013D000C20B68E776E0C8010E940EF89093D80C23
:1013E0008093D70C6CED78E0C8010E940EF89093C2
:1013F000290B8093280B61EE78E0C8010E940EF85B
:101400009093270B8093260B009709F4B3C00E949A
:1014100052F9082F10E00115110509F4ABC0000FB7
:10142000111F000F111F8091240B9091250B892B08
:1014300009F08FC0C8010F941D1D9093250B809358
:10144000240B1092D50B1092D40B1092A30B109278
:10145000A20B1092D30B1092D70B1092D60B7801DF
:10146000013022E012071CF0E12C42E0F42EC7010B
:1014700001960F941D1D9093D90B8093D80B9093D8
:10148000D20B8093D10B8E0D9F1D9093CC0B80932C
:10149000CB0B0F9446046093CD0B7093CE0B8093CF
:1014A000CF0B9093D00B90E080E0E091D80BF091BF
:1014B000D90BE80FF91F10820196E816F906ACF770
:1014C00082E090E09093D50B8093D40B8091A20B97
:1014D0009091A30B009741F061E00F94010060E050
:1014E0008091A20B0E94D3FF80E98093C9001092E3
:1014F000C8001092CD0083E08093CC008EE08093F2
:10150000CA00F0922F02E0922E022091D80B309167
:10151000D90B80912E0290912F02820F931F9093EE
:10152000CC0B8093CB0B232B09F462C068E47AE1E7
:1015300089ED90E10F94A6124AE050E0B80189EDE0
:1015400090E10F949E118AE29AE19093CA0B8093E6
:10155000C90B6EE97AE18CE290E10F94A6124AE0A1
:1015600050E0B8018CE290E10F9497118CE290E189
:101570000F94551067EE78E080912E0B90912F0B11
:101580000E940EF88C01009709F472C00E9452F973
:10159000882309F46DC06FEF680FC8010E94C0F87E
:1015A000DC011996ED90FC909091C70B992359F0AE
:1015B000809170008E7F809370001092C70B109204
:1015C0002A021092290282E18093280291110E943E
:1015D0005DD0C7010E9485D001E010E0E016F10661
:1015E00074F060E0C8010E94B9D00F5F1F4FF6CFC2
:1015F00061E37AE189ED90E10F945817A4CF63E29B
:101600007AE189ED90E10F94A6120E9416DDAB01FC
:10161000BC012AE030E089ED90E10F94531089ED90
:1016200090E10F94551062E87AE18CE290E10F941A
:10163000A6124AE050E0B7018CE290E10F949711B6
:101640008CE290E10F9455106CE77AE189ED90E11E
:101650000F94A6120E9416DDAB01BC012AE030E017
:1016600089ED90E10F94531089ED90E10F9455109E
:1016700000912E0B10912F0B6BEE78E0C8010E94A9
:101680000EF89093320B8093310B62EF78E0C80133
:101690000E940EF89093DE0C8093DD0C892BA1F054
:1016A0008091DF0C811110C08091C50B9091C60B09
:1016B000892B09F47CC081E08093DF0C6CE67AE131
:1016C0008CE290E10F94A61210922D0B10922C0B2D
:1016D000E091DB0CF091DC0C309709F415C3C68067
:1016E000D7800091DB0C1091DC0C0115110509F479
:1016F00004C3C114D10409F400C3F60180858F70BE
:10170000853099F7C6010E9452F9823070F3B60114
:10171000CE0101960E948A34CE0101960E942D28A6
:101720008823E1F18A859B85009709F457C2DC0183
:10173000ED91FC910484F585E02D1995892B49F0F4
:101740008A859B85DC01ED91FC910284F385E02D77
:1017500019958A859B85DC01ED91FC910680F781C6
:10176000E02D1995892BD1F0CE0101960E94ED3024
:10177000882341F040E051E060E070E0CE01019646
:101780000E94762B8D819E81892B41F040E052E0B2
:1017900060E070E0CE0101960E94762BD601129691
:1017A000CD90DC90CE0101960E947C349ACF62E00D
:1017B0007AE189ED90E10F94A61289ED90E10F9402
:1017C00055106CEF79E189ED90E10F94A6120E941B
:1017D00016DDAB01BC012AE030E089ED90E10F9409
:1017E000531089ED90E10F9455108FE090E00F9425
:1017F0001D1D8C0188E1F8018183128210821686FA
:1018000015860E948AFC1093C60B0093C50B012B12
:1018100069F46DEE79E184E390E10F94A61284E31C
:1018200090E10F9455101092DF0C4ECF0E948AFC6D
:101830008091C50B9091C60B0E948FD2882309F42A
:1018400099C065ED79E18CE290E10F945817809191
:10185000C50B9091C60B0E942ED4E091C50BF09160
:10186000C60B81E0808365EB79E189ED90E10F940F
:1018700058178091C50B9091C60B0E943CD469EA21
:1018800079E1811102C065E979E189ED90E10F9478
:1018900058178091DD0C9091DE0C892B21F28091FC
:1018A000BE0B9091BF0B892B09F0EAC083E190E059
:1018B0000F941D1D8C018091C50B9091C60B2BE1DF
:1018C0003DEAD80152963C932E93519716969C93DD
:1018D0008E93159714961C9214971C9289E011967A
:1018E0008C93119781E012968C93129713968C9398
:1018F0001093BF0B0093BE0B0F9446046B017C0149
:10190000B0E1CB0EB7E2DB1EE11CF11CD80115964D
:10191000ED91FC9116978FEF8387148613821482C2
:1019200015821682178210861186128614961C92D2
:10193000BB24B394BE01625E7F4FF801858196811E
:101940000E9416D518160CF096C00F9446046C151C
:101950007D058E059F0508F08EC0DE015E9698E03D
:1019600080E0915019F1ED91E827F0E0EC55F74D4A
:101970008491F7CF0E941AD68091C50B9091C60B27
:101980000E948FD2882359F068E779E18CE290E1D8
:101990000F94A6128CE290E10F9455107ACF6CE56B
:1019A00079E184E390E10F9458173DCF9DA19813FE
:1019B000C1CFD8018C91811138C015968D919C9121
:1019C0000E943CD4BE01625E7F4FF8018581968102
:1019D0000E940FD440E064EBD80115968D919C9144
:1019E0000E94E9D3F80185809680C4010E9475D3D6
:1019F000C4010E94E7D067E88FE89EE00E9441AEF4
:101A000060E88FE89EE00E9441AE0E947CFCC40129
:101A10000E9475D3A82ED80115968D919C910E9495
:101A20003CD4A5FC02C0F801B082AE014F5F5F4F0D
:101A3000BE01625E7F4FC8010E947DD4D80111961D
:101A4000AC908E8D803109F4C4C2BE01625E7F4FBE
:101A5000C8010E94ECD48A1508F0B4C0F801818155
:101A6000D80111968C93119714968C9114978F5FCF
:101A700014968C935FCFE091BE0BF091BF0B128256
:101A8000E091DD0CF091DE0CE680F7803FE7D32E8D
:101A90008091DD0C9091DE0C892B09F40CCEE114C1
:101AA000F10409F408CEBE01625E7F4FF701808128
:101AB00091810E94A2DE882309F4FDCD65E479E1DD
:101AC00089ED90E10F94A612D7016D917C9189ED7B
:101AD00090E10F94B01189ED90E10F9455100091B1
:101AE000BE0B1091BF0BAE014F5F5F4FBE01625E38
:101AF0007F4FC8010E94D2D4882309F45EC08E8D26
:101B0000803109F45AC0DD82F801858196810E94F6
:101B10003CD4BE01625E7F4FD80115968D919C9199
:101B20000E940FD440E06EE4F801858196810E9406
:101B3000E9D340E06B81D80115968D919C910E946C
:101B4000E9D340E06C81F801858196810E94E9D358
:101B50008E8D803141F040E06D81D80115968D91D8
:101B60009C910E94E9D3F801858196810E943CD422
:101B7000BE01625E7F4FD80115968D919C910E94A7
:101B80000FD4F801408168E4858196810E94E9D3F1
:101B900064E170E080E090E00F944602D8018C91FF
:101BA000882331F06AE070E080E090E00F94460214
:101BB000F801858196810E943CD4D7011296ED9060
:101BC000FC9066CF8E8D803111F48CE049CFBE0140
:101BD000625E7F4FC8010E94ECD442CF70E060E0AB
:101BE000CE0101960E9438298C01912C812C97FFFF
:101BF00006C011950195110988248394912CCE017A
:101C000001960E94ED30E82EF12C8985853091F007
